:020000040800F2
:10000000501700201903000805A7000815A50008CF
:1000100001A70008A908000859C900082B03000817
:100020000000000000000000000000002D03000898
:10003000F91900080000000001040008AD030008E1
:1000400035030008350300083503000835030008B0
:1000500035030008350300083503000835030008A0
:100060003503000835030008350300083503000890
:100070003503000835030008350300083503000880
:100080003503000835030008350300083503000870
:100090003503000835030008350300083503000860
:1000A0003503000835030008350300083503000850
:1000B0003503000835030008051A0008151A000862
:1000C000251A000835030008350300083503000829
:1000D0000000000035030008350300083503000860
:1000E00035030008350300084DAC0008350300084F
:1000F0003503000835030008350300083503000800
:1001000035030008350300083503000835030008EF
:1001100035030008350300083503000835030008DF
:100120003503000835030008A9C8000849C90008BC
:1001300035030008350300083503000835030008BF
:1001400035030008350300083503000835030008AF
:10015000350300083503000835030008350300089F
:10016000350300083503000835030008350300088F
:10017000350300083503000835030008350300087F
:10018000350300083503000835030008350300086F
:10019000350300083503000835030008350300085F
:1001A000350300083503000835030008350300084F
:1001B000350300083503000835030008350300083F
:1001C000350300083503000835030008350300082F
:1001D000350300083503000835030008350300081F
:1001E000350300083503000835030008350300080F
:1001F00035030008350300083503000835030008FF
:10020000350300083503000835030008000000002E
:10021000000000003503000800000000350300085E
:1002200035030008350300083503000835030008CE
:1002300035030008350300083503000835030008BE
:1002400035030008350300083503000800F002F804
:1002500000F052F814A696E8000CB244B344DA4514
:1002600001D100F049F8BAE80F000FA696E8300077
:10027000A5EB040504EB0607AAEB0704A7F10107A9
:100280004FEA15154FEA3414A4F10104AC4201D32E
:1002900000F032F813F0010F18BFFB1A43F001030E
:1002A00000F001F8DBE7184744DA000064DA0000E8
:1002B000103A24BF78C878C1FAD8520724BF30C892
:1002C00030C144BF04680C607047000070470000F4
:1002D0000023002400250026103A28BF78C1FBD84F
:1002E000520728BF30C148BF0B6070471FB50DF0E3
:1002F000BBFC1FBD10B510BD00F098FA1146FFF70A
:10030000F5FF0DF071FC00F0B6FA03B4FFF7F2FF51
:1003100003BC00F0B9FA00000A4880470A480047C9
:10032000FEE7FEE7FEE7FEE7FEE7FEE7FEE7FEE7A5
:10033000FEE7FEE7FEE7000004480549054A064BD4
:100340007047000015AB00084D0200085011002056
:1003500050170020501300205013002072B64FF0A9
:10036000E0201749C0F8081D1648016841F0010156
:10037000016015481249096801604FF0E0201349F7
:1003800041614FF0070101614FF00001C0F8181DF5
:100390004FF07F41C0F81C1D0D49C0F8201D70476B
:1003A000FFF7FEBF01B5BDE80140704701B500F0A1
:1003B00099F8BDE801407047FFF7FEBFFFF7FEBFA9
:1003C00000000008001000E0840300209F252600A4
:1003D0000000FF404FF000002E4A1060EFF3148041
:1003E00020F0040080F3148862B64FF080504FF084
:1003F000E021C1F8040DBFF34F8FBFF36F8FFEE70D
:100400002548264A4FF00003016891B10360EFF3DD
:10041000098C2CE9F00F1EF0100F01D12CED108A81
:100420001F4C4CF804EDC1F808C025680DB18D6172
:10043000236072B61168D1B1016062B64F68184C82
:100440008D6907F101074F602560D1F80CC08CF36E
:100450000B88D1F808C05CF804EB1EF0100F01D136
:10046000BCEC108ABCE8F00F8CF30988704772B6B8
:100470001168016009B962B6F9E74FF000674FF003
:10048000E028C8F8047D62B6D8E700BFB0EE400AA5
:1004900070470000FC020020EC020020F002002067
:1004A000E8080020026922F00702A2F144026FF07E
:1004B000430313604FF0000353609360D3601361F4
:1004C00053619361D361136253629362D362136386
:1004D00053634FF0FF339363D1634FF08073136422
:1004E000826070472249086800F101000860214BD2
:1004F0001A683AB1A2F101021A601AB91E4B4FF004
:10050000010018601D490868026822B11C4B4FF0B9
:1005100001021A6008E000F104001A4B1A689042C8
:1005200001D1194B18680860134B1A6812B91449A5
:100530000868C8B101B51249086808B10DF03EF865
:100540000D4B1A6872B10CF0ADFF1048016849B943
:100550000F4801680F4A13680F484FF080529942C4
:1005600000D00260BDE80140BFF34F8F704700002C
:1005700034040020E80800209803002090030020A5
:10058000940300202004002024040020FC0200200A
:10059000EC020020F002002004ED00E053EA020C1F
:1005A00000F069802DE9F04B4FF00006002B1FBFD3
:1005B000B3FA83F503FA05F424FA05F65E4012BF98
:1005C0001643B2FA82F502FA05F4C5F120051EBF02
:1005D00022FA05FC44EA0C04203556EA044C4FEAA2
:1005E000144418BF641C4FF000084FF000099042FB
:1005F00071EB030C39D3002919BFB1FA81F701FA65
:1006000007F6B0FA80F700FA07F6C7F120071EBF19
:1006100020FA07FC46EA0C062037B6FBF4FCA7EBF1
:100620000507103F07F01F0BCBF120062CFA06F64A
:100630000CFA0BFB44BFB3460026202FA4BF5E4636
:100640004FF0000B5BEA060C08BF4FF0010B19EBF3
:100650000B0948EB0608ABFB027C06FB02CC0BFB4C
:1006600003CCC01B71EB0C01C1E70B4602464146AF
:100670004846BDE8F08B13B5084318BF4FF0FF3074
:100680000146AFF30080BDE81C407047032A40F2EA
:10069000308010F0030C00F0158011F8013BBCF124
:1006A000020F624498BF11F801CB00F8013B38BF3C
:1006B00011F8013BA2F1040298BF00F801CB38BF4A
:1006C00000F8013B11F0030300F07980083AC0F014
:1006D000088051F8043B083A51F804CBA0E8081010
:1006E000F5E7121D5CBF51F8043B40F8043BAFF343
:1006F0000080D20724BF11F8013B11F801CB48BF9D
:1007000011F8012B24BF00F8013B00F801CB48BFD2
:1007100000F8012B704702F0FF0343EA032242EA8C
:10072000024200F002B84FF000020429C0F012802B
:1007300010F0030C00F01B80CCF1040CBCF1020F94
:1007400018BF00F8012BA8BF20F8022BA1EB0C0169
:1007500000F00DB85FEAC17C24BF00F8012B00F85F
:10076000012B48BF00F8012B70474FF0000200B585
:10077000134694469646203922BFA0E80C50A0E8C4
:100780000C50B1F12001BFF4F7AF090728BFA0E872
:100790000C5048BF0CC05DF804EB890028BF40F83E
:1007A000042B08BF704748BF20F8022B11F0804F80
:1007B00018BF00F8012B704770477047704710B59D
:1007C000203AC0F00B80B1E81850A0E81850B1E80A
:1007D0001850A0E81850203ABFF4F5AF5FEA027C49
:1007E00024BFB1E81850A0E8185044BF18C918C079
:1007F000BDE810405FEA827C24BF51F8043B40F81A
:10080000043B08BF7047D20728BF31F8023B48BFFE
:1008100011F8012B28BF20F8023B48BF00F8012B3C
:100820007047000000487047100000207546FFF731
:10083000F9FFAE4605006946534620F0070085469D
:1008400018B020B5FFF778FDBDE820404FF0000656
:100850004FF000074FF000084FF0000BAC46ACE83B
:10086000C009ACE8C009ACE8C009ACE8C00921F097
:1008700007018D46704710B50446AFF3008020464F
:10088000BDE81040FFF741BD01491820ABBEFEE7AF
:10089000260002007047000082B001900020009006
:1008A000009802B070470000FFE7FEE785B00490B3
:1008B0000498006A039004980068406920F443009B
:1008C00003990843049909684861049B1A695869A7
:1008D0009969DB6918431043084303900498016841
:1008E00001205022C4F202029142029000F067817E
:1008F000FFE70498016801205022C5F202029142EC
:10090000029000F05C81FFE7049801680120D0228A
:10091000C4F202029142029000F05181FFE7049874
:1009200001680120D022C5F202029142029000F03B
:100930004681FFE704980168012040F25012C4F29A
:1009400002029142029000F03A81FFE704980168A8
:10095000012040F25012C5F202029142029000F0D2
:100960002E81FFE704980168012040F2D012C4F202
:1009700002029142029000F02281FFE70498016890
:10098000012040F2D012C5F202029142029000F022
:100990001681FFE704980168012040F25022C4F25A
:1009A00002029142029000F00A81FFE70498016878
:1009B000012040F25022C5F202029142029000F062
:1009C000FE80FFE704980168012040F2D022C4F2C3
:1009D00002029142029000F0F280FFE70498016861
:1009E000012040F2D022C5F202029142029000F0B2
:1009F000E680FFE704980168012040F25032C4F21B
:100A000002029142029000F0DA80FFE70498016848
:100A1000012040F25032C5F202029142029000F0F1
:100A2000CE80FFE704980168012040F2D032C4F282
:100A300002029142029000F0C280FFE70498016830
:100A4000012040F2D032C5F202029142029000F041
:100A5000B680FFE704980168012041F25002C4F219
:100A600002029142029000F0AA80FFE70498016818
:100A7000012041F25002C5F202029142029000F0C0
:100A80009E80FFE704980168012041F2D002C4F281
:100A900002029142029000F09280FFE70498016800
:100AA000012041F2D002C5F202029142029000F010
:100AB0008680FFE704980168012041F25012C4F2D9
:100AC0000202914202907AD0FFE704980168012067
:100AD00041F25012C5F20202914202906FD0FFE73C
:100AE00004980168012041F2D012C4F2020291423E
:100AF000029064D0FFE704980168012041F2D0120F
:100B0000C5F202029142029059D0FFE704980168B1
:100B1000012041F25022C4F20202914202904ED0D2
:100B2000FFE704980168012041F25022C5F2020259
:100B30009142029043D0FFE704980168012041F2FE
:100B4000D022C4F202029142029038D0FFE704980A
:100B50000168012041F2D022C5F2020291420290C6
:100B60002DD0FFE704980168012041F25032C4F211
:100B700002029142029022D0FFE70498016801200E
:100B800041F25032C5F202029142029017D0FFE7C3
:100B900004980168012041F2D032C4F2020291426D
:100BA00002900CD0FFE7049800684EF63041CAF678
:100BB000FD710844B0FA80F040090290FFE7029806
:100BC000C007B8B1FFE70498426A836AC06A00218F
:100BD000CFF6F07101EB035101F07C7108436FF027
:100BE0000F0101EB021101F47C71014303980843EA
:100BF0000390FFE704980068006C00F080200399E0
:100C00000843049909680864049988680A791043BC
:100C1000096B084303900498C068B0F5806F40F0FA
:100C20007C81FFE70498016801205022C4F202028F
:100C30009142019000F06781FFE70498016801206C
:100C40005022C5F202029142019000F05C81FFE760
:100C5000049801680120D022C4F20202914201905E
:100C600000F05181FFE7049801680120D022C5F20D
:100C700002029142019000F04681FFE7049801686A
:100C8000012040F25012C4F202029142019000F0A1
:100C90003A81FFE704980168012040F25012C5F242
:100CA00002029142019000F02E81FFE70498016852
:100CB000012040F2D012C4F202029142019000F0F1
:100CC0002281FFE704980168012040F2D012C5F2AA
:100CD00002029142019000F01681FFE7049801683A
:100CE000012040F25022C4F202029142019000F031
:100CF0000A81FFE704980168012040F25022C5F202
:100D000002029142019000F0FE80FFE70498016822
:100D1000012040F2D022C4F202029142019000F080
:100D2000F280FFE704980168012040F2D022C5F26A
:100D300002029142019000F0E680FFE7049801680A
:100D4000012040F25032C4F202029142019000F0C0
:100D5000DA80FFE704980168012040F25032C5F2C2
:100D600002029142019000F0CE80FFE704980168F2
:100D7000012040F2D032C4F202029142019000F010
:100D8000C280FFE704980168012040F2D032C5F22A
:100D900002029142019000F0B680FFE704980168DA
:100DA000012041F25002C4F202029142019000F08F
:100DB000AA80FFE704980168012041F25002C5F2C1
:100DC00002029142019000F09E80FFE704980168C2
:100DD000012041F2D002C4F202029142019000F0DF
:100DE0009280FFE704980168012041F2D002C5F229
:100DF00002029142019000F08680FFE704980168AA
:100E0000012041F25012C4F20202914201907AD0C4
:100E1000FFE704980168012041F25012C5F2020276
:100E2000914201906FD0FFE704980168012041F2E0
:100E3000D012C4F202029142019064D0FFE70498FC
:100E40000168012041F2D012C5F2020291420190E4
:100E500059D0FFE704980168012041F25022C4F202
:100E60000202914201904ED0FFE7049801680120F0
:100E700041F25022C5F202029142019043D0FFE7B5
:100E800004980168012041F2D022C4F2020291428A
:100E9000019038D0FFE704980168012041F2D02288
:100EA000C5F20202914201902DD0FFE7049801683B
:100EB000012041F25032C4F202029142019022D04C
:100EC000FFE704980168012041F25032C5F20202A6
:100ED0009142019017D0FFE704980168012041F288
:100EE000D032C4F20202914201900CD0FFE7049884
:100EF00000684EF63041CAF6FD710844B0FA80F041
:100F000040090190FFE70198C00728B1FFE7039867
:100F100040F480600390FFE70CE00498C068B0F5EF
:100F2000007F05D1FFE7039840F40070039000E0D4
:100F3000FFE7FFE70498416B039808430390049888
:100F40000068406C42F20011C3F6C04108400399AA
:100F5000084304990968486404980168002088647B
:100F600004980168012040F25032C4F2020291421A
:100F700000904ED0FFE704980168012040F2503203
:100F8000C5F202029142009043D0FFE70498016845
:100F9000012040F2D032C4F202029142009038D0D7
:100FA000FFE704980168012040F2D032C5F2020246
:100FB000914200902DD0FFE704980168012041F292
:100FC0005032C4F202029142009022D0FFE704980E
:100FD0000168012041F25032C5F2020291420090B4
:100FE00017D0FFE704980168012041F2D032C4F223
:100FF0000202914200900CD0FFE7049800684EF680
:101000003041CAF6FD710844B0FA80F04009009002
:10101000FFE70098C00740B1FFE70498016800208F
:101020004865049909688865FFE70498016800200D
:10103000C86705B07047000083B002900191029B21
:101040001A6958699969D3F81CC040EA0C00DB6B37
:1010500018431043084301990860029800788006FD
:1010600000281BD5FFE702994A6A8B6AC86A896B18
:1010700008430021CFF6F07101EB035101F07C71C0
:1010800008436FF00F0101EB021101F47C7140EA9B
:1010900001020199086810430860FFE7029841685F
:1010A000006B40F2FF22114008430199486002980A
:1010B000C068B0F5806F0DD1FFE702980078800618
:1010C000002806D5FFE70199486840F48060486031
:1010D000FFE70DE00298C068B0F5007F06D1FFE79A
:1010E0000199486840F40070486000E0FFE7FFE7BE
:1010F0000298426B01994868104348600298406C1E
:1011000070B1FFE70299086C4A6C896C104301F0DA
:101110003F0140EA01420199486810434860FFE7F7
:101120000298B0F8680001998860029800788007FA
:10113000002859D5FFE70298C16C0020CFF6FF7058
:1011400000EB01400021C0F2FF7100EA01020199A9
:101150008868104388600298006DB0F1FF3F06DC9C
:10116000FFE70199886840F08050886005E00199A8
:10117000886820F080508860FFE70298406DB0F1E9
:10118000FF3F06DCFFE70199886840F00050886067
:1011900005E00199886820F000508860FFE7029818
:1011A000806DB0F1FF3F06DCFFE70199886840F0F1
:1011B0008040886005E00199886820F08040886060
:1011C000FFE70298C06DB0F1FF3F06DCFFE7019931
:1011D000886840F00040886005E00199886820F048
:1011E00000408860FFE7FFE70298006E0199C86041
:1011F0000298406E019908610298007880070028E3
:101200006AD5FFE70298006DB0F1FF3F0ADCFFE707
:101210000298006D4042009000986FF35F30019992
:10122000486106E00298006D6FF35F3001994861F4
:10123000FFE70298406DB0F1FF3F0FDCFFE7029837
:10124000406D4042009000990020C1F6FF7000EA16
:10125000014201994869104348610BE00298416DD1
:101260000020C1F6FF7000EA01420199486910436D
:101270004861FFE70298806DB0F1FF3F09DCFFE7AE
:101280000298806D40420090BDF80000019988618D
:1012900005E00298B0F8580001998861FFE70298CC
:1012A000C06DB0F1FF3F0BDCFFE70298C06D40421C
:1012B0000090009A0199886940EA0240886107E03D
:1012C0000298C26D0199886940EA02408861FFE78F
:1012D00001990020C86103E0019900204861FFE7FF
:1012E0000298006801990862029800788007002837
:1012F00006D5FFE70199086A40F4E060086205E05E
:101300000199086A40F4A0600862FFE703B07047E3
:1013100086B00490039102920498039908430299BD
:1013200008434FF6FF718843019000200090049815
:1013300018B1FFE7049800900EE0039818B1FFE79A
:101340000398009007E0029818B1FFE70298009018
:1013500000E0FFE7FFE7FFE70198BDF80210B0EB00
:10136000014F03D0FFE70120059002E00020059027
:10137000FFE7059806B0704785B00390029101928F
:1013800000200090039828B1FFE7039890F8200010
:10139000009012E0029828B1FFE7029890F8200030
:1013A000009009E0019828B1FFE7019890F820002B
:1013B000009000E0FFE7FFE7FFE7029858B1FFE782
:1013C0000098029991F82010884203D0FFE702208C
:1013D000049011E0FFE7019858B1FFE700980199E8
:1013E00091F82010884203D0FFE70320049003E027
:1013F000FFE700200490FFE7049805B07047000065
:1014000089B0079006910592002004900390029005
:10141000059800680190069828BBFFE7FFE704984D
:101420000799896888421DD2FFE7049838B9FFE719
:10143000079800684FF6FC71084003900EE003988F
:10144000029003980799498800EB0140019950F8F0
:1014500021004FF6FC7108400390FFE7049801302B
:101460000490DCE734E0FFE70499079882680020E5
:10147000914200900AD2FFE7039806994FF6FC725A
:101480001140401A18BF01200090FFE70098C007E4
:10149000E8B1FFE7049838B9FFE7079800684FF60E
:1014A000FC71084003900EE003980290039807999E
:1014B000498800EB0140019950F821004FF6FC717A
:1014C00008400390FFE7049801300490CCE7FFE761
:1014D000069860B1FFE7039806994FF6FC72114039
:1014E000884203D0FFE70120089029E0FFE7049835
:1014F0000599886002980799498840EA0140059952
:10150000486003980799498840EA01400599C860F6
:101510000598C068019950F8210070B1FFE705995E
:10152000C868019A50F822004FF6FC721040079AE2
:10153000528840EA02400861FFE700200890FFE778
:10154000089809B07047000083B0029001910092A2
:10155000029890F820008007002811D5FFE7019835
:1015600030B1FFE701990020CFF601600860FFE786
:10157000009820B1FFE7009907200860FFE710E01E
:10158000019830B1FFE701990020CFF60100086013
:10159000FFE7009820B1FFE7009905200860FFE70A
:1015A000FFE703B07047000084B003900399886B95
:1015B000C96B084302900398016801205022C4F2CD
:1015C00002029142019000F06781FFE703980168F1
:1015D00001205022C5F202029142019000F05C818C
:1015E000FFE7039801680120D022C4F20202914271
:1015F000019000F05181FFE7039801680120D0229B
:10160000C5F202029142019000F04681FFE7039883
:101610000168012040F25012C4F20202914201908E
:1016200000F03A81FFE703980168012040F2501270
:10163000C5F202029142019000F02E81FFE703986B
:101640000168012040F2D012C4F2020291420190DE
:1016500000F02281FFE703980168012040F2D012D8
:10166000C5F202029142019000F01681FFE7039853
:101670000168012040F25022C4F20202914201901E
:1016800000F00A81FFE703980168012040F2502230
:10169000C5F202029142019000F0FE80FFE703983C
:1016A0000168012040F2D022C4F20202914201906E
:1016B00000F0F280FFE703980168012040F2D02299
:1016C000C5F202029142019000F0E680FFE7039824
:1016D0000168012040F25032C4F2020291420190AE
:1016E00000F0DA80FFE703980168012040F25032F1
:1016F000C5F202029142019000F0CE80FFE703980C
:101700000168012040F2D032C4F2020291420190FD
:1017100000F0C280FFE703980168012040F2D03258
:10172000C5F202029142019000F0B680FFE70398F3
:101730000168012041F25002C4F20202914201907C
:1017400000F0AA80FFE703980168012041F25002EF
:10175000C5F202029142019000F09E80FFE70398DB
:101760000168012041F2D002C4F2020291420190CC
:1017700000F09280FFE703980168012041F2D00257
:10178000C5F202029142019000F08680FFE70398C3
:101790000168012041F25012C4F20202914201900C
:1017A0007AD0FFE703980168012041F25012C5F298
:1017B0000202914201906FD0FFE703980168012077
:1017C00041F2D012C4F202029142019064D0FFE7CC
:1017D00003980168012041F2D012C5F20202914241
:1017E000019059D0FFE703980168012041F250228F
:1017F000C4F20202914201904ED0FFE703980168C3
:10180000012041F25022C5F202029142019043D0E0
:10181000FFE703980168012041F2D022C4F20202DE
:101820009142019038D0FFE703980168012041F20E
:10183000D022C5F20202914201902DD0FFE7039819
:101840000168012041F25032C4F20202914201903B
:1018500022D0FFE703980168012041F25032C5F21F
:1018600002029142019017D0FFE70398016801201E
:1018700041F2D032C4F20202914201900CD0FFE753
:10188000039800684EF63041CAF6FD710844B0FA7C
:1018900080F040090190FFE70198C00730B1FFE7F1
:1018A0000398016C029808430290FFE703980068D0
:1018B000406920F44300029908430399096848618C
:1018C000039801680020086403990A68496C516410
:1018D00003990968886403990968C86403990968C9
:1018E000086503980168012040F25032C4F20202F8
:1018F000914200904ED0FFE703980168012040F22A
:101900005032C5F202029142009043D0FFE70398A3
:101910000168012040F2D032C4F2020291420090EC
:1019200038D0FFE703980168012040F2D032C5F2B9
:101930000202914200902DD0FFE703980168012038
:1019400041F25032C4F202029142009022D0FFE7ED
:1019500003980168012041F25032C5F2020291421F
:10196000009017D0FFE703980168012041F2D032C0
:10197000C4F20202914200900CD0FFE70398006885
:101980004EF63041CAF6FD710844B0FA80F04009C5
:101990000090FFE70098C00740B1FFE70398016897
:1019A00000204865039909688865FFE70398016886
:1019B0000020C86704B0704784B003900291019280
:1019C000009303980068806C4FF6FF718843BDF860
:1019D00000100844039909688864039801684FF46B
:1019E000FE40C860029803990968C8640198039989
:1019F0000968086504B070477047000072B6FFE7D9
:101A0000FEE7000080B540F6F410C2F2000000F0DE
:101A1000A1FD80BD80B540F66C20C2F2000000F050
:101A200099FD80BD80B540F6E420C2F2000000F0D0
:101A300091FD80BD80B584B002900191029818B1EB
:101A4000FFE7019820B9FFE701208DF80F001AE0A9
:101A5000029800788006002801D5FFE7FFE702988A
:101A6000406C08B1FFE7FFE7029800788007002884
:101A700001D5FFE7FFE702980199FFF7DDFA0020A3
:101A80008DF80F00FFE79DF80F0004B080BD000047
:101A900080B584B0029001F08FFA0190029820B9CD
:101AA000FFE701208DF80F00AFE1029801680120E7
:101AB0005022C4F202029142009000F06781FFE7D9
:101AC0000298016801205022C5F202029142009062
:101AD00000F05C81FFE7029801680120D022C4F287
:101AE00002029142009000F05181FFE702980168E4
:101AF0000120D022C5F202029142009000F04681FE
:101B0000FFE702980168012040F25012C4F202027D
:101B10009142009000F03A81FFE7029801680120AD
:101B200040F25012C5F202029142009000F02E8164
:101B3000FFE702980168012040F2D012C4F20202CD
:101B40009142009000F02281FFE702980168012095
:101B500040F2D012C5F202029142009000F01681CC
:101B6000FFE702980168012040F25022C4F202020D
:101B70009142009000F00A81FFE70298016801207D
:101B800040F25022C5F202029142009000F0FE8025
:101B9000FFE702980168012040F2D022C4F202025D
:101BA0009142009000F0F280FFE702980168012066
:101BB00040F2D022C5F202029142009000F0E6808D
:101BC000FFE702980168012040F25032C4F202029D
:101BD0009142009000F0DA80FFE70298016801204E
:101BE00040F25032C5F202029142009000F0CE80E5
:101BF000FFE702980168012040F2D032C4F20202ED
:101C00009142009000F0C280FFE702980168012035
:101C100040F2D032C5F202029142009000F0B6804C
:101C2000FFE702980168012041F25002C4F202026B
:101C30009142009000F0AA80FFE70298016801201D
:101C400041F25002C5F202029142009000F09E80E3
:101C5000FFE702980168012041F2D002C4F20202BB
:101C60009142009000F09280FFE702980168012005
:101C700041F2D002C5F202029142009000F086804B
:101C8000FFE702980168012041F25012C4F20202FB
:101C9000914200907AD0FFE702980168012041F25A
:101CA0005012C5F20202914200906FD0FFE70298F5
:101CB0000168012041F2D012C4F202029142009068
:101CC00064D0FFE702980168012041F2D012C5F20A
:101CD00002029142009059D0FFE70298016801206A
:101CE00041F25022C4F20202914200904ED0FFE72E
:101CF00002980168012041F25022C5F2020291428D
:101D0000009043D0FFE702980168012041F2D02201
:101D1000C4F202029142009038D0FFE702980168B5
:101D2000012041F2D022C5F20202914200902DD052
:101D3000FFE702980168012041F25032C4F202022A
:101D40009142009022D0FFE702980168012041F201
:101D50005032C5F202029142009017D0FFE702987C
:101D60000168012041F2D032C4F202029142009097
:101D70000CD0FFE7029800684EF63041CAF6FD71BC
:101D80000844B0FA80F040090090FFE70098C007CF
:101D900008B1FFE7FFE7FFE70299002081F84C0058
:101DA000FFE70299022081F854000298016848690F
:101DB00040F006004861FFE7029800684069C007EC
:101DC00098B1FFE701F0F8F80199401A06280BD303
:101DD000FFE70299102088650299032081F85400DA
:101DE00001208DF80F0010E0E6E70298FFF7DCFB1A
:101DF0000299886C0865029900208865029A012181
:101E000082F854108DF80F00FFE79DF80F0004B022
:101E100080BD000080B58CB00A90099108920A98A4
:101E200018B1FFE7089820B9FFE701208DF82F00CF
:101E3000B9E00A984069012807D1FFE70A99042010
:101E4000086101208DF82F00ADE00A98006809991B
:101E5000089AFFF75DFA38B1FFE70A990520086193
:101E600001208DF82F009EE00A9800680999089AD1
:101E7000FFF782FA38B1FFE70A99042008610120D0
:101E80008DF82F008FE00A99022008730A9900202C
:101E90000861089807A906AAFFF756FB0A98006888
:101EA000E0B9FFE7099838B9FFE708980A99086090
:101EB0000A990120886010E009980A99086008983A
:101EC0004FF6FC710840079908430999069A41F8B2
:101ED00022000A9902208860FFE75BE0099878B940
:101EE000FFE70A9800684FF6FC710840079908431D
:101EF0000899069A41F8220008980A99086044E077
:101F0000069801900A98099901AAFFF779FAA0BBEF
:101F1000FFE703980A99896888421BD1FFE70A986E
:101F2000406860B1FFE70A9840684FF6FC710840CE
:101F3000079908430899069A41F82200FFE7089894
:101F40004FF6FC710840079908430999069A41F831
:101F5000220011E00998069A50F82200089941F8E9
:101F6000220008984FF6FC71084007990843099928
:101F7000069A41F82200FFE706E00A990620086168
:101F800001208DF82F000EE0FFE70A9988680130E4
:101F90008860FFE70A99002008610A9A01211173FD
:101FA0008DF82F00FFE79DF82F000CB080BD0000DA
:101FB00085B003900291039818B1FFE7029820B909
:101FC000FFE701208DF81300BFE00398006D20B9F2
:101FD000FFE701208DF81300B7E0039890F8540054
:101FE0008DF80700039890F85400022805D0FFE709
:101FF0009DF8070005280DD1FFE70399402088656B
:10200000FFE70399002081F84C00FFE701208DF8DD
:1020100013009AE00298007B022806D1FFE702999C
:10202000012008618DF813008FE0039801680120FA
:1020300040F25032C4F20202914200904ED0FFE7CB
:1020400003980168012040F25032C5F20202914229
:10205000009043D0FFE703980168012040F2D0329E
:10206000C4F202029142009038D0FFE70398016861
:10207000012040F2D032C5F20202914200902DD0F0
:10208000FFE703980168012041F25032C4F20202D6
:102090009142009022D0FFE703980168012041F2AD
:1020A0005032C5F202029142009017D0FFE7039828
:1020B0000168012041F2D032C4F202029142009044
:1020C0000CD0FFE7039800684EF63041CAF6FD7168
:1020D0000844B0FA80F040090090FFE70098C0077C
:1020E00078B9FFE70298006890F820008007002880
:1020F00007D5FFE702990320086101208DF813003E
:1021000023E00398006D81280CD1FFE70298406816
:1021100038B9FFE702990420086101208DF8130007
:1021200013E00BE00298406838B1FFE70299042001
:10213000086101208DF8130007E0FFE7029803997A
:10214000486700208DF81300FFE79DF8130005B0E5
:102150007047000080B58AB00890089820B9FFE762
:1021600001208DF8270056E00898006838B9FFE78D
:1021700008990220086101208DF827004BE008989B
:10218000406888B1FFE7089801684068884204D138
:10219000FFE700208DF827003DE008990420086142
:1021A00001208DF8270036E008984069012807D102
:1021B000FFE708990420086101208DF827002AE034
:1021C0000899022008730899002000900861089877
:1021D000006807A906AAFFF7B7F9009906980190C9
:1021E000089801AAFFF70CF90098089909684FF6BA
:1021F000FC721140079A1143049A069B42F823107F
:10220000089A1168516008990861089A01211173B0
:102210008DF82700FFE79DF827000AB080BD000079
:1022200080B586B00490049820B1FFE70498406F11
:1022300020B9FFE701208DF8170090E00498006DA9
:1022400020B9FFE701208DF8170088E0049890F886
:1022500054008DF80F0004980068406900F4803045
:1022600002909DF80F00012809D0FFE79DF80F00AC
:10227000022863D1FFE7029800285FD0FFE70498A7
:1022800090F85400012852D1FFE7FFE7049890F836
:102290004C00012804D1FFE702208DF817005EE012
:1022A0000499012081F84C00FFE7FFE70499022020
:1022B00081F854000499496F0873049900208865D7
:1022C0000499496F086104980168486940F4BA406C
:1022D00048610498406E38B1FFE704980168486986
:1022E00040F400704861FFE70498006F38B1FFE7E1
:1022F00004980168486940F400504861FFE7049879
:10230000406F006801A90022FFF71EF904980168D8
:10231000406F40880004086004980168406F0068BE
:102320004FF6FC721040019A1043C867FFE704980B
:102330000168486940F0010048610CE004994020C0
:102340008865FFE70499002081F84C00FFE7012031
:102350008DF8170003E000208DF81700FFE79DF8C7
:10236000170006B080BD000080B584B0029000F078
:1023700023FE0190029820B9FFE701208DF80F009D
:1023800079E0029890F8540002280DD0FFE70299F6
:1023900020208865FFE70299002081F84C00FFE7C4
:1023A00001208DF80F0066E002980168486940F04E
:1023B000040048610299052081F85400FFE7029863
:1023C000006800698004002827D4FFE700F0F4FDCE
:1023D0000199401A06281FD3FFE70299886D40F043
:1023E000100088650299032081F85400029890F843
:1023F00050000006002805D5FFE70298416F012034
:102400000873FFE7FFE70299002081F84C00FFE71F
:1024100001208DF80F002EE0D1E70298016848698D
:1024200040F0020048610299042081F854000298AB
:1024300001684FF4FE40C8600299012081F8540001
:10244000029890F850000006002809D5FFE702988E
:10245000416F012008730298016800208864FFE73B
:10246000FFE70299002081F84C00FFE7FFE700201A
:102470008DF80F00FFE79DF80F0004B080BD00004D
:1024800082B00090009820B9FFE701208DF8070086
:102490001CE0009890F85400022807D0FFE700994C
:1024A0002020886501208DF807000FE000990420A6
:1024B00081F8540000980168486942F20402104310
:1024C0004861FFE700208DF80700FFE79DF807004F
:1024D00002B0704785B003900291039820B9FFE7DE
:1024E00001208DF813002AE00398006840F6FF7180
:1024F00088430190039800685038C0F3C41101204C
:10250000884000909DF80800C006002813D5FFE71A
:10251000029800F01100112806D1FFE7009A0199F6
:1025200048681043486005E0009A01994868904364
:102530004860FFE7FFE700208DF81300FFE79DF8F4
:10254000130005B07047000081B000900098806DC6
:1025500001B0704780B584B003900398006840F6DE
:10256000FF7188430290039800685038C0F3C4118B
:102570000120884001900298C068019908400090AD
:10258000009808B9FFE74DE103980068006940052D
:10259000002813D5FFE7039800684069400500282C
:1025A0000BD5FFE7039801684FF48060C86003997A
:1025B000886D40F001008865FFE7FFE70398006839
:1025C00000690005002813D5FFE7039800684069FB
:1025D000000500280BD5FFE7039801684FF4006061
:1025E000C8600399886D40F002008865FFE7FFE747
:1025F000039800680069C004002813D5FFE703981A
:1026000000684069C00400280BD5FFE70398016803
:102610004FF48050C8600399886D40F004008865CD
:10262000FFE7FFE70398006800694004002813D51E
:10263000FFE7039800684069400400280BD5FFE7D6
:10264000039801684FF48040C8600399886D40F09A
:1026500008008865FFE7FFE70398006800698005C8
:10266000002816D5FFE70398006840698005002818
:102670000ED5FFE7039801684FF40070C860039817
:10268000406E20B1FFE70398416E8847FFE7FFE700
:10269000FFE70398006800698004002850D5FFE731
:1026A0000398006840698004002848D5FFE7039834
:1026B00001684FF40050C860039890F85400042853
:1026C0002FD1FFE703980168486920F40050486162
:1026D00003980168486940F00200486103990120AD
:1026E00081F85400039890F850000006002809D59E
:1026F000FFE70398416F01200873039801680020E9
:102700008864FFE7FFE70399002081F84C00FFE7AA
:102710000398C06E20B1FFE70398C16E8847FFE7BA
:1027200080E00399052081F854000398006F20B1E0
:10273000FFE70398016F8847FFE7FFE7FFE7FFE741
:10274000039800680069C005002842D5FFE7039898
:1027500000684069C00500283AD5FFE7039890F863
:1027600050000006002814D5FFE703980068C06FEA
:1027700070B9FFE703980068806C40B9FFE70399E0
:10278000012081F854000399496F0873FFE7FFE7C0
:102790000AE003980068806C28B9FFE703990120DC
:1027A00081F85400FFE7FFE7039801684FF4407099
:1027B000C860FFE70399002081F84C00FFE7039809
:1027C000006E20B1FFE70398016E8847FFE7FFE73F
:1027D000FFE70398806D28B3FFE703980168486915
:1027E00040F0020048610399012081F854000398E9
:1027F00090F850000006002805D5FFE70398416FC8
:1028000001200873FFE7FFE70399002081F84C00DF
:10281000FFE70398806E20B1FFE70398816E884739
:10282000FFE7FFE704B080BD80B584B0029000F000
:10283000C3FB0190029820B9FFE701208DF80F003B
:10284000CEE10298C068B0F5007F01D0FFE7FFE756
:102850000298406BB0F5805F01D1FFE7FFE7029877
:10286000016801205022C4F202029142009000F05F
:102870006781FFE70298016801205022C5F2020239
:102880009142009000F05C81FFE70298016801200E
:10289000D022C4F202029142009000F05181FFE781
:1028A000029801680120D022C5F2020291420090F4
:1028B00000F04681FFE702980168012040F25012C3
:1028C000C4F202029142009000F03A81FFE70298C0
:1028D0000168012040F25012C5F2020291420090BC
:1028E00000F02E81FFE702980168012040F2D0122B
:1028F000C4F202029142009000F02281FFE70298A8
:102900000168012040F2D012C5F20202914200900B
:1029100000F01681FFE702980168012040F2502282
:10292000C4F202029142009000F00A81FFE702988F
:102930000168012040F25022C5F20202914200904B
:1029400000F0FE80FFE702980168012040F2D022EB
:10295000C4F202029142009000F0F280FFE7029878
:102960000168012040F2D022C5F20202914200909B
:1029700000F0E680FFE702980168012040F2503243
:10298000C4F202029142009000F0DA80FFE7029860
:102990000168012040F25032C5F2020291420090DB
:1029A00000F0CE80FFE702980168012040F2D032AB
:1029B000C4F202029142009000F0C280FFE7029848
:1029C0000168012040F2D032C5F20202914200902B
:1029D00000F0B680FFE702980168012041F2500242
:1029E000C4F202029142009000F0AA80FFE7029830
:1029F0000168012041F25002C5F2020291420090AA
:102A000000F09E80FFE702980168012041F2D002A9
:102A1000C4F202029142009000F09280FFE7029817
:102A20000168012041F2D002C5F2020291420090F9
:102A300000F08680FFE702980168012041F2501201
:102A4000C4F20202914200907AD0FFE70298016836
:102A5000012041F25012C5F20202914200906FD063
:102A6000FFE702980168012041F2D012C4F202028D
:102A70009142009064D0FFE702980168012041F282
:102A8000D012C5F202029142009059D0FFE702989D
:102A90000168012041F25022C4F2020291420090EA
:102AA0004ED0FFE702980168012041F25022C5F2A2
:102AB00002029142009043D0FFE702980168012092
:102AC00041F2D022C4F202029142009038D0FFE7D6
:102AD00002980168012041F2D022C5F2020291421F
:102AE00000902DD0FFE702980168012041F250329A
:102AF000C4F202029142009022D0FFE702980168DE
:102B0000012041F25032C5F202029142009017D0EA
:102B1000FFE702980168012041F2D032C4F20202BC
:102B2000914200900CD0FFE7029800684EF63041C9
:102B3000CAF6FD710844B0FA80F040090090FFE742
:102B40000098C00708B1FFE7FFE7FFE70299002000
:102B500081F84C00FFE7029890F8540060B9FFE755
:102B600002990020086602994866029988660299CF
:102B7000C86602990867FFE70299022081F85400AD
:102B800002980168486940F006004861FFE7029832
:102B900000684069C00798B1FFE700F00DFA01999D
:102BA000401A06280BD3FFE7029910208865029986
:102BB000032081F8540001208DF80F0010E0E6E7B3
:102BC0000298FDF773FE0299486B08650299002090
:102BD0008865029A012182F854108DF80F00FFE7F2
:102BE0009DF80F0004B080BD80B586B004900391BD
:102BF00002920193049820B9FFE701208DF8170095
:102C00005FE00498006D20B1FFE701208DF8170008
:102C100057E0FFE7049890F84C00012804D1FFE743
:102C200002208DF817004CE00499012081F84C0037
:102C3000FFE7FFE7049890F85400012830D1FFE740
:102C40000499022081F854000499002088650498B2
:102C50000399029A019BFEF7AFFE04980168486948
:102C600040F4BA4048610498406E38B1FFE70498D8
:102C70000168486940F400704861FFE70498006FFC
:102C800038B1FFE704980168486940F40050486192
:102C9000FFE704980168486940F0010048610CE0D2
:102CA000049940208865FFE70499002081F84C00D2
:102CB000FFE701208DF8170003E000208DF81700D2
:102CC000FFE79DF8170006B080BD000085B00490B6
:102CD000039100200090FFE7039800680099C84026
:102CE000002800F06681FFE703980068009A012140
:102CF0009140084001900198002800F05681FFE7BC
:102D000003984068022805D0FFE70398406812281E
:102D100028D1FFE7049800996FF0030202EA5101FD
:102D20000844006A0290009800F0070081000F201C
:102D300000FA01F10298884302900398006900F0BC
:102D40000F00009901F00701890000FA01F10298D3
:102D50000843029002980499009B02EA530211442E
:102D60000862FFE704980068029000984100032081
:102D700000FA01F10298884302900398406800F03D
:102D800003000099490000FA01F1029808430290FB
:102D90000298049908600398406801280FD0FFE763
:102DA0000398406802280AD0FFE70398406811287A
:102DB00005D0FFE70398406812282FD1FFE7049859
:102DC0008068029000984100032000FA01F1029807
:102DD000884302900398C0680099490000FA01F105
:102DE0000298084302900298049988600498406809
:102DF00002900099012000FA01F1029888430290A4
:102E000003984068C0F30010009900FA01F102989D
:102E100008430290029804994860FFE703984068CD
:102E200000F0030003280CD1FFE70398406800F08E
:102E3000030003281DD1FFE703988068012818D0FC
:102E4000FFE70498C068029000984100032000FA50
:102E500001F1029888430290039880680099490024
:102E600000FA01F102980843029002980499C860A0
:102E7000FFE70398C079C006002840F19580FFE77E
:102E8000009820F0030042F26002C4F2024280582F
:102E90000290009800F00300C1000F2000FA01F139
:102EA00002988843029004984FF60041CBF6FD51FA
:102EB0000840800A009901F00301C90000FA01F1FD
:102EC0000298084302900298009921F0030188506B
:102ED00042F20000C4F20240006802900199029898
:102EE0008843029003988079C006002805D5FFE743
:102EF0000199029808430290FFE7029842F200010C
:102F0000C4F20241086042F20400C4F202400068C8
:102F10000290019902988843029003988079800674
:102F2000002805D5FFE70199029808430290FFE7C2
:102F3000029842F20401C4F20241086042F28400A5
:102F4000C4F20240006802900199029888430290FE
:102F5000039880798007002805D5FFE7019902983A
:102F600008430290FFE7029842F28401C4F2024152
:102F7000086042F28000C4F20240006802900199A9
:102F800002988843029003988079C00728B1FFE730
:102F90000199029808430290FFE7029842F28001EB
:102FA000C4F202410860FFE7FFE70098013000909B
:102FB00092E605B07047000041F24810C2F20000EE
:102FC0000068704740F20800C2F20000027841F247
:102FD0004811C2F200010868104408607047000000
:102FE00080B582B0032000F0B7F805F0FBF840F69A
:102FF0002041C4F20241096801F00F024DF68241FE
:10300000C0F60001895CC84040F20001C2F2000134
:103010000860042005F04AFF0F2000F011F820B1ED
:10302000FFE701208DF8070005E000F071F80020AF
:103030008DF80700FFE79DF8070002B080BD000093
:1030400080B58CB00B90FFE740F6A440C4F202407C
:10305000016841F400610160006800F400600090C4
:103060000098FFE705A802A905F030F805F092F8EE
:1030700004900498400945F6C521C0F67C21A0FBC8
:1030800001014FF0FF3000EBD110039040F65C30AF
:10309000C2F2000042F60041C4F201010160632166
:1030A000C1600399416000210161816005F068FF02
:1030B0008DF807009DF8070010BBFFE740F65C3075
:1030C000C2F2000005F0B4FF8DF807009DF807007C
:1030D000A8B9FFE70B980F280CD8FFE70B992A2017
:1030E000002200F021F80B9840F20C01C2F200011E
:1030F000086003E001208DF80700FFE7FFE7FFE726
:103100002A2000F007F89DF807000CB080BD0000F1
:103110007047000080B582B0ADF80600BDF906002A
:1031200009F01CFC02B080BD80B586B0ADF8160079
:103130000491039209F02AFC0290BDF91600019057
:1031400002980499039A07F0DFFA0146019809F002
:1031500025FC06B080BD000080B582B001900198CA
:1031600009F03EFC02B080BD89B0089040F63440C2
:10317000C4F2024000686FF35F20059040F62840DB
:10318000C4F20240016801F0030107910168C1F334
:10319000052106910068C0F300100490049840F6E1
:1031A0003841C4F20241096889B2C90800FB01F044
:1031B00000EE100AB8EE400A8DED020A06980028CB
:1031C00000F03D81FFE707980090012808D0FFE755
:1031D0000098022830D0FFE70098032849D065E026
:1031E00040F60040C4F202400068C0F3C10149F259
:1031F0000000C0F2D030C84003909DED030AB8EE45
:10320000400A9DED061AB8EE411A80EE010A9DEDC6
:10321000051AB8EE411A9DED022A9FED8F3A82EE13
:10322000032A31EE021AB7EE002A31EE021A20EE1E
:10323000010A8DED010A65E09DED060AB8EE401A1F
:103240009FED860A80EE010A9DED051AB8EE411A3F
:103250009DED022A9FED803A82EE032A31EE021A9A
:10326000B7EE002A31EE021A20EE010A8DED010AB6
:1032700048E09DED060AB8EE401A9FED760A80EE12
:10328000010A9DED051AB8EE411A9DED022A9FED47
:10329000723A82EE032A31EE021AB7EE002A31EEBC
:1032A000021A20EE010A8DED010A2BE040F60040E3
:1032B000C4F202400068C0F3C10149F20000C0F24C
:1032C000D030C84003909DED030AB8EE400A9DED52
:1032D000061AB8EE411A80EE010A9DED051AB8EE05
:1032E000411A9DED022A9FED5C3A82EE032A31EEEF
:1032F000021AB7EE002A31EE021A20EE010A8DED15
:10330000010AFFE740F60040C4F202400068800175
:10331000002827D5FFE740F62840C4F202400068A5
:10332000C003002819D5FFE79DED010A40F634409F
:10333000C4F20240006880B2400A01EE100AB8EE02
:10334000411AB7EE002A31EE021A80EE010A0898FF
:10335000BCEEC00A80ED000A03E008990020086076
:10336000FFE703E0089900200860FFE740F600400F
:10337000C4F2024000688001002827D5FFE740F62C
:103380002840C4F2024000688003002819D5FFE7F6
:103390009DED010A40F63440C4F202400068C0F3DB
:1033A000064001EE100AB8EE411AB7EE002A31EEDF
:1033B000021A80EE010A0898BCEEC00A80ED010AEC
:1033C00003E0089900204860FFE703E00899002027
:1033D0004860FFE740F60040C4F202400068800108
:1033E000002827D5FFE740F62840C4F202400068D5
:1033F0004003002819D5FFE79DED010A40F634404F
:10340000C4F202400068C0F3066001EE100AB8EE94
:10341000411AB7EE002A31EE021A80EE010A08982E
:10342000BCEEC00A80ED020A03E008990020886023
:10343000FFE703E0089900208860FFE707E00899AC
:10344000002008600899486008998860FFE709B083
:10345000704700BF20BCBE4B000000460024744AE9
:1034600089B0089040F63C40C4F2024000686FF317
:103470005F20059040F62C40C4F20240016801F044
:10348000030107910168C1F3052106910068C0F3AB
:1034900000100490049840F64041C4F202410968CB
:1034A00089B2C90800FB01F000EE100AB8EE400A2C
:1034B0008DED020A0698002800F03D81FFE707988D
:1034C0000090012808D0FFE70098022830D0FFE7DD
:1034D0000098032849D065E040F60040C4F202405D
:1034E0000068C0F3C10149F20000C0F2D030C8400A
:1034F00003909DED030AB8EE400A9DED061AB8EE62
:10350000411A80EE010A9DED051AB8EE411A9DEDB3
:10351000022A9FED8F3A82EE032A31EE021AB7EEAD
:10352000002A31EE021A20EE010A8DED010A65E053
:103530009DED060AB8EE401A9FED860A80EE010A5C
:103540009DED051AB8EE411A9DED022A9FED803AD5
:1035500082EE032A31EE021AB7EE002A31EE021A89
:1035600020EE010A8DED010A48E09DED060AB8EE55
:10357000401A9FED760A80EE010A9DED051AB8EE1D
:10358000411A9DED022A9FED723A82EE032A31EE36
:10359000021AB7EE002A31EE021A20EE010A8DED72
:1035A000010A2BE040F60040C4F202400068C0F37C
:1035B000C10149F20000C0F2D030C84003909DED37
:1035C000030AB8EE400A9DED061AB8EE411A80EEE5
:1035D000010A9DED051AB8EE411A9DED022A9FEDF4
:1035E0005C3A82EE032A31EE021AB7EE002A31EE7F
:1035F000021A20EE010A8DED010AFFE740F60040B5
:10360000C4F2024000680001002827D5FFE740F619
:103610002C40C4F202400068C003002819D5FFE71F
:103620009DED010A40F63C40C4F20240006880B2C1
:10363000400A01EE100AB8EE411AB7EE002A31EE48
:10364000021A80EE010A0898BCEEC00A80ED000A5A
:1036500003E0089900200860FFE703E008990020D4
:103660000860FFE740F60040C4F202400068000135
:10367000002827D5FFE740F62C40C4F2024000683E
:103680008003002819D5FFE79DED010A40F63C4074
:10369000C4F202400068C0F3064001EE100AB8EE22
:1036A000411AB7EE002A31EE021A80EE010A08989C
:1036B000BCEEC00A80ED010A03E0089900204860D2
:1036C000FFE703E0089900204860FFE740F600406C
:1036D000C4F2024000680001002827D5FFE740F649
:1036E0002C40C4F2024000684003002819D5FFE7CF
:1036F0009DED010A40F63C40C4F202400068C0F370
:10370000066001EE100AB8EE411AB7EE002A31EE5B
:10371000021A80EE010A0898BCEEC00A80ED020A87
:1037200003E0089900208860FFE703E00899002083
:103730008860FFE707E00899002008600899486062
:1037400008998860FFE709B0704700BF20BCBE4BF6
:10375000000000460024744A89B0089040F64440B6
:10376000C4F2024000686FF35F20059040F63040DD
:10377000C4F20240016801F0030107910168C1F33E
:10378000052106910068C0F300100490049840F6EB
:103790004841C4F20241096889B2C90800FB01F03E
:1037A00000EE100AB8EE400A8DED020A06980028D5
:1037B00000F03D81FFE707980090012808D0FFE75F
:1037C0000098022830D0FFE70098032849D065E030
:1037D00040F60040C4F202400068C0F3C10149F263
:1037E0000000C0F2D030C84003909DED030AB8EE4F
:1037F000400A9DED061AB8EE411A80EE010A9DEDD1
:10380000051AB8EE411A9DED022A9FED8F3A82EE1D
:10381000032A31EE021AB7EE002A31EE021A20EE28
:10382000010A8DED010A65E09DED060AB8EE401A29
:103830009FED860A80EE010A9DED051AB8EE411A49
:103840009DED022A9FED803A82EE032A31EE021AA4
:10385000B7EE002A31EE021A20EE010A8DED010AC0
:1038600048E09DED060AB8EE401A9FED760A80EE1C
:10387000010A9DED051AB8EE411A9DED022A9FED51
:10388000723A82EE032A31EE021AB7EE002A31EEC6
:10389000021A20EE010A8DED010A2BE040F60040ED
:1038A000C4F202400068C0F3C10149F20000C0F256
:1038B000D030C84003909DED030AB8EE400A9DED5C
:1038C000061AB8EE411A80EE010A9DED051AB8EE0F
:1038D000411A9DED022A9FED5C3A82EE032A31EEF9
:1038E000021AB7EE002A31EE021A20EE010A8DED1F
:1038F000010AFFE740F60040C4F202400068800081
:10390000002827D5FFE740F63040C4F202400068A7
:10391000C003002819D5FFE79DED010A40F6444099
:10392000C4F20240006880B2400A01EE100AB8EE0C
:10393000411AB7EE002A31EE021A80EE010A089809
:10394000BCEEC00A80ED000A03E008990020086080
:10395000FFE703E0089900200860FFE740F6004019
:10396000C4F2024000688000002827D5FFE740F637
:103970003040C4F2024000688003002819D5FFE7F8
:103980009DED010A40F64440C4F202400068C0F3D5
:10399000064001EE100AB8EE411AB7EE002A31EEE9
:1039A000021A80EE010A0898BCEEC00A80ED010AF6
:1039B00003E0089900204860FFE703E00899002031
:1039C0004860FFE740F60040C4F202400068800013
:1039D000002827D5FFE740F63040C4F202400068D7
:1039E0004003002819D5FFE79DED010A40F6444049
:1039F000C4F202400068C0F3066001EE100AB8EE9F
:103A0000411AB7EE002A31EE021A80EE010A089838
:103A1000BCEEC00A80ED020A03E00899002088602D
:103A2000FFE703E0089900208860FFE707E00899B6
:103A3000002008600899486008998860FFE709B08D
:103A4000704700BF20BCBE4B000000460024744AF3
:103A500080B59CB01B911A901A981B9980F0007049
:103A6000084300285BD1FFE740F6F040C4F2024073
:103A7000016801F440710E9100688007002809D5A3
:103A8000FFE70E98B0F5807F04D1FFE74FF40040C8
:103A9000109042E040F6F040C4F20240006800019D
:103AA000002809D5FFE70E98B0F5007F04D1FFE7A5
:103AB0004FF4FA4010902FE040F60040C4F202406C
:103AC00000688003002823D5FFE70E98B0F5407FFB
:103AD0001ED1FFE740F61C40C4F20240006800F42B
:103AE0007C50B0F5007F0FD3FFE740F61C40C4F2D6
:103AF00002400068C0F3052147F64000C0F27D1087
:103B0000B0FBF1F0109002E000201090FFE702E01F
:103B100000201090FFE7FFE7FFE702F012BC1A98C1
:103B20000C901B990D9180F001000843002800F0D3
:103B3000C682FFE70D990C9880F002000843002828
:103B400000F03B83FFE70D990C9880F004000843D8
:103B5000002800F0A783FFE70D990C9880F008007B
:103B60000843002800F01E84FFE70D990C9880F0B0
:103B700010000843002800F09884FFE70D990C9886
:103B800080F020000843002800F01285FFE70D991F
:103B90000C9880F040000843002800F08C85FFE777
:103BA0000D990C9880F080000843002800F00686EC
:103BB000FFE70D990C9880F480700843002800F00E
:103BC0008086FFE70D990C9880F400700843002868
:103BD00000F0FA86FFE70D990C9880F480600843A6
:103BE000002800F07487FFE70D990C9880F40060BE
:103BF0000843002800F0E987FFE70D990C9880F44E
:103C000080500843002801F05E80FFE70D990C9872
:103C100080F400500843002801F06181FFE70D990E
:103C20000C9880F480400843002801F0AA81FFE747
:103C30000D990C9880F400400843002801F0F381AE
:103C4000FFE70D990C9880F480300843002801F0BC
:103C50008E82FFE70D990C9880F40030084300280D
:103C600001F0C282FFE70D990C9880F48020084390
:103C7000002801F06583FFE70D990C9880F400207F
:103C80000843002800F0BF80FFE70D990C9880F4EE
:103C900080100843002800F04381FFE70D990C983D
:103CA00080F400100843002801F07E80FFE70D99A2
:103CB0000C9880F480000843002800F0BE81FFE7E4
:103CC0000D990C9880F400000843002800F0D6817C
:103CD000FFE70D990C9880F080600843002802F0FF
:103CE0009882FFE70D990C9880F000600843002847
:103CF00001F0B986FFE70D990C9880F080500843D9
:103D0000002801F02F87FFE70D990C9880F00050F4
:103D10000843002801F0B387FFE70D990C9880F065
:103D200080400843002802F03380FFE70D990C988B
:103D300080F000400843002802F0AE80FFE70C98B6
:103D40000D9981F001010843002802F02981FFE765
:103D50000C980D9981F002010843002802F0A4811B
:103D6000FFE70C980D9981F004010843002801F049
:103D70004386FFE70C980D9981F00801084300285D
:103D800002F00782FFE70C980D9981F010010843BB
:103D9000002802F09482FFE70C980D9981F0200131
:103DA0000843002801F07883FFE70C980D9981F013
:103DB00040010843002801F01B84FFE70C980D998F
:103DC00081F080010843002801F0BE84FFE70C98D1
:103DD0000D9981F480710843002801F06185FFE7A7
:103DE0000C980D9981F400710843002801F0488077
:103DF000FFE70C980D9981F480610843002801F0D9
:103E0000648102F09ABA40F6E840C4F202400068C9
:103E100000F4E0200E900E980B90A0B1FFE70B98F5
:103E2000B0F5803F15D0FFE70B98B0F5003F16D0F6
:103E3000FFE70B98B0F5403F17D0FFE70B98B0F5C0
:103E4000802F18D067E017A8FFF78EF91898109008
:103E500064E014A8FFF704FB149810905EE011A82A
:103E6000FFF77AFC1198109058E048F20000C0F279
:103E7000BB00109052E040F6E840C4F202400068F7
:103E800000F040400F9040F60040C4F2024000684D
:103E90008007002811D5FFE70F9870B9FFE740F6BB
:103EA0000040C4F202400068C0F3C10149F20000C2
:103EB000C0F2D030C84010902CE040F60040C4F270
:103EC00002400068800500280BD5FFE70F98B0F18D
:103ED000804F06D1FFE740F60010C0F23D00109081
:103EE00017E040F60040C4F202400068800300285A
:103EF0000BD5FFE70F98B0F1004F06D1FFE747F66B
:103F00004000C0F27D10109002E000201090FFE70A
:103F1000FFE7FFE702E000201090FFE702F010BA91
:103F200040F6E840C4F20240006800F460100E90D1
:103F30000E980A90A0B1FFE70A98B0F5002F15D0AF
:103F4000FFE70A98B0F5801F16D0FFE70A98B0F592
:103F5000C01F17D0FFE70A98B0F5001F18D067E020
:103F600017A8FFF701F91898109064E014A8FFF75C
:103F700077FA149810905EE011A8FFF7EDFB119806
:103F8000109058E048F20000C0F2BB00109052E0E0
:103F900040F6E840C4F20240006800F040400F9054
:103FA00040F60040C4F2024000688007002811D5A6
:103FB000FFE70F9870B9FFE740F60040C4F20240F7
:103FC0000068C0F3C10149F20000C0F2D030C8401F
:103FD00010902CE040F60040C4F2024000688005DA
:103FE00000280BD5FFE70F98B0F1804F06D1FFE70F
:103FF00040F60010C0F23D00109017E040F600407F
:10400000C4F202400068800300280BD5FFE70F9838
:10401000B0F1004F06D1FFE747F64000C0F27D1037
:10402000109002E000201090FFE7FFE7FFE702E0BA
:1040300000201090FFE702F083B940F6E440C4F29C
:104040000240006800F040000E900E9830B9FFE783
:1040500017A8FFF789F8189810900DE00E984028DF
:1040600006D1FFE714A8FFF7FBF91698109002E0BD
:1040700000201090FFE7FFE702F062B940F6E4404D
:10408000C4F20240006800F080000E900E9830B933
:10409000FFE717A8FFF768F8189810900DE00E9842
:1040A000802806D1FFE714A8FFF7DAF916981090D8
:1040B00002E000201090FFE7FFE702F041B940F670
:1040C000D840C4F20240006800F007000E900E983D
:1040D00020B9FFE704F05EF810906CE040F6004075
:1040E000C4F202400068000100280AD5FFE70E98DC
:1040F000012806D1FFE714A8FFF7B2F91598109030
:1041000058E040F60040C4F20240006880000028F9
:104110000AD5FFE70E98022806D1FFE711A8FFF79E
:104120001BFB1298109044E040F60040C4F202409D
:1041300000688007002812D5FFE70E9803280ED1EB
:10414000FFE740F60040C4F202400068C0F3C1013E
:1041500049F20000C0F2D030C840109028E040F68C
:104160000040C4F202400068800500280AD5FFE73D
:104170000E98042806D1FFE740F60010C0F23D007B
:10418000109014E040F6F040C4F20240006880074E
:10419000002808D5FFE70E98052804D1FFE74FF463
:1041A0000040109002E000201090FFE7FFE7FFE7DB
:1041B000FFE7FFE7FFE702F0C3B840F6D840C4F2DC
:1041C0000240006800F038000E900E9820B9FFE71A
:1041D00003F0CCFF109063E040F60040C4F20240D0
:1041E0000068000100280AD5FFE70E98082806D1CC
:1041F000FFE714A8FFF734F9159810904FE00E98D8
:10420000102806D1FFE711A8FFF7A6FA1298109020
:1042100044E040F60040C4F20240006880070028F5
:1042200012D5FFE70E9818280ED1FFE740F60040A0
:10423000C4F202400068C0F3C10149F20000C0F2BC
:10424000D030C840109028E040F60040C4F2024050
:104250000068800500280AD5FFE70E98202806D1BF
:10426000FFE740F60010C0F23D00109014E040F669
:10427000F040C4F2024000688007002808D5FFE73C
:104280000E98282804D1FFE74FF40040109002E078
:1042900000201090FFE7FFE7FFE7FFE7FFE7FFE7FA
:1042A00002F04EB840F6D840C4F20240006800F474
:1042B000E0700E900E9820B9FFE703F057FF1090C2
:1042C0006EE040F60040C4F20240006800010028A1
:1042D0000AD5FFE70E98402806D1FFE714A8FFF79C
:1042E000BFF8159810905AE040F60040C4F2024022
:1042F0000068800000280AD5FFE70E98802806D1C4
:10430000FFE711A8FFF728FA1298109046E040F650
:104310000040C4F2024000688007002812D5FFE781
:104320000E98C0280ED1FFE740F60040C4F20240CC
:104330000068C0F3C10149F20000C0F2D030C840AB
:1043400010902AE040F60040C4F202400068800568
:1043500000280BD5FFE70E98B0F5807F06D1FFE768
:1043600040F60010C0F23D00109015E040F6F0401D
:10437000C4F2024000688007002809D5FFE70E98C4
:10438000B0F5A07F04D1FFE74FF40040109002E0A9
:1043900000201090FFE7FFE7FFE7FFE7FFE7FFE7F9
:1043A00001F0CEBF40F6D840C4F20240006800F4ED
:1043B00060600E900E9820B9FFE703F0D7FE1090D2
:1043C00071E040F60040C4F202400068000100289D
:1043D0000BD5FFE70E98B0F5007F06D1FFE714A8D4
:1043E000FFF73EF8159810905CE040F60040C4F2EC
:1043F00002400068800000280BD5FFE70E98B0F55A
:10440000806F06D1FFE711A8FFF7A6F91298109068
:1044100047E040F60040C4F20240006880070028F0
:1044200013D5FFE70E98B0F5C06F0ED1FFE740F649
:104430000040C4F202400068C0F3C10149F200002C
:10444000C0F2D030C84010902AE040F60040C4F2DC
:1044500002400068800500280BD5FFE70E98B0F5F4
:10446000006F06D1FFE740F60010C0F23D0010904B
:1044700015E040F6F040C4F20240006880070028D2
:1044800009D5FFE70E98B0F5206F04D1FFE74FF490
:104490000040109002E000201090FFE7FFE7FFE7E8
:1044A000FFE7FFE7FFE701F04BBF40F6D840C4F25B
:1044B0000240006800F4E0400E900E9820B9FFE73B
:1044C00003F054FE109071E040F60040C4F2024048
:1044D0000068000100280BD5FFE70E98B0F5805F5B
:1044E00006D1FFE714A8FEF7BBFF159810905CE01B
:1044F00040F60040C4F202400068800000280BD55E
:10450000FFE70E98B0F5005F06D1FFE711A8FFF7AF
:1045100023F91298109047E040F60040C4F20240A0
:1045200000688007002813D5FFE70E98B0F5405FBC
:104530000ED1FFE740F60040C4F202400068C0F32D
:10454000C10149F20000C0F2D030C84010902AE00A
:1045500040F60040C4F202400068800500280BD5F8
:10456000FFE70E98B0F5804F06D1FFE740F6001048
:10457000C0F23D00109015E040F6F040C4F2024059
:1045800000688007002809D5FFE70E98B0F5A04F16
:1045900004D1FFE74FF40040109002E0002010909B
:1045A000FFE7FFE7FFE7FFE7FFE7FFE701F0C8BE30
:1045B00040F6D840C4F20240006800F460300E902B
:1045C0000E9820B9FFE703F0D1FD109071E040F69E
:1045D0000040C4F202400068000100280BD5FFE74C
:1045E0000E98B0F5004F06D1FFE714A8FEF738FF8C
:1045F000159810905CE040F60040C4F2024000685C
:10460000800000280BD5FFE70E98B0F5803F06D15B
:10461000FFE711A8FFF7A0F81298109047E040F6C6
:104620000040C4F2024000688007002813D5FFE76D
:104630000E98B0F5C03F0ED1FFE740F60040C4F23F
:1046400002400068C0F3C10149F20000C0F2D0305E
:10465000C84010902AE040F60040C4F202400068D2
:10466000800500280BD5FFE70E98B0F5003F06D176
:10467000FFE740F60010C0F23D00109015E040F654
:10468000F040C4F2024000688007002809D5FFE727
:104690000E98B0F5203F04D1FFE74FF40040109092
:1046A00002E000201090FFE7FFE7FFE7FFE7FFE7EA
:1046B000FFE701F045BE40F6D840C4F20240006872
:1046C00000F4E0100E900E9820B9FFE703F04EFDC5
:1046D000109071E040F60040C4F202400068000112
:1046E00000280BD5FFE70E98B0F5802F06D1FFE725
:1046F00014A8FEF7B5FE159810905CE040F6004057
:10470000C4F202400068800000280BD5FFE70E9835
:10471000B0F5002F06D1FFE711A8FFF71DF812989A
:10472000109047E040F60040C4F202400068800765
:10473000002813D5FFE70E98B0F5402F0ED1FFE704
:1047400040F60040C4F202400068C0F3C10149F2E3
:104750000000C0F2D030C84010902AE040F600407F
:10476000C4F202400068800500280BD5FFE70E98D0
:10477000B0F5801F06D1FFE740F60010C0F23D0003
:10478000109015E040F6F040C4F202400068800747
:10479000002809D5FFE70E98B0F5A01F04D1FFE768
:1047A0004FF40040109002E000201090FFE7FFE778
:1047B000FFE7FFE7FFE7FFE701F0C2BD40F6D840A3
:1047C000C4F20240006800F460000E900E9820B918
:1047D000FFE703F0CBFC109071E040F60040C4F21C
:1047E00002400068000100280BD5FFE70E98B0F5E5
:1047F000001F06D1FFE714A8FEF732FE15981090AF
:104800005CE040F60040C4F20240006880000028EE
:104810000BD5FFE70E98B0F5800F06D1FFE711A882
:10482000FEF79AFF1298109047E040F60040C4F25D
:10483000024000688007002813D5FFE70E98B0F506
:10484000C00F0ED1FFE740F60040C4F202400068FE
:10485000C0F3C10149F20000C0F2D030C84010904E
:104860002AE040F60040C4F20240006880050028BB
:104870000BD5FFE70E98B0F5000F06D1FFE740F625
:104880000010C0F23D00109015E040F6F040C4F278
:10489000024000688007002809D5FFE70E98B0F5B0
:1048A000200F04D1FFE74FF40040109002E00020F9
:1048B0001090FFE7FFE7FFE7FFE7FFE7FFE701F003
:1048C0003FBD40F6D840C4F20240006800F0E0600E
:1048D0000E900E9820B9FFE703F048FC109071E0AD
:1048E00040F60040C4F202400068000100280BD5E9
:1048F000FFE70E98B0F1807F06D1FFE714A8FEF71E
:10490000AFFD159810905CE040F60040C4F2024004
:104910000068800000280BD5FFE70E98B0F1007FFB
:1049200006D1FFE711A8FEF717FF1298109047E095
:1049300040F60040C4F2024000688007002813D50A
:10494000FFE70E98B0F1407F0ED1FFE740F6004040
:10495000C4F202400068C0F3C10149F20000C0F295
:10496000D030C84010902AE040F60040C4F2024027
:104970000068800500280BD5FFE70E98B0F1806F26
:1049800006D1FFE740F60010C0F23D00109015E0A0
:1049900040F6F040C4F2024000688007002809D5C4
:1049A000FFE70E98B0F1A06F04D1FFE74FF400408D
:1049B000109002E000201090FFE7FFE7FFE7FFE71D
:1049C000FFE7FFE701F0BCBC40F6D840C4F202406C
:1049D000006800F060500E900E9820B9FFE703F0D9
:1049E000C5FB109071E040F60040C4F20240006840
:1049F000000100280BD5FFE70E98B0F1006F06D13B
:104A0000FFE714A8FEF72CFD159810905CE040F627
:104A10000040C4F202400068800000280BD5FFE788
:104A20000E98B0F1805F06D1FFE711A8FEF794FE63
:104A30001298109047E040F60040C4F2024000682F
:104A40008007002813D5FFE70E98B0F1C05F0ED1A4
:104A5000FFE740F60040C4F202400068C0F3C10125
:104A600049F20000C0F2D030C84010902AE040F671
:104A70000040C4F202400068800500280BD5FFE723
:104A80000E98B0F1005F06D1FFE740F60010C0F2CB
:104A90003D00109015E040F6F040C4F2024000687E
:104AA0008007002809D5FFE70E98B0F1205F04D1F8
:104AB000FFE74FF40040109002E000201090FFE765
:104AC000FFE7FFE7FFE7FFE7FFE701F039BC40F64C
:104AD000DC40C4F20240006800F007000E900E981F
:104AE00020B9FFE703F042FB10906CE040F6004075
:104AF000C4F202400068000100280AD5FFE70E98C2
:104B0000012806D1FFE714A8FEF7AAFC159810901B
:104B100058E040F60040C4F20240006880000028DF
:104B20000AD5FFE70E98022806D1FFE711A8FEF785
:104B300013FE1298109044E040F60040C4F2024088
:104B400000688007002812D5FFE70E9803280ED1D1
:104B5000FFE740F60040C4F202400068C0F3C10124
:104B600049F20000C0F2D030C840109028E040F672
:104B70000040C4F202400068800500280AD5FFE723
:104B80000E98042806D1FFE740F60010C0F23D0061
:104B9000109014E040F6F040C4F202400068800734
:104BA000002808D5FFE70E98052804D1FFE74FF449
:104BB0000040109002E000201090FFE7FFE7FFE7C1
:104BC000FFE7FFE7FFE701F0BBBB40F6DC40C4F2C4
:104BD0000240006800F070000E900E9820B9FFE7C8
:104BE00003F0C4FA10906CE040F60040C4F20240BA
:104BF0000068000100280AD5FFE70E98102806D1AA
:104C0000FFE714A8FEF72CFC1598109058E040F62A
:104C10000040C4F202400068800000280AD5FFE787
:104C20000E98202806D1FFE711A8FEF795FD1298EF
:104C3000109044E040F60040C4F202400068800753
:104C4000002812D5FFE70E9830280ED1FFE740F676
:104C50000040C4F202400068C0F3C10149F2000004
:104C6000C0F2D030C840109028E040F60040C4F2B6
:104C700002400068800500280AD5FFE70E9840280A
:104C800006D1FFE740F60010C0F23D00109014E09E
:104C900040F6F040C4F2024000688007002808D5C2
:104CA000FFE70E98502804D1FFE74FF40040109022
:104CB00002E000201090FFE7FFE7FFE7FFE7FFE7D4
:104CC000FFE701F03DBB40F6E040C4F2024000685F
:104CD00000F0E0600E900E9820B9FFE703F06EFA46
:104CE00010905FE00E98B0F1807F06D1FFE714A826
:104CF000FEF7B6FB1598109053E00E98B0F1007FC8
:104D000006D1FFE711A8FEF727FD1298109047E0A3
:104D100040F60040C4F2024000688007002813D526
:104D2000FFE70E98B0F1407F0ED1FFE740F600405C
:104D3000C4F202400068C0F3C10149F20000C0F2B1
:104D4000D030C84010902AE040F60040C4F2024043
:104D50000068800500280BD5FFE70E98B0F1806F42
:104D600006D1FFE740F60010C0F23D00109015E0BC
:104D700040F6F040C4F2024000688007002809D5E0
:104D8000FFE70E98B0F1A06F04D1FFE74FF40040A9
:104D9000109002E000201090FFE7FFE7FFE7FFE739
:104DA000FFE7FFE701F0CCBA40F6E840C4F202406A
:104DB000006800F007000E900E9820B9FFE703F09E
:104DC000BBF910905AE00E98012804D1FFE703F0D8
:104DD00009FA109051E00E98022806D1FFE714A8B6
:104DE000FEF73EFB1698109046E040F60040C4F2F5
:104DF00002400068800300280AD5FFE70E980328C8
:104E000006D1FFE747F64000C0F27D10109032E077
:104E100040F60040C4F2024000688007002812D526
:104E2000FFE70E9804280ED1FFE740F60040C4F2D9
:104E300002400068C0F3C10149F20000C0F2D03066
:104E4000C840109016E040F60040C4F202400068EE
:104E5000800500280AD5FFE70E98052806D1FFE750
:104E600040F60010C0F23D00109002E000201090CB
:104E7000FFE7FFE7FFE7FFE7FFE7FFE701F060BAC3
:104E800040F6E840C4F20240006800F008000E90CE
:104E900040F6F040C4F2024000688007002807D5C1
:104EA000FFE70E9820B9FFE74FF40040109014E0A0
:104EB00040F6F040C4F2024000680001002808D526
:104EC000FFE70E98082804D1FFE74FF4FA4010904E
:104ED00002E000201090FFE7FFE701F031BA40F652
:104EE000E440C4F20240006800F440300E900E9896
:104EF00020B9FFE703F03AF9109040E00E98B0F5C2
:104F0000803F06D1FFE711A8FEF726FC139810900A
:104F100034E040F60040C4F20240006880070028F8
:104F200013D5FFE70E98B0F5003F0ED1FFE740F62E
:104F30000040C4F202400068C0F3C10149F2000021
:104F4000C0F2D030C840109017E040F60040C4F2E4
:104F500002400068800500280BD5FFE70E98B0F5E9
:104F6000403F06D1FFE740F60010C0F23D00109030
:104F700002E000201090FFE7FFE7FFE7FFE701F006
:104F8000DFB940F6E440C4F20240006800F440207B
:104F90000E900E9820B9FFE703F0E8F8109040E07B
:104FA0000E98B0F5802F06D1FFE711A8FEF7D4FBCD
:104FB0001398109034E040F60040C4F202400068BC
:104FC0008007002813D5FFE70E98B0F5002F0ED10B
:104FD000FFE740F60040C4F202400068C0F3C101A0
:104FE00049F20000C0F2D030C840109017E040F6FF
:104FF0000040C4F202400068800500280BD5FFE79E
:105000000E98B0F5402F06D1FFE740F60010C0F231
:105010003D00109002E000201090FFE7FFE7FFE75F
:10502000FFE701F08DB940F6E440C4F202400068A9
:1050300000F440100E900E9820B9FFE703F0BEF880
:10504000109040E00E98B0F5801F06D1FFE711A840
:10505000FEF782FB1398109034E040F60040C4F253
:10506000024000688007002813D5FFE70E98B0F5CE
:10507000001F0ED1FFE740F60040C4F20240006876
:10508000C0F3C10149F20000C0F2D030C840109016
:1050900017E040F60040C4F2024000688005002896
:1050A0000BD5FFE70E98B0F5401F06D1FFE740F69D
:1050B0000010C0F23D00109002E000201090FFE7C9
:1050C000FFE7FFE7FFE701F03BB940F6E440C4F239
:1050D0000240006800F440000E900E9820B9FFE7EF
:1050E00003F06CF8109040E00E98B0F5800F06D1F8
:1050F000FFE711A8FEF730FB1398109034E040F65C
:105100000040C4F2024000688007002813D5FFE782
:105110000E98B0F5000F0ED1FFE740F60040C4F244
:1051200002400068C0F3C10149F20000C0F2D03073
:10513000C840109017E040F60040C4F202400068FA
:10514000800500280BD5FFE70E98B0F5400F06D17B
:10515000FFE740F60010C0F23D00109002E0002092
:105160001090FFE7FFE7FFE7FFE701F0E9B840F63F
:10517000E440C4F20240006800F040700E900E98C7
:1051800020B9FFE702F0F2FF10902BE00E98B0F18B
:10519000807F06D1FFE711A8FEF7DEFA1398109082
:1051A0001FE040F60040C4F202400068800700287B
:1051B00013D5FFE70E98B0F1007F0ED1FFE740F660
:1051C0000040C4F202400068C0F3C10149F200008F
:1051D000C0F2D030C840109002E000201090FFE7ED
:1051E000FFE7FFE701F0ACB840F6DC40C4F2024054
:1051F000006800F4E0600E900E980990C8B1FFE7D7
:105200000998B0F5807F18D0FFE70998B0F5007FC6
:1052100019D0FFE70998B0F5407F1AD0FFE7099849
:10522000B0F5806F26D0FFE70998B0F5A06F32D0B7
:1052300081E002F0C3FF109080E014A8FEF710F99F
:10524000149810907AE011A8FEF786FA139810903F
:1052500074E040F6F040C4F2024000688007002885
:1052600004D5FFE74FF40040109002E000201090BA
:10527000FFE763E040F6F040C4F20240006800013E
:10528000002804D5FFE74FF4FA40109002E0002018
:105290001090FFE752E040F6E840C4F20240006898
:1052A00000F040400F9040F60040C4F20240006819
:1052B0008007002811D5FFE70F9870B9FFE740F687
:1052C0000040C4F202400068C0F3C10149F200008E
:1052D000C0F2D030C84010902CE040F60040C4F23C
:1052E00002400068800500280BD5FFE70F98B0F159
:1052F000804F06D1FFE740F60010C0F23D0010904D
:1053000017E040F60040C4F2024000688003002825
:105310000BD5FFE70F98B0F1004F06D1FFE747F636
:105320004000C0F27D10109002E000201090FFE7D6
:10533000FFE7FFE702E000201090FFE701F000B870
:1053400040F6DC40C4F20240006800F4E0400E90F9
:105350000E980890C8B1FFE70898B0F5805F18D0A4
:10536000FFE70898B0F5005F19D0FFE70898B0F59F
:10537000405F1AD0FFE70898B0F5804F26D0FFE7CE
:105380000898B0F5A04F32D081E002F0EFFE109007
:1053900080E014A8FEF764F8149810907AE011A841
:1053A000FEF7DAF91398109074E040F6F040C4F27A
:1053B000024000688007002804D5FFE74FF4004052
:1053C000109002E000201090FFE763E040F6F0400C
:1053D000C4F2024000680001002804D5FFE74FF442
:1053E000FA40109002E000201090FFE752E040F6F3
:1053F000E840C4F20240006800F040400F9040F6E0
:105400000040C4F2024000688007002811D5FFE781
:105410000F9870B9FFE740F60040C4F20240006800
:10542000C0F3C10149F20000C0F2D030C840109072
:105430002CE040F60040C4F20240006880050028DD
:105440000BD5FFE70F98B0F1804F06D1FFE740F68C
:105450000010C0F23D00109017E040F60040C4F28A
:1054600002400068800300280BD5FFE70F98B0F1D9
:10547000004F06D1FFE747F64000C0F27D101090C4
:1054800002E000201090FFE7FFE7FFE702E00020C6
:105490001090FFE700F054BF40F6DC40C4F2024039
:1054A000006800F4E0200E900E980790C8B1FFE766
:1054B0000798B0F5803F18D0FFE70798B0F5003F98
:1054C00019D0FFE70798B0F5403F1AD0FFE70798DB
:1054D000B0F5802F26D0FFE70798B0F5A02F32D087
:1054E00081E002F06BFE109080E014A8FDF7B8FF99
:1054F000149810907AE011A8FEF72EF913981090E6
:1055000074E040F6F040C4F20240006880070028D2
:1055100004D5FFE74FF40040109002E00020109007
:10552000FFE763E040F6F040C4F20240006800018B
:10553000002804D5FFE74FF4FA40109002E0002065
:105540001090FFE752E040F6E840C4F202400068E5
:1055500000F040400F9040F60040C4F20240006866
:105560008007002811D5FFE70F9870B9FFE740F6D4
:105570000040C4F202400068C0F3C10149F20000DB
:10558000C0F2D030C84010902CE040F60040C4F289
:1055900002400068800500280BD5FFE70F98B0F1A6
:1055A000804F06D1FFE740F60010C0F23D0010909A
:1055B00017E040F60040C4F2024000688003002873
:1055C0000BD5FFE70F98B0F1004F06D1FFE747F684
:1055D0004000C0F27D10109002E000201090FFE724
:1055E000FFE7FFE702E000201090FFE700F0A8BE11
:1055F00040F6DC40C4F20240006800F4E0000E9087
:105600000E980690C8B1FFE70698B0F5801F18D035
:10561000FFE70698B0F5001F19D0FFE70698B0F530
:10562000401F1AD0FFE70698B0F5800F26D0FFE79D
:105630000698B0F5A00F32D081E002F0BFFD1090C7
:1056400080E014A8FDF70CFF149810907AE011A8E0
:10565000FEF782F81398109074E040F6F040C4F220
:10566000024000688007002804D5FFE74FF400409F
:10567000109002E000201090FFE763E040F6F04059
:10568000C4F2024000680001002804D5FFE74FF48F
:10569000FA40109002E000201090FFE752E040F640
:1056A000E840C4F20240006800F040400F9040F62D
:1056B0000040C4F2024000688007002811D5FFE7CF
:1056C0000F9870B9FFE740F60040C4F2024000684E
:1056D000C0F3C10149F20000C0F2D030C8401090C0
:1056E0002CE040F60040C4F202400068800500282B
:1056F0000BD5FFE70F98B0F1804F06D1FFE740F6DA
:105700000010C0F23D00109017E040F60040C4F2D7
:1057100002400068800300280BD5FFE70F98B0F126
:10572000004F06D1FFE747F64000C0F27D10109011
:1057300002E000201090FFE7FFE7FFE702E0002013
:105740001090FFE700F0FCBD40F6DC40C4F20240E0
:10575000006800F0E0600E900E980590C8B1FFE779
:105760000598B0F1807F18D0FFE70598B0F1007F71
:1057700019D0FFE70598B0F1407F1AD0FFE70598F0
:10578000B0F1806F26D0FFE70598B0F1A06F32D05E
:1057900081E002F013FD109080E014A8FDF760FE98
:1057A000149810907AE011A8FDF7D6FF1398109086
:1057B00074E040F6F040C4F2024000688007002820
:1057C00004D5FFE74FF40040109002E00020109055
:1057D000FFE763E040F6F040C4F2024000680001D9
:1057E000002804D5FFE74FF4FA40109002E00020B3
:1057F0001090FFE752E040F6E840C4F20240006833
:1058000000F040400F9040F60040C4F202400068B3
:105810008007002811D5FFE70F9870B9FFE740F621
:105820000040C4F202400068C0F3C10149F2000028
:10583000C0F2D030C84010902CE040F60040C4F2D6
:1058400002400068800500280BD5FFE70F98B0F1F3
:10585000804F06D1FFE740F60010C0F23D001090E7
:1058600017E040F60040C4F20240006880030028C0
:105870000BD5FFE70F98B0F1004F06D1FFE747F6D1
:105880004000C0F27D10109002E000201090FFE771
:10589000FFE7FFE702E000201090FFE700F050BDB7
:1058A00040F6DC40C4F20240006800F0E0400E9098
:1058B0000E980490C8B1FFE70498B0F1805F18D04B
:1058C000FFE70498B0F1005F19D0FFE70498B0F14A
:1058D000405F1AD0FFE70498B0F1804F26D0FFE771
:1058E0000498B0F1A04F32D081E002F067FC109034
:1058F00080E014A8FDF7B4FD149810907AE011A888
:10590000FDF72AFF1398109074E040F6F040C4F2BF
:10591000024000688007002804D5FFE74FF40040EC
:10592000109002E000201090FFE763E040F6F040A6
:10593000C4F2024000680001002804D5FFE74FF4DC
:10594000FA40109002E000201090FFE752E040F68D
:10595000E840C4F20240006800F040400F9040F67A
:105960000040C4F2024000688007002811D5FFE71C
:105970000F9870B9FFE740F60040C4F2024000689B
:10598000C0F3C10149F20000C0F2D030C84010900D
:105990002CE040F60040C4F2024000688005002878
:1059A0000BD5FFE70F98B0F1804F06D1FFE740F627
:1059B0000010C0F23D00109017E040F60040C4F225
:1059C00002400068800300280BD5FFE70F98B0F174
:1059D000004F06D1FFE747F64000C0F27D1010905F
:1059E00002E000201090FFE7FFE7FFE702E0002061
:1059F0001090FFE700F0A4BC40F6E840C4F202407B
:105A0000006800F440700E9040F60040C4F202407E
:105A100000688003002809D5FFE70E9830B9FFE73A
:105A200047F64000C0F27D1010901AE00E98B0F5D5
:105A3000807F06D1FFE717A8FDF796FB1898109016
:105A40000EE00E98B0F5007F06D1FFE714A8FDF731
:105A500007FD1598109002E000201090FFE7FFE787
:105A6000FFE700F06DBC40F6E040C4F20240006881
:105A700000F007000E900E98039004286DD803994B
:105A8000DFE801F003090F151B0017A8FDF76CFBF9
:105A90001898109064E014A8FDF7E2FC1498109098
:105AA0005EE011A8FDF758FE1198109058E048F2FA
:105AB0000000C0F2BB00109052E040F6E840C4F293
:105AC0000240006800F040400F9040F60040C4F2F1
:105AD000024000688007002811D5FFE70F9870B9D1
:105AE000FFE740F60040C4F202400068C0F3C10185
:105AF00049F20000C0F2D030C84010902CE040F6CF
:105B00000040C4F202400068800500280BD5FFE782
:105B10000F98B0F1804F06D1FFE740F60010C0F2B9
:105B20003D00109017E040F60040C4F202400068CB
:105B3000800300280BD5FFE70F98B0F1004F06D186
:105B4000FFE747F64000C0F27D10109002E0002011
:105B50001090FFE7FFE7FFE702E000201090FFE76B
:105B600000F0EEBB40F6E040C4F20240006800F0F6
:105B700038000E900E980290202800F27C80029946
:105B8000DFE801F01179797979797979177979797B
:105B9000797979791D797979797979792379797927
:105BA00079797979290017A8FDF7DEFA189810900D
:105BB00064E014A8FDF754FC149810905EE011A85E
:105BC000FDF7CAFD1198109058E048F20000C0F2AD
:105BD000BB00109052E040F6E840C4F2024000687A
:105BE00000F040400F9040F60040C4F202400068D0
:105BF0008007002811D5FFE70F9870B9FFE740F63E
:105C00000040C4F202400068C0F3C10149F2000044
:105C1000C0F2D030C84010902CE040F60040C4F2F2
:105C200002400068800500280BD5FFE70F98B0F10F
:105C3000804F06D1FFE740F60010C0F23D00109003
:105C400017E040F60040C4F20240006880030028DC
:105C50000BD5FFE70F98B0F1004F06D1FFE747F6ED
:105C60004000C0F27D10109002E000201090FFE78D
:105C7000FFE7FFE702E000201090FFE760E340F657
:105C8000E040C4F20240006800F4E0700E900E980C
:105C9000019088B1FFE70198402813D0FFE70198F1
:105CA000802815D0FFE70198C02817D0FFE701989A
:105CB000B0F5807F18D067E017A8FDF755FA18985F
:105CC000109064E014A8FDF7CBFB149810905EE0F0
:105CD00011A8FDF741FD1198109058E048F200001E
:105CE000C0F2BB00109052E040F6E840C4F202401F
:105CF000006800F040400F9040F60040C4F20240BF
:105D000000688007002811D5FFE70F9870B9FFE7FA
:105D100040F60040C4F202400068C0F3C10149F2FD
:105D20000000C0F2D030C84010902CE040F6004097
:105D3000C4F202400068800500280BD5FFE70F98E9
:105D4000B0F1804F06D1FFE740F60010C0F23D00F1
:105D5000109017E040F60040C4F202400068800353
:105D600000280BD5FFE70F98B0F1004F06D1FFE7F1
:105D700047F64000C0F27D10109002E00020109025
:105D8000FFE7FFE7FFE702E000201090FFE7D7E220
:105D900040F6E040C4F20240006800F460600E90FB
:105DA0000E9820B9FFE702F0F5F9109073E040F685
:105DB0000040C4F202400068000100280BD5FFE754
:105DC0000E98B0F5007F06D1FFE714A8FDF748FB59
:105DD000159810905EE040F60040C4F20240006862
:105DE000800000280BD5FFE70E98B0F5806F06D134
:105DF000FFE711A8FDF7B0FC1298109049E040F6BB
:105E00000040C4F2024000688007002813D5FFE775
:105E10000E98B0F5C06F0ED1FFE740F60040C4F217
:105E200002400068C0F3C10149F20000C0F2D03066
:105E3000C84010902CE040F60040C4F202400068D8
:105E4000800500280BD5FFE70E98B0F5006F06D14E
:105E5000FFE740F60010C0F23D00109017E040F65A
:105E60000040C4F202400068800300280BD5FFE721
:105E70000E98B0F5206F06D1FFE747F64000C0F25C
:105E80007D10109002E000201090FFE7FFE7FFE791
:105E9000FFE7FFE7FFE753E240F6E040C4F20240CD
:105EA000006800F4E0400E900E9820B9FFE702F081
:105EB00085F9109073E040F60040C4F2024000689B
:105EC000000100280BD5FFE70E98B0F5805F06D1E2
:105ED000FFE714A8FDF7C4FA159810905EE040F6AD
:105EE0000040C4F202400068800000280BD5FFE7A4
:105EF0000E98B0F5005F06D1FFE711A8FDF72CFC66
:105F00001298109049E040F60040C4F20240006848
:105F10008007002813D5FFE70E98B0F5405F0ED13B
:105F2000FFE740F60040C4F202400068C0F3C10140
:105F300049F20000C0F2D030C84010902CE040F68A
:105F40000040C4F202400068800500280BD5FFE73E
:105F50000E98B0F5804F06D1FFE740F60010C0F272
:105F60003D00109017E040F60040C4F20240006887
:105F7000800300280BD5FFE70E98B0F5A04F06D19F
:105F8000FFE747F64000C0F27D10109002E00020CD
:105F90001090FFE7FFE7FFE7FFE7FFE7FFE7CFE14D
:105FA00040F6E040C4F20240006800F460300E9019
:105FB0000E9820B9FFE702F0EDF8109073E040F67C
:105FC0000040C4F202400068000100280BD5FFE742
:105FD0000E98B0F5004F06D1FFE714A8FDF740FA80
:105FE000159810905EE040F60040C4F20240006850
:105FF000800000280BD5FFE70E98B0F5803F06D152
:10600000FFE711A8FDF7A8FB1298109049E040F6B1
:106010000040C4F2024000688007002813D5FFE763
:106020000E98B0F5C03F0ED1FFE740F60040C4F235
:1060300002400068C0F3C10149F20000C0F2D03054
:10604000C84010902CE040F60040C4F202400068C6
:10605000800500280BD5FFE70E98B0F5003F06D16C
:10606000FFE740F60010C0F23D00109017E040F648
:106070000040C4F202400068800300280BD5FFE70F
:106080000E98B0F5203F06D1FFE747F64000C0F27A
:106090007D10109002E000201090FFE7FFE7FFE77F
:1060A000FFE7FFE7FFE74BE140F6E440C4F20240C0
:1060B000006800F003000E900E980090032864D84A
:1060C0000099DFE801F002060C1202F035F810909A
:1060D0005EE017A8FDF748F81898109058E014A84B
:1060E000FDF7BEF91698109052E040F6E840C4F271
:1060F0000240006800F040400F9040F60040C4F2BB
:10610000024000688007002811D5FFE70F9870B99A
:10611000FFE740F60040C4F202400068C0F3C1014E
:1061200049F20000C0F2D030C84010902CE040F698
:106130000040C4F202400068800500280BD5FFE74C
:106140000F98B0F1804F06D1FFE740F60010C0F283
:106150003D00109017E040F60040C4F20240006895
:10616000800300280BD5FFE70F98B0F1004F06D150
:10617000FFE747F64000C0F27D10109002E00020DB
:106180001090FFE7FFE7FFE702E000201090FFE735
:10619000D6E040F6E840C4F20240006800F0C000DB
:1061A0000E9040F6F040C4F20240006880070028DC
:1061B00007D5FFE70E9820B9FFE74FF40040109095
:1061C00026E040F6F040C4F20240006800010028DA
:1061D00008D5FFE70E98402804D1FFE74FF4FA40B6
:1061E000109014E040F60040C4F2024000688005C0
:1061F000002808D5FFE70E98802804D1FFE748F271
:106200001200109002E000201090FFE7FFE7FFE788
:1062100096E040F6E840C4F20240006800F030002A
:106220000E9040F60040C4F202400068800400284E
:1062300009D5FFE70E9830B9FFE746F60040C0F2F7
:10624000DC2010903AE040F60040C4F202400068C2
:10625000800100280AD5FFE70E98102806D1FFE735
:1062600017A8FCF781FF1898109026E040F6F04040
:10627000C4F2024000688007002808D5FFE70E98A6
:10628000202804D1FFE74FF40040109014E040F6BE
:10629000F040C4F2024000680001002808D5FFE782
:1062A0000E98302804D1FFE74FF4FA40109002E036
:1062B00000201090FFE7FFE7FFE7FFE740E040F630
:1062C000E440C4F20240006800F030000E900E98E6
:1062D000102806D1FFE717A8FCF746FF1898109082
:1062E0002EE040F60040C4F2024000688000002822
:1062F0000AD5FFE70E98202806D1FFE711A8FDF781
:106300002BFA1298109016E040F60040C4F20240BA
:106310000068800400280AD5FFE70E98302806D1CF
:10632000FFE746F60040C0F2DC20109002E00020BB
:106330001090FFE7FFE7FFE702E000201090FFE783
:10634000FFE710981CB080BD80B5ACB02B9000204A
:106350008DF8A3008DF8A2002B98C078C00760B11B
:10636000FFE740F6E841C4F20241086820F04040EF
:106370002B9A926D10430860FFE72B980068C007C6
:10638000002837D0FFE72B98C06D2790052817D835
:106390002799DFE801F003040B12131414E02B9883
:1063A000083004F0E7F98DF8A3000DE02B983030A9
:1063B00004F096FA8DF8A30006E005E004E003E09F
:1063C00001208DF8A300FFE79DF8A30060B9FFE767
:1063D00040F6D841C4F20241086820F007002B9A29
:1063E000D26D1043086004E09DF8A3008DF8A20070
:1063F000FFE7FFE72B9800788007002840F14A80EC
:10640000FFE72B98006E2690282829D82699DFE8E8
:1064100001F015272727272727271627272727278C
:1064200027271D2727272727272724272727272709
:1064300027272527272727272727260014E02B98FB
:10644000083004F097F98DF8A3000DE02B98303058
:1064500004F046FA8DF8A30006E005E004E003E04E
:1064600001208DF8A300FFE79DF8A30060B9FFE7C6
:1064700040F6D841C4F20241086820F038002B9A57
:10648000126E1043086004E09DF8A3008DF8A2008E
:10649000FFE7FFE72B9800784007002847D5FFE784
:1064A0002B98406E2590B0B1FFE72598402813D077
:1064B000FFE72598802816D0FFE72598C02819D037
:1064C000FFE72598B0F5807F15D0FFE72598B0F558
:1064D000A07F11D011E014E02B98083004F04AF9A5
:1064E0008DF8A3000DE02B98303004F0F9F98DF809
:1064F000A30006E005E004E003E001208DF8A3001E
:10650000FFE79DF8A30060B9FFE740F6D841C4F269
:106510000241086820F4E0702B9A526E1043086024
:1065200004E09DF8A3008DF8A200FFE7FFE72B9899
:106530000078000700284AD5FFE72B98806E24904A
:10654000C8B1FFE72498B0F5007F15D0FFE7249885
:10655000B0F5806F17D0FFE72498B0F5C06F19D061
:10656000FFE72498B0F5006F15D0FFE72498B0F549
:10657000206F11D011E014E02B98083004F0FAF8E5
:106580008DF8A3000DE02B98303004F0A9F98DF8B8
:10659000A30006E005E004E003E001208DF8A3007D
:1065A000FFE79DF8A30060B9FFE740F6D841C4F2C9
:1065B0000241086820F460602B9A926E10430860D4
:1065C00004E09DF8A3008DF8A200FFE7FFE72B98F9
:1065D0000078C00600284AD5FFE72B98C06E2390AC
:1065E000C8B1FFE72398B0F5805F15D0FFE7239887
:1065F000B0F5005F17D0FFE72398B0F5405F19D0E2
:10660000FFE72398B0F5804F15D0FFE72398B0F54A
:10661000A04F11D011E014E02B98083004F0AAF834
:106620008DF8A3000DE02B98303004F059F98DF867
:10663000A30006E005E004E003E001208DF8A300DC
:10664000FFE79DF8A30060B9FFE740F6D841C4F228
:106650000241086820F4E0402B9AD26E1043086093
:1066600004E09DF8A3008DF8A200FFE7FFE72B9858
:106670000078800600284AD5FFE72B98006F22900B
:10668000C8B1FFE72298B0F5004F15D0FFE7229878
:10669000B0F5803F17D0FFE72298B0F5C03F19D082
:1066A000FFE72298B0F5003F15D0FFE72298B0F53C
:1066B000203F11D011E014E02B98083004F05AF874
:1066C0008DF8A3000DE02B98303004F009F98DF817
:1066D000A30006E005E004E003E001208DF8A3003C
:1066E000FFE79DF8A30060B9FFE740F6D841C4F288
:1066F0000241086820F460302B9A126F1043086042
:1067000004E09DF8A3008DF8A200FFE7FFE72B98B7
:106710000078400600284AD5FFE72B98406F21906B
:10672000C8B1FFE72198B0F5802F15D0FFE7219879
:10673000B0F5002F17D0FFE72198B0F5402F19D002
:10674000FFE72198B0F5801F15D0FFE72198B0F53D
:10675000A01F11D011E014E02B98083004F00AF8C3
:106760008DF8A3000DE02B98303004F0B9F88DF8C7
:10677000A30006E005E004E003E001208DF8A3009B
:10678000FFE79DF8A30060B9FFE740F6D841C4F2E7
:106790000241086820F4E0102B9A526F1043086001
:1067A00004E09DF8A3008DF8A200FFE7FFE72B9817
:1067B0000078000600284AD5FFE72B98806F2090CC
:1067C000C8B1FFE72098B0F5001F15D0FFE720986B
:1067D000B0F5800F17D0FFE72098B0F5C00F19D0A3
:1067E000FFE72098B0F5000F15D0FFE72098B0F52F
:1067F000200F11D011E014E02B98083003F0BAFFFD
:106800008DF8A3000DE02B98303004F069F88DF876
:10681000A30006E005E004E003E001208DF8A300FA
:10682000FFE79DF8A30060B9FFE740F6D841C4F246
:106830000241086820F460002B9A926F10430860B0
:1068400004E09DF8A3008DF8A200FFE7FFE72B9876
:106850004078C00700284AD0FFE72B98C06F1F90F0
:10686000C8B1FFE71F98B0F1807F15D0FFE71F98F0
:10687000B0F1007F17D0FFE71F98B0F1407F19D02B
:10688000FFE71F98B0F1806F15D0FFE71F98B0F1B8
:10689000A06F11D011E014E02B98083003F06AFFCC
:1068A0008DF8A3000DE02B98303004F019F88DF826
:1068B000A30006E005E004E003E001208DF8A3005A
:1068C000FFE79DF8A30060B9FFE740F6D841C4F2A6
:1068D0000241086820F0E0602B9AD26F10430860F4
:1068E00004E09DF8A3008DF8A200FFE7FFE72B98D6
:1068F0004078800700284CD5FFE72B98D0F880001F
:106900001E90C8B1FFE71E98B0F1006F15D0FFE7E9
:106910001E98B0F1805F17D0FFE71E98B0F1C05FFE
:1069200019D0FFE71E98B0F1005F15D0FFE71E9861
:10693000B0F1205F11D011E014E02B98083003F083
:1069400019FF8DF8A3000DE02B98303003F0C8FF3D
:106950008DF8A30006E005E004E003E001208DF8D7
:10696000A300FFE79DF8A30068B9FFE740F6D84110
:10697000C4F20241086820F060502B9AD2F88020BF
:106980001043086004E09DF8A3008DF8A200FFE723
:10699000FFE72B9840784007002839D5FFE72B9870
:1069A000D0F884001D90052817D81D99DFE801F064
:1069B00003040B12131414E02B98083003F0DAFED2
:1069C0008DF8A3000DE02B98303003F089FF8DF88F
:1069D000A30006E005E004E003E001208DF8A30039
:1069E000FFE79DF8A30068B9FFE740F6DC41C4F279
:1069F0000241086820F007002B9AD2F88420104347
:106A0000086004E09DF8A3008DF8A200FFE7FFE70F
:106A10002B9840780007002847D5FFE72B98D0F83F
:106A200088001C90A0B1FFE71C98102811D0FFE748
:106A30001C98202814D0FFE71C98302817D0FFE7B7
:106A40001C98402814D0FFE71C98502811D011E062
:106A500014E02B98083003F08DFE8DF8A3000DE0B4
:106A60002B98303003F03CFF8DF8A30006E005E0E2
:106A700004E003E001208DF8A300FFE79DF8A300E8
:106A800068B9FFE740F6DC41C4F20241086820F033
:106A900070002B9AD2F888201043086004E09DF81B
:106AA000A3008DF8A200FFE7FFE72B984078C0060F
:106AB00000284CD5FFE72B98D0F88C001B90C8B16C
:106AC000FFE71B98B0F1807F15D0FFE71B98B0F16E
:106AD000007F17D0FFE71B98B0F1407F19D0FFE788
:106AE0001B98B0F1806F15D0FFE71B98B0F1A06F35
:106AF00011D011E014E02B98083003F03BFE8DF824
:106B0000A3000DE02B98303003F0EAFE8DF8A300CF
:106B100006E005E004E003E001208DF8A300FFE7B4
:106B20009DF8A30068B9FFE740F6E041C4F20241D6
:106B3000086820F0E0602B9AD2F88C20104308609F
:106B400004E09DF8A3008DF8A200FFE7FFE72B9873
:106B50004078800600283AD5FFE72B98D0F89000BF
:106B60001A9078B1FFE71A98B0F5803F0BD0FFE795
:106B70001A98B0F5003F0DD0FFE71A98B0F5403FE6
:106B800009D009E00CE02B98303003F0A9FE8DF815
:106B9000A30005E004E003E001208DF8A300FFE777
:106BA0009DF8A30068B9FFE740F6E441C4F2024152
:106BB000086820F440302B9AD2F8902010430860E7
:106BC00004E09DF8A3008DF8A200FFE7FFE72B98F3
:106BD0004078400600283AD5FFE72B98D0F894007B
:106BE000199078B1FFE71998B0F5802F0BD0FFE727
:106BF0001998B0F5002F0DD0FFE71998B0F5402F88
:106C000009D009E00CE02B98303003F069FE8DF8D4
:106C1000A30005E004E003E001208DF8A300FFE7F6
:106C20009DF8A30068B9FFE740F6E441C4F20241D1
:106C3000086820F440202B9AD2F894201043086072
:106C400004E09DF8A3008DF8A200FFE7FFE72B9872
:106C50004078000600283AD5FFE72B98D0F8980036
:106C6000189078B1FFE71898B0F5801F0BD0FFE7B8
:106C70001898B0F5001F0DD0FFE71898B0F5401F29
:106C800009D009E00CE02B98303003F029FE8DF894
:106C9000A30005E004E003E001208DF8A300FFE776
:106CA0009DF8A30068B9FFE740F6E441C4F2024151
:106CB000086820F440102B9AD2F8982010430860FE
:106CC00004E09DF8A3008DF8A200FFE7FFE72B98F2
:106CD0004079400700283AD5FFE72B98D0F89C0070
:106CE000179078B1FFE71798B0F5800F0BD0FFE74A
:106CF0001798B0F5000F0DD0FFE71798B0F5400FCB
:106D000009D009E00CE02B98303003F0E9FD8DF854
:106D1000A30005E004E003E001208DF8A300FFE7F5
:106D20009DF8A30068B9FFE740F6E441C4F20241D0
:106D3000086820F440002B9AD2F89C201043086089
:106D400004E09DF8A3008DF8A200FFE7FFE72B9871
:106D50008078C007A0B3FFE72B98D0F8A00016906A
:106D600050B1FFE71698B0F1807F06D0FFE7169884
:106D7000B0F1007F08D008E00BE02B98303003F032
:106D8000AFFD8DF8A30004E003E001208DF8A3001F
:106D9000FFE79DF8A30068B9FFE740F6E441C4F2BD
:106DA0000241086820F040702B9AD2F8A0201043CE
:106DB000086004E09DF8A3008DF8A200FFE7FFE75C
:106DC0002B9840790007002811D5FFE7FFE740F630
:106DD0001C41C4F20241086820F4004008602B986E
:106DE000D0F80421086810430860FFE7FFE72B98FC
:106DF0008078800700284CD5FFE72B98D0F8A400B6
:106E00001590C8B1FFE71598B0F5807F15D0FFE762
:106E10001598B0F5007F17D0FFE71598B0F5407FC3
:106E200019D0FFE71598B0F5806F15D0FFE71598DA
:106E3000B0F5A06F11D011E014E02B98083003F0EA
:106E400099FC8DF8A3000DE02B98303003F048FD3D
:106E50008DF8A30006E005E004E003E001208DF8D2
:106E6000A300FFE79DF8A30068B9FFE740F6DC4107
:106E7000C4F20241086820F4E0602B9AD2F8A42002
:106E80001043086004E09DF8A3008DF8A200FFE71E
:106E9000FFE72B988078400700284CD5FFE72B9818
:106EA000D0F8A8001490C8B1FFE71498B0F5805F3F
:106EB00015D0FFE71498B0F5005F17D0FFE71498DE
:106EC000B0F5405F19D0FFE71498B0F5804F15D0AA
:106ED000FFE71498B0F5A04F11D011E014E02B9803
:106EE000083003F047FC8DF8A3000DE02B983030FC
:106EF00003F0F6FC8DF8A30006E005E004E003E0F3
:106F000001208DF8A300FFE79DF8A30068B9FFE713
:106F100040F6DC41C4F20241086820F4E0402B9ABC
:106F2000D2F8A8201043086004E09DF8A3008DF873
:106F3000A200FFE7FFE72B980079800600284CD5D8
:106F4000FFE72B98D0F8AC001390C8B1FFE7139877
:106F5000B0F5803F15D0FFE71398B0F5003F17D08C
:106F6000FFE71398B0F5403F19D0FFE71398B0F54D
:106F7000802F15D0FFE71398B0F5A02F11D011E0A6
:106F800014E02B98083003F0F5FB8DF8A3000DE01A
:106F90002B98303003F0A4FC8DF8A30006E005E048
:106FA00004E003E001208DF8A300FFE79DF8A300B3
:106FB00068B9FFE740F6DC41C4F20241086820F4FA
:106FC000E0202B9AD2F8AC201043086004E09DF832
:106FD000A3008DF8A200FFE7FFE72B980079400699
:106FE00000284CD5FFE72B98D0F8B0001290C8B11C
:106FF000FFE71298B0F5801F15D0FFE71298B0F5A3
:10700000001F17D0FFE71298B0F5401F19D0FFE717
:107010001298B0F5800F15D0FFE71298B0F5A00FC9
:1070200011D011E014E02B98083003F0A3FB8DF889
:10703000A3000DE02B98303003F052FC8DF8A30034
:1070400006E005E004E003E001208DF8A300FFE77F
:107050009DF8A30068B9FFE740F6DC41C4F20241A5
:10706000086820F4E0002B9AD2F8B02010430860A2
:1070700004E09DF8A3008DF8A200FFE7FFE72B983E
:107080000079000600284CD5FFE72B98D0F8B40013
:107090001190C8B1FFE71198B0F1807F15D0FFE7DC
:1070A0001198B0F1007F17D0FFE71198B0F1407F41
:1070B00019D0FFE71198B0F1806F15D0FFE7119854
:1070C000B0F1A06F11D011E014E02B98083003F05C
:1070D00051FB8DF8A3000DE02B98303003F000FC3D
:1070E0008DF8A30006E005E004E003E001208DF840
:1070F000A300FFE79DF8A30068B9FFE740F6DC4175
:10710000C4F20241086820F0E0602B9AD2F8B42063
:107110001043086004E09DF8A3008DF8A200FFE78B
:10712000FFE72B984079C00700284CD0FFE72B9849
:10713000D0F8B8001090C8B1FFE71098B0F1805FA8
:1071400015D0FFE71098B0F1005F17D0FFE7109857
:10715000B0F1405F19D0FFE71098B0F1804F15D023
:10716000FFE71098B0F1A04F11D011E014E02B9878
:10717000083003F0FFFA8DF8A3000DE02B983030B3
:1071800003F0AEFB8DF8A30006E005E004E003E0A9
:1071900001208DF8A300FFE79DF8A30068B9FFE781
:1071A00040F6DC41C4F20241086820F0E0402B9A2E
:1071B000D2F8B8201043086004E09DF8A3008DF8D1
:1071C000A200FFE7FFE72B988078000700284ED544
:1071D000FFE72B98D0F8C0000F90A0B1FFE70F9801
:1071E000B0F5803F18D0FFE70F98B0F5003F1AD0F8
:1071F000FFE70F98B0F5403F1CD0FFE70F98B0F5C0
:10720000802F18D018E040F62841C4F202410868E7
:1072100040F40030086013E02B98083003F0AAFA1D
:107220008DF8A3000CE02B98303003F059FB8DF85B
:10723000A30005E004E003E001208DF8A300FFE7D0
:107240009DF8A30068B9FFE740F6E841C4F20241A7
:10725000086820F4E0202B9AD2F8C0201043086080
:1072600004E09DF8A3008DF8A200FFE7FFE72B984C
:107270008078C00600284DD5FFE72B98D0F8C400D1
:107280000E90A0B1FFE70E98B0F5002F18D0FFE7E1
:107290000E98B0F5801F1AD0FFE70E98B0F5C01F0A
:1072A0001CD0FFE70E98B0F5001F17D017E040F68E
:1072B0002841C4F20241086840F40030086012E03E
:1072C0002B98083003F056FA8DF8A3000BE02B98AA
:1072D000303003F005FB8DF8A30004E003E001204B
:1072E0008DF8A300FFE79DF8A30068B9FFE740F61B
:1072F000E841C4F20241086820F460102B9AD2F8E9
:10730000C4201043086004E09DF8A3008DF8A2009B
:10731000FFE7FFE72B9880788006002834D5FFE749
:107320002B98D0F8D4000D90022809D3FFE70D98D0
:10733000022806D0FFE70D980338032808D308E099
:107340000BE02B98083003F015FA8DF8A30004E049
:1073500003E001208DF8A300FFE79DF8A30068B9C2
:10736000FFE740F6E841C4F20241086820F0070058
:107370002B9AD2F8D4201043086004E09DF8A300B3
:107380008DF8A200FFE7FFE72B98407980070028DF
:1073900027D5FFE72B98D0F8D8000C9020B1FFE755
:1073A0000C98082801D001E004E003E001208DF8EA
:1073B000A300FFE79DF8A30068B9FFE740F6E841A6
:1073C000C4F20241086820F008002B9AD2F8D820B5
:1073D0001043086004E09DF8A3008DF8A200FFE7C9
:1073E000FFE72B98C0788007002840F1B580FFE7C1
:1073F00040F62401C4F20241086840F00100086030
:10740000FBF7DAFD2990FFE740F62400C4F20240C2
:107410000068C00760B9FFE7FBF7CEFD2999401A65
:10742000032804D3FFE703208DF8A30000E0EBE777
:107430009DF8A300002840F08980FFE740F6F04067
:10744000C4F20240006800F440702A902A98D0B13B
:10745000FFE72A982B99D1F8F810884213D0FFE75C
:1074600040F6F041C4F20241086820F440702A90CE
:10747000086840F480300860086820F480300860B4
:107480002A980860FFE79DF8A800C007E0B1FFE771
:10749000FBF792FD2990FFE740F6F040C4F202406E
:1074A0000068800700280ED4FFE7FBF785FD2999C7
:1074B000401A41F28931884204D3FFE703208DF856
:1074C000A30000E0E8E7FFE79DF8A300C0BBFFE7EB
:1074D000FFE72B98D0F8F80000F44070B0F5407F3B
:1074E00013D1FFE740F61C41C4F20241086820F4C2
:1074F0007C502B9AD2F8F8204FF6F043C0F6FF7379
:107500001A4040EA1210086008E040F61C41C4F23C
:107510000241086820F47C500860FFE740F6F04123
:10752000C4F20241086820F4407008602B98D0F83B
:10753000F8206FF31F32086810430860FFE704E08B
:107540009DF8A3008DF8A200FFE704E09DF8A300DA
:107550008DF8A200FFE7FFE72B98C07840070028CE
:1075600039D5FFE72B98D0F8C8000B9060B1FFE742
:107570000B98102809D0FFE70B9820280ED0FFE7C2
:107580000B9830280BD00BE00EE040F62841C4F2F7
:107590000241086840F40030086005E004E003E0C0
:1075A00001208DF8A300FFE79DF8A30068B9FFE76D
:1075B00040F6E841C4F20241086820F030002B9AFE
:1075C000D2F8C8201043086004E09DF8A3008DF8AD
:1075D000A200FFE7FFE72B9880784006002835D50A
:1075E000FFE72B98D0F8CC000A9020B1FFE70A986B
:1075F000402809D00FE040F62841C4F20241086853
:1076000040F4003008600AE02B98083003F0B2F82C
:107610008DF8A30003E001208DF8A300FFE79DF89B
:10762000A30068B9FFE740F6E441C4F202410868EC
:1076300020F040002B9AD2F8CC201043086004E0E0
:107640009DF8A3008DF8A200FFE7FFE72B98807854
:107650000006002835D5FFE72B98D0F8D000099018
:1076600020B1FFE70998802809D00FE040F62841B3
:10767000C4F20241086840F4003008600AE02B9828
:10768000083003F077F88DF8A30003E001208DF8AF
:10769000A300FFE79DF8A30068B9FFE740F6E441C7
:1076A000C4F20241086820F080002B9AD2F8D02062
:1076B0001043086004E09DF8A3008DF8A200FFE7E6
:1076C000FFE72B98C0780007002840D5FFE72B98EC
:1076D000D0F8E000089004281ED80899DFE801F0EF
:1076E000030C131A1B0040F62841C4F2024108683B
:1076F00040F40030086013E02B98083003F03AF8AB
:107700008DF8A3000CE02B98303003F0E9F88DF8E9
:10771000A30005E004E003E001208DF8A300FFE7EB
:107720009DF8A30068B9FFE740F6E041C4F20241CA
:10773000086820F007002B9AD2F8E0201043086078
:1077400004E09DF8A3008DF8A200FFE7FFE72B9867
:10775000C078C006002840F14F80FFE72B98D0F892
:10776000E400079020282CD80799DFE801F0112ABF
:107770002A2A2A2A2A2A1A2A2A2A2A2A2A2A212A82
:107780002A2A2A2A2A2A282A2A2A2A2A2A2A290086
:1077900040F62841C4F20241086840F40030086015
:1077A00013E02B98083002F0E5FF8DF8A3000CE001
:1077B0002B98303003F094F88DF8A30005E004E036
:1077C00003E001208DF8A300FFE79DF8A30068B94E
:1077D000FFE740F6E041C4F20241086820F03800BB
:1077E0002B9AD2F8E4201043086004E09DF8A3002F
:1077F0008DF8A200FFE7FFE72B98C07880060028ED
:107800004BD5FFE72B98D0F8E800069088B1FFE74A
:107810000698402816D0FFE70698802819D0FFE781
:107820000698C0281CD0FFE70698B0F5807F18D0D6
:1078300018E040F62841C4F20241086840F40030E4
:10784000086013E02B98083002F094FF8DF8A30035
:107850000CE02B98303003F043F88DF8A30005E0DE
:1078600004E003E001208DF8A300FFE79DF8A300EA
:1078700068B9FFE740F6E041C4F20241086820F42D
:10788000E0702B9AD2F8E8201043086004E09DF8DD
:10789000A3008DF8A200FFE7FFE72B98C078400611
:1078A00000284CD5FFE72B98D0F8EC000590C8B124
:1078B000FFE70598B0F5007F15D0FFE70598B0F514
:1078C000806F17D0FFE70598B0F5C06F19D0FFE7BC
:1078D0000598B0F5006F15D0FFE70598B0F5206F5B
:1078E00011D011E014E02B98083002F043FF8DF81E
:1078F000A3000DE02B98303002F0F2FF8DF8A300CA
:1079000006E005E004E003E001208DF8A300FFE7B6
:107910009DF8A30068B9FFE740F6E041C4F20241D8
:10792000086820F460602B9AD2F8EC2010430860BD
:1079300004E09DF8A3008DF8A200FFE7FFE72B9875
:10794000C078000600284CD5FFE72B98D0F8F0004F
:107950000490C8B1FFE70498B0F5805F15D0FFE749
:107960000498B0F5005F17D0FFE70498B0F5405FCA
:1079700019D0FFE70498B0F5804F15D0FFE70498C1
:10798000B0F5A04F11D011E014E02B98083002F0B0
:10799000F1FE8DF8A3000DE02B98303002F0A0FF2F
:1079A0008DF8A30006E005E004E003E001208DF877
:1079B000A300FFE79DF8A30068B9FFE740F6E041A8
:1079C000C4F20241086820F4E0402B9AD2F8F0207B
:1079D0001043086004E09DF8A3008DF8A200FFE7C3
:1079E000FFE72B980079C00700284CD0FFE72B98C1
:1079F000D0F8F4000390C8B1FFE70398B0F5004F4A
:107A000015D0FFE70398B0F5803F17D0FFE7039844
:107A1000B0F5C03F19D0FFE70398B0F5003F15D08F
:107A2000FFE70398B0F5203F11D011E014E02B9848
:107A3000083002F09FFE8DF8A3000DE02B98303047
:107A400002F04EFF8DF8A30006E005E004E003E03D
:107A500001208DF8A300FFE79DF8A30068B9FFE7B8
:107A600040F6E041C4F20241086820F460302B9AED
:107A7000D2F8F4201043086004E09DF8A3008DF8CC
:107A8000A200FFE7FFE72B9800798007002838D590
:107A9000FFE72B98D0F8DC000290032816D8029953
:107AA000DFE801F002030C1314E040F62841C4F2B1
:107AB0000241086840F4003008600BE02B98083061
:107AC00002F058FE8DF8A30004E003E001208DF8D9
:107AD000A300FFE79DF8A30068B9FFE740F6E44183
:107AE000C4F20241086820F003002B9AD2F8DC208F
:107AF0001043086004E09DF8A3008DF8A200FFE7A2
:107B0000FFE72B980079400700283CD5FFE72B982A
:107B1000D0F8BC00019050B1FFE70198B0F5807F2C
:107B200006D0FFE70198B0F5007F0AD010E013E01F
:107B300040F62841C4F20241086840F40030086071
:107B40000AE02B98083002F015FE8DF8A30003E040
:107B500001208DF8A300FFE79DF8A30068B9FFE7B7
:107B600040F6E841C4F20241086820F440702B9AC4
:107B7000D2F8BC201043086004E09DF8A3008DF803
:107B8000A200FFE7FFE72B980079C00600283BD54D
:107B9000FFE72B98D0F800010090102808D0FFE7ED
:107BA000009820280DD0FFE70098302810D010E072
:107BB00040F62841C4F20241086840F400300860F1
:107BC0000BE02B98303002F08BFE8DF8A30004E020
:107BD00003E001208DF8A300FFE79DF8A30068B93A
:107BE000FFE740F6E441C4F20241086820F03000AB
:107BF0002B9AD2F800211043086004E09DF8A300FE
:107C00008DF8A200FFE7FFE72B9800790007002816
:107C10000DD5FFE740F6E841C4F20241086820F0C4
:107C2000C0002B9AD2F8FC2010430860FFE79DF8B3
:107C3000A2002CB080BD000080B586B004900391F6
:107C4000049820B9FFE701208DF817003AE2039865
:107C500042F20001C4F20201096801F00F018842FA
:107C600016D9FFE742F20000C4F20200016821F0D9
:107C70000F01039A11430160006800F00F0003999F
:107C8000884204D0FFE701208DF817001AE2FFE7D1
:107C900004980078C00600281BD5FFE704984069C7
:107CA00040F62041C4F20241096801F4E041B0EB22
:107CB000112F0DD9FFE740F62041C4F202410868B8
:107CC00020F4E040049A526940EA02200860FFE78D
:107CD000FFE704980078000700281BD5FFE7049809
:107CE000006940F62041C4F20241096801F4E061F4
:107CF000B0EB111F0DD9FFE740F62041C4F202415D
:107D0000086820F4E060049A126940EA02100860F2
:107D1000FFE7FFE7049800784007002819D5FFE740
:107D20000498C06840F62041C4F20241096801F09D
:107D3000700188420CD9FFE740F62041C4F20241AD
:107D4000086820F07000049AD26810430860FFE7CA
:107D5000FFE7049800788007002819D5FFE704980A
:107D6000806840F62041C4F20241096801F00F0129
:107D700088420CD9FFE740F62041C4F2024108686E
:107D800020F00F00049A926810430860FFE7FFE7B5
:107D900004980078C007002800F0D180FFE704981D
:107DA000406803280ED1FFE740F60040C4F20240CD
:107DB00000688001002804D4FFE701208DF8170037
:107DC00080E135E00498406802280ED1FFE740F6D4
:107DD0000040C4F2024000688003002804D4FFE79A
:107DE00001208DF817006DE121E00498406801281A
:107DF0000ED1FFE740F60040C4F202400068800563
:107E0000002804D4FFE701208DF817005AE10DE0A7
:107E100040F60040C4F2024000688007002804D405
:107E2000FFE701208DF817004CE1FFE7FFE7FFE7D0
:107E300040F61C41C4F20241086820F00300049A95
:107E4000526810430860FBF7B7F801900498406847
:107E500003281AD1FFE7FFE740F61C40C4F20240B6
:107E6000006800F0180018280ED0FFE7FBF7A4F810
:107E70000199401A41F28931884204D3FFE7032077
:107E80008DF817001EE1E7E758E0049840680228E3
:107E90001AD1FFE7FFE740F61C40C4F20240006839
:107EA00000F0180010280ED0FFE7FBF785F80199C5
:107EB000401A41F28931884204D3FFE703208DF84C
:107EC0001700FFE0E7E738E00498406801281AD17E
:107ED000FFE7FFE740F61C40C4F20240006800F0F4
:107EE000180008280ED0FFE7FBF766F80199401A42
:107EF00041F28931884204D3FFE703208DF817004F
:107F0000E0E0E7E718E0FFE740F61C40C4F202407B
:107F1000006810F0180F0ED0FFE7FBF74DF801993D
:107F2000401A41F28931884204D3FFE703208DF8DB
:107F30001700C7E0E8E7FFE7FFE7FFE7FFE7049880
:107F400000788007002819D5FFE70498806840F67C
:107F50002041C4F20241096801F00F0188420CD2AD
:107F6000FFE740F62041C4F20241086820F00F000C
:107F7000049A926810430860FFE7FFE7039842F213
:107F80000001C4F20201096801F00F01884216D213
:107F9000FFE742F20000C4F20200016821F00F0185
:107FA000039A11430160006800F00F0003998842B2
:107FB00004D0FFE701208DF8170083E0FFE7049865
:107FC00000784007002819D5FFE70498C06840F6FC
:107FD0002041C4F20241096801F0700188420CD2CC
:107FE000FFE740F62041C4F20241086820F070002B
:107FF000049AD26810430860FFE7FFE7049800780E
:10800000000700281BD5FFE70498006940F62041CF
:10801000C4F20241096801F4E061B0EB111F0DD216
:10802000FFE740F62041C4F20241086820F4E06016
:10803000049A126940EA02100860FFE7FFE704981B
:108040000078C00600281BD5FFE70498406940F679
:108050002041C4F20241096801F4E041B0EB112F64
:108060000DD2FFE740F62041C4F20241086820F437
:10807000E040049A526940EA02200860FFE7FFE707
:1080800000F0B0F840F62041C4F20241096801F066
:108090000F024DF68241C0F60001895CC84040F2F3
:1080A0000001C2F20001086040F20C00C2F20000C0
:1080B0000068FAF7C5FF8DF80B009DF80B008DF8EE
:1080C0001700FFE79DF8170006B080BD83B002904F
:1080D000019102991F20086040F61C40C4F2024042
:1080E000006800F003000299486040F62040C4F2A6
:1080F000024000680090009800F00F00029988602C
:10810000009800F070000299C860009800F4E060E8
:10811000000902990861009800F4E040000A029901
:10812000486142F20000C4F20200006800F00F0053
:108130000199086003B0704780B500F053F840F62D
:108140002041C4F20241096801F00F024DF682415C
:10815000C0F60001895C01F01F0120FA01F140F234
:108160000000C2F200000160006880BD80B5FFF72A
:10817000E3FF40F62041C4F202410968C1F3021254
:108180004DF69241C0F60001895C01F01F01C84024
:1081900080BD000080B5FFF7CFFF40F62041C4F25C
:1081A00002410968C1F302224DF69241C0F6000176
:1081B000895C01F01F01C84080BD000080B5FFF759
:1081C000BBFF40F62041C4F202410968C1F302320C
:1081D0004DF69241C0F60001895C01F01F01C840D4
:1081E00080BD000089B040F61C40C4F20240006827
:1081F00000F01800082806D1FFE740F60010C0F292
:108200003D00049048E140F61C40C4F20240006882
:1082100010F0180F21D1FFE740F60040C4F20240F1
:10822000006800F020010020B0EB511F0ED0FFE7E6
:1082300040F60040C4F202400068C0F3C10149F2B8
:108240000000C0F2D030C840049005E049F20000C0
:10825000C0F2D0300490FFE71DE140F61C40C4F2AC
:108260000240006800F01800102806D1FFE747F62A
:108270004000C0F27D1004900CE140F61C40C4F2B6
:108280000240006800F01800182840F0FC80FFE76A
:1082900040F62840C4F20240016801F00301089151
:1082A0000168C1F3052106910068C0F30010059034
:1082B000059840F63841C4F20241096889B2C908FC
:1082C00000FB01F000EE100AB8EE400A8DED020A44
:1082D0000698002800F0D380FFE708980090012856
:1082E00009D0FFE70098022800F08D80FFE7009892
:1082F000032864D088E040F60040C4F202400068E1
:1083000000F020010020B0EB511F33D0FFE740F612
:108310000040C4F202400068C0F3C10149F200000D
:10832000C0F2D030C84003909DED030AB8EE400A79
:108330009DED061AB8EE411A80EE010A40F634406F
:10834000C4F2024000686FF35F2001EE100AB8EE3D
:10835000411A9DED022A9FED533A82EE032A31EE37
:10836000021AB7EE002A31EE021A20EE010A8DED54
:10837000010A23E09DED060AB8EE401A9FED4A0A75
:1083800080EE010A40F63440C4F2024000686FF308
:108390005F2001EE100AB8EE411A9DED022A9FED12
:1083A000413A82EE032A31EE021AB7EE002A31EE8C
:1083B000021A20EE010A8DED010AFFE748E09DED6B
:1083C000060AB8EE401A9FED360A80EE010A40F622
:1083D0003440C4F2024000686FF35F2001EE100ADF
:1083E000B8EE411A9DED022A9FED2E3A82EE032A45
:1083F00031EE021AB7EE002A31EE021A20EE010A1F
:108400008DED010A24E0FFE79DED060AB8EE401A63
:108410009FED260A80EE010A40F63440C4F2024085
:1084200000686FF35F2001EE100AB8EE411A9DED6F
:10843000022A9FED1C3A82EE032A31EE021AB7EEB1
:10844000002A31EE021A20EE010A8DED010AFFE743
:1084500040F63440C4F20240006881B2012000EBD3
:10846000512007909DED010A9DED071AB8EE411AC3
:1084700080EE010ABCEEC00A8DED040A02E0002085
:108480000490FFE705E049F20000C0F2D03004900C
:10849000FFE7FFE7FFE7FFE7049809B0704700BF79
:1084A00020BCBE4B000000460024744C0024744ADB
:1084B00080B588B00690069828B9FFE701208DF8AE
:1084C0001F0000F0EFBC40F61C40C4F20240006800
:1084D00000F01800049040F62840C4F20240006802
:1084E00000F00300039006980078C006002840F1D1
:1084F0008080FFE70498082808D0FFE70498182830
:108500001DD1FFE70398022819D1FFE70698C0693B
:1085100028B9FFE701208DF81F0000F0C3BCFFE77A
:1085200040F61841C4F20241086820F47C10069A13
:10853000126A40EA02400860FFE7FFE758E0069849
:10854000C06988B3FFE740F60041C4F20241086801
:1085500040F480700860FAF72FFD0590FFE740F6C1
:108560000040C4F202400068800500280DD4FFE7F7
:10857000FAF722FD0599401A032805D3FFE70320E7
:108580008DF81F0000F08EBCE9E7FFE740F61841C8
:10859000C4F20241086820F47C10069A126A40EA8C
:1085A00002400860FFE722E040F60041C4F20241C9
:1085B000086820F480700860FAF7FEFC0590FFE779
:1085C00040F60040C4F202400068800500280DD546
:1085D000FFE7FAF7F1FC0599401A032805D3FFE7F6
:1085E00003208DF81F0000F05DBCE9E7FFE7FFE71F
:1085F000FFE706980078C007002800F0B980FFE781
:108600000498102808D0FFE7049818280ED1FFE737
:10861000039803280AD1FFE70698406828B9FFE7C6
:1086200001208DF81F0000F03DBCA0E0FFE7069898
:108630004068B0F5803F09D1FFE740F60041C4F241
:108640000241086840F48030086056E006984068AF
:1086500088B9FFE740F60041C4F20241086820F4FF
:1086600080300860086820F480100860086820F4F2
:108670008020086040E006984068B0F5A02F11D136
:10868000FFE740F60041C4F20241086840F4802050
:108690000860086820F480100860086840F48030A2
:1086A000086028E006984068B0F5A81F11D1FFE7E0
:1086B00040F60041C4F20241086840F4802008609E
:1086C000086840F480100860086840F48030086052
:1086D00010E040F60041C4F20241086820F4803006
:1086E0000860086820F480200860086820F4801082
:1086F0000860FFE7FFE7FFE7FFE7FFE7069840684E
:10870000D0B1FFE7FAF758FC0590FFE740F60040CC
:10871000C4F202400068800300280CD4FFE7FAF797
:108720004BFC0599401A652804D3FFE703208DF818
:108730001F00B7E3EAE719E0FAF73EFC0590FFE710
:1087400040F60040C4F202400068800300280CD5C7
:10875000FFE7FAF731FC0599401A652804D3FFE7D3
:1087600003208DF81F009DE3EAE7FFE7FFE7FFE73F
:10877000069800788007002840F1C380FFE704983E
:1087800040B1FFE7049818285ED1FFE7039801285D
:108790005AD1FFE70698C06820B9FFE701208DF89D
:1087A0001F007FE3049840BBFFE740F60040C4F29F
:1087B0000240006800F018000699096988421BD041
:1087C000FFE740F60041C4F20241086820F01800BB
:1087D000069A126910430860FFF7AEFC40F20C00E5
:1087E000C2F200000068FAF72BFC20B1FFE701207D
:1087F0008DF81F0056E3FFE7FFE7FAF7DDFB059072
:10880000FFE740F60040C4F20240006880070028FD
:108810000CD4FFE7FAF7D0FB0599401A032804D3DC
:10882000FFE703208DF81F003CE3EAE740F6104124
:10883000C4F20241086820F4FE00069A526940EA38
:1088400002400860FFE75BE00698C068A8B3FFE756
:1088500040F60041C4F20241086820F01800069A70
:10886000126910430860086840F001000860FAF7D8
:10887000A3FB0590FFE740F60040C4F20240006809
:10888000800700280CD4FFE7FAF796FB0599401AF9
:10889000032804D3FFE703208DF81F0002E3EAE773
:1088A00040F61041C4F20241086820F4FE00069A26
:1088B000526940EA0240086021E040F60041C4F2FB
:1088C0000241086820F001000860FAF775FB059086
:1088D000FFE740F60040C4F202400068800700282D
:1088E0000CD5FFE7FAF768FB0599401A032804D373
:1088F000FFE703208DF81F00D4E2EAE7FFE7FFE778
:10890000FFE7069800780007002849D5FFE706989A
:10891000806910B3FFE740F6F041C4F202410868F5
:1089200040F080600860FAF747FB0590FFE740F6EB
:10893000F040C4F202400068000100280CD4FFE7B8
:10894000FAF73AFB0599401A032804D3FFE70320FE
:108950008DF81F00A6E2EAE721E040F6F041C4F2FC
:108960000241086820F080600860FAF725FB059056
:10897000FFE740F6F040C4F2024000680001002822
:108980000CD5FFE7FAF718FB0599401A032804D322
:10899000FFE703208DF81F0084E2EAE7FFE7FFE727
:1089A000069800784007002840F1CC80FFE740F6A9
:1089B0002400C4F202400068C00708BBFFE740F68D
:1089C0002401C4F20241086840F001000860FAF78F
:1089D000F3FA0590FFE740F62400C4F20240006875
:1089E000C00760B9FFE7FAF7E7FA0599401A0328CC
:1089F00004D3FFE703208DF81F0053E2EBE7FFE706
:108A0000FFE706988068012809D1FFE740F6F041AA
:108A1000C4F20241086840F00100086054E0069882
:108A2000806888B9FFE740F6F041C4F20241086867
:108A300020F001000860086820F0800008600868E5
:108A400020F0040008603EE006988068052811D1F7
:108A5000FFE740F6F041C4F20241086840F004002C
:108A60000860086820F080000860086840F0010095
:108A7000086027E006988068852811D1FFE740F656
:108A8000F041C4F20241086840F004000860086840
:108A900040F080000860086840F00100086010E0C5
:108AA00040F6F041C4F20241086820F0010008607D
:108AB000086820F004000860086820F08000086062
:108AC000FFE7FFE7FFE7FFE7FFE706988068E0B111
:108AD000FFE7FAF771FA0590FFE740F6F040C4F2BD
:108AE00002400068800700280ED4FFE7FAF764FA16
:108AF0000599401A41F28931884204D3FFE70320E7
:108B00008DF81F00CEE1E8E71BE0FAF755FA059073
:108B1000FFE740F6F040C4F20240006880070028FA
:108B20000ED5FFE7FAF748FA0599401A41F2893164
:108B3000884204D3FFE703208DF81F00B2E1E8E785
:108B4000FFE7FFE7069800788006002849D5FFE791
:108B50000698406A10B3FFE740F60041C4F20241B4
:108B6000086840F480500860FAF726FA0590FFE79D
:108B700040F60040C4F202400068800400280CD493
:108B8000FFE7FAF719FA0599401A032804D3FFE71B
:108B900003208DF81F0085E1EAE721E040F600415F
:108BA000C4F20241086820F480500860FAF704FA21
:108BB0000590FFE740F60040C4F2024000688004E0
:108BC00000280CD5FFE7FAF7F7F90599401A0328B2
:108BD00004D3FFE703208DF81F0063E1EAE7FFE716
:108BE000FFE70698806A002800F05881FFE70498A4
:108BF000182800F0D580FFE70698806A022840F028
:108C0000A180FFE740F60041C4F20241086820F06D
:108C100080700860FAF7D0F90590FFE740F6004051
:108C2000C4F202400068800100280CD5FFE7FAF783
:108C3000C3F90599401A032804D3FFE703208DF8F0
:108C40001F002FE1EAE7FFE740F62841C4F20241A6
:108C5000086843F603729043069BDA6A1B6B42EA8C
:108C60000322104308600699486BD1F838C0CB6BDB
:108C70000A6C01386FF35F204FF60061CFF6FF7189
:108C800001EB4C2189B208440021CFF6FF7101EBC2
:108C9000034101F4FE0108444FF07F4101EB026102
:108CA00001F0FE41084440F63441C4F2024108603C
:108CB000FFE740F62841C4F202410091086820F025
:108CC000100008600698C06CC00040F63842C4F23C
:108CD00002421060086840F010000860086820F048
:108CE0000C00069A526C10430860086820F02000BF
:108CF000069A926C10430860086840F4803008605F
:108D000040F60041C4F20241086840F080700860FB
:108D1000FAF752F90590FFE740F60040C4F202402E
:108D20000068800100280CD4FFE7FAF745F905999F
:108D3000401A032804D3FFE703208DF81F00B1E099
:108D4000EAE72CE040F60041C4F20241086820F056
:108D500080700860FAF730F90590FFE740F60040B0
:108D6000C4F202400068800100280CD5FFE7FAF742
:108D700023F90599401A032804D3FFE703208DF84F
:108D80001F008FE0EAE740F62841C4F2024108687C
:108D90004FF6FC72CFF6F87210400860FFE77CE0F7
:108DA00040F62840C4F202400068029040F6344089
:108DB000C4F20240006801900698806A012837D00A
:108DC000FFE7029800F003000699C96A88422FD194
:108DD000FFE7029800F47C510698006BB0EB112F6E
:108DE00026D1FFE701986FF35F200699496B01399F
:108DF00088421DD1FFE7BDF804100698806B01384A
:108E0000B0EB512F14D1FFE7019800F4FE01069852
:108E1000C06B0138B0EB114F0AD1FFE7019800F0A9
:108E2000FE410698006C0138B0EB116F04D0FFE7EB
:108E300001208DF81F0035E040F63840C4F20240B2
:108E4000006881B20698C06CB0EBD10F24D0FFE768
:108E500040F62841C4F20241086820F01000086082
:108E6000FAF7AAF80590FFE7FAF7A6F80599401A6D
:108E700008B9FFE7F8E70698C06CC00040F6384133
:108E8000C4F20241086040F62841C4F20241086879
:108E900040F010000860FFE7FFE7FFE700208DF8D3
:108EA0001F00FFE79DF81F0008B080BD82B0019051
:108EB00001980090042843D80099DFE801F00C1DC8
:108EC0002F4103004EF21001CEF20001086840F07D
:108ED0000400086035E04EF21001CEF2000108688F
:108EE00020F00400086040F6E441C4F20241086842
:108EF00020F00C00086024E04EF21001CEF20001D8
:108F0000086820F00400086040F6E441C4F2024121
:108F10000868012262F38300086012E04EF210013B
:108F2000CEF20001086820F00400086040F6E44139
:108F3000C4F202410868022262F38300086000E084
:108F4000FFE702B07047000081B0009001B07047A9
:108F500081B0009001B0704781B0009001B07047BF
:108F600081B0009001B0704781B0009001B07047AF
:108F700081B0009001B0704781B0009001B070479F
:108F800080B582B00090009820B9FFE701208DF8ED
:108F9000070045E0009890F83D0040B9FFE70099D0
:108FA000002081F83C00009800F03EF8FFE70099AF
:108FB000022081F83D00009951F8040B01F04EFEAB
:108FC0000099012081F84800FFE70099012081F80D
:108FD0003E00009981F83F00009981F84000009917
:108FE00081F84100009981F84200009981F843001E
:108FF000FFE7FFE70099012081F84400009981F81C
:109000004500009981F84600009981F84700FFE784
:109010000099012081F83D0000208DF80700FFE74E
:109020009DF8070002B080BD81B0009001B070478C
:1090300083B00190019890F83D00012804D0FFE72B
:1090400001208DF80B00B8E00199022081F83D0065
:1090500001980168C86840F00100C8600198006884
:1090600042F60041C4F20101884200F08280FFE72D
:109070000198006842F60041C5F20101884278D0AB
:10908000FFE701980068B0F1804F72D0FFE70198C8
:109090000068B0F1A04F6CD0FFE70198006840F283
:1090A0000041C4F20001884263D0FFE701980068E4
:1090B00040F20041C5F2000188425AD0FFE7019812
:1090C000006840F60001C4F20001884251D0FFE779
:1090D0000198006840F60001C5F20001884248D0BE
:1090E000FFE70198006840F60041C4F200018842A1
:1090F0003FD0FFE70198006840F60041C5F200014B
:10910000884236D0FFE70198006843F20041C4F27C
:10911000010188422DD0FFE70198006843F2004129
:10912000C5F20101884224D0FFE70198006841F6AA
:109130000001C4F2000188421BD0FFE701980068DB
:1091400041F60001C5F20001884212D0FFE7019804
:10915000006844F20001C4F20101884209D0FFE72F
:109160000198006844F20001C5F20101884219D15A
:10917000FFE70198006880680721C0F201010840FC
:109180000090009806280CD0FFE70098B0F5803FCB
:1091900007D0FFE701980168086840F00100086007
:1091A000FFE706E001980168086840F001000860E8
:1091B000FFE700208DF80B00FFE79DF80B0003B0E0
:1091C0007047000081B0009001B0704780B584B056
:1091D000039003980068C0680290039800680069D3
:1091E00001909DF804008007002824D5FFE79DF832
:1091F0000800800700281DD5FFE7039801686FF07D
:1092000002000861039901200877039800688069CB
:10921000800720B1FFE70398FFF7D4FF06E003982B
:1092200000F054F9039800F055F9FFE70399002086
:109230000877FFE7FFE79DF804004007002825D5E1
:10924000FFE79DF80800400700281ED5FFE70398B8
:1092500001686FF004000861039902200877039801
:109260000068806910F4407F04D0FFE70398FFF79F
:10927000A9FF06E0039800F029F9039800F02AF905
:10928000FFE7039900200877FFE7FFE79DF8040058
:109290000007002824D5FFE79DF8080000070028F4
:1092A0001DD5FFE7039801686FF008000861039976
:1092B0000420087703980068C069800720B1FFE7A1
:1092C0000398FFF77FFF06E0039800F0FFF803988C
:1092D00000F000F9FFE7039900200877FFE7FFE7B8
:1092E0009DF80400C006002825D5FFE79DF808007A
:1092F000C00600281ED5FFE7039801686FF0100034
:10930000086103990820087703980068C06910F481
:10931000407F04D0FFE70398FFF754FF06E003986F
:1093200000F0D4F8039800F0D5F8FFE70399002087
:109330000877FFE7FFE79DF80400C00778B1FFE773
:109340009DF80800C00748B1FFE7039801686FF077
:1093500001000861039800F0C1F8FFE7FFE70198FA
:1093600000F08000802806D0FFE79DF80500800609
:10937000002810D5FFE79DF808000006002809D551
:10938000FFE7039801686FF4025008610398FFF744
:10939000DFFDFFE7FFE79DF80500C00780B1FFE7AD
:1093A0009DF808000006002809D5FFE7039801682A
:1093B0006FF4807008610398FFF7C6FDFFE7FFE7D1
:1093C0009DF804004006002810D5FFE79DF808002E
:1093D0004006002809D5FFE7039801686FF04000B8
:1093E0000861039800F08CF8FFE7FFE79DF80400A0
:1093F0008006002810D5FFE79DF8080080060028A9
:1094000009D5FFE7039801686FF020000861039811
:10941000FFF7A2FDFFE7FFE79DF80600C006002862
:1094200010D5FFE79DF80A00C006002809D5FFE720
:10943000039801686FF4801008610398FFF794FDAA
:10944000FFE7FFE79DF806008006002810D5FFE73C
:109450009DF80A008006002809D5FFE703980168F7
:109460006FF4001008610398FFF77AFDFFE7FFE74C
:109470009DF806004006002810D5FFE79DF80A0079
:109480004006002809D5FFE7039801686FF48000C3
:1094900008610398FFF76CFDFFE7FFE79DF8060002
:1094A0000006002810D5FFE79DF80A0000060028F6
:1094B00009D5FFE7039801686FF40000086103987D
:1094C000FFF75AFDFFE7FFE704B080BD81B00090D1
:1094D00001B0704781B0009001B0704780B582B094
:1094E00001900198006842F60041C4F201018842EF
:1094F00003D1FFE7F9F766FDFFE702B080BD00008A
:1095000081B0009001B0704783B00190FFE70198EF
:1095100090F88400012804D1FFE702208DF80B00A9
:109520002CE00199012081F88400FFE7FFE7019911
:109530002420C1F888000198006800680090019814
:109540000168086820F001000860009820F00050D1
:109550000090019900204866009801990968086008
:1095600001992020C1F88800FFE70199002081F8C7
:109570008400FFE700208DF80B00FFE79DF80B004B
:1095800003B0704780B586B004900391ADF80A200F
:109590000498D0F88C00202844D1FFE7039820B12C
:1095A000FFE7BDF80A0020B9FFE701208DF817009A
:1095B0003CE004990120C8660499002008670498DB
:1095C0000399BDF80A2002F0EBFE8DF809009DF822
:1095D000090010BBFFE70498C06E012818D1FFE70F
:1095E0000498016810200862FFE7FFE7049800680C
:1095F00050E8000F40F010000190FFE70199049837
:10960000026842E800100028F0D1FFE7FFE703E01E
:1096100001208DF80900FFE7FFE79DF809008DF8AC
:10962000170003E002208DF81700FFE79DF81700F0
:1096300006B080BD80B584B00390ADF80A100398E1
:10964000006844F20041C4F20001884228D1FFE7DB
:10965000BDF80A2040F27000C2F20000009040F213
:10966000E901C2F200010191F7F710F8009A01999F
:10967000BDF80A300020D054012082F8500040F696
:109680003C40C2F20000C822FFF77CFF40F6F41015
:10969000C2F200000168486920F400704861FFE7E9
:1096A00004B080BD81B0009001B0704780B584B037
:1096B00002900191FFE7029890F88400012804D1FC
:1096C000FFE702208DF80F0032E00299012081F8B7
:1096D0008400FFE7FFE702992420C1F88800029880
:1096E00000680068009002980168086820F0010096
:1096F000086002980068806820F060600199084363
:10970000029909688860029801F056FC0098029955
:109710000968086002992020C1F88800FFE70299D3
:10972000002081F88400FFE700208DF80F00FFE79C
:109730009DF80F0004B080BD80B584B00290019107
:10974000FFE7029890F88400012804D1FFE7022087
:109750008DF80F0032E00299012081F88400FFE7C4
:10976000FFE702992420C1F8880002980068006889
:10977000009002980168086820F0010008600298D3
:109780000068806820F060400199084302990968E8
:109790008860029801F010FC00980299096808603E
:1097A00002992020C1F88800FFE70299002081F883
:1097B0008400FFE700208DF80F00FFE79DF80F0001
:1097C00004B080BD81B0009001B0704781B00090BE
:1097D00001B0704780B586B00490FFE7FFE70498BA
:1097E000006850E8000F20F490700390FFE70399A1
:1097F0000498026842E800100028F0D1FFE7FFE774
:10980000FFE7FFE70498006850E8020F4FF6FE718B
:10981000CEF6FF7108400290FFE7029904980268B3
:1098200042E802100028EDD1FFE7FFE70498C06E80
:10983000012814D1FFE7FFE7FFE70498006850E82C
:10984000000F20F010000190FFE7019904980268D2
:1098500042E800100028F0D1FFE7FFE7FFE7049897
:10986000006880684006002824D5FFE70498D0F8F7
:109870008000F0B1FFE70498D0F880100020C8669F
:109880000498D0F88000F8F76FFD88B1FFE70498DE
:10989000D0F88000F8F758FE102808D1FFE70499A7
:1098A0001020C1F8900003208DF8170019E0FFE7A1
:1098B000FFE7FFE704990020A1F85E0004990A6819
:1098C0000F21116204990A68916941F008019161C0
:1098D000049A2021C2F88C100499C8668DF81700EC
:1098E000FFE79DF8170006B080BD000081B0009032
:1098F00001B0704780B58EB00D900D980068C069BA
:109900000C900D98006800680B900D9800688068B6
:109910000A900C9840F60F01084009900998E0B9A8
:10992000FFE79DF830008006002815D5FFE79DF879
:109930002C008006002806D4FFE79DF82B00C00607
:10994000002809D5FFE70D98406F20B1FFE70D987B
:10995000416F8847FFE76CE2FFE70998002800F0B5
:10996000F980FFE70A980121C1F20001084209D1FC
:10997000FFE70B9840F22011C0F20041084200F0CE
:10998000E980FFE79DF83000C00788B1FFE79DF848
:109990002D00C00760B1FFE70D9801680120086243
:1099A0000D99D1F8900040F00100C1F89000FFE758
:1099B0009DF830008007002811D5FFE79DF82800AA
:1099C000C00760B1FFE70D980168022008620D9999
:1099D000D1F8900040F00400C1F89000FFE79DF836
:1099E00030004007002811D5FFE79DF82800C00788
:1099F00060B1FFE70D980168042008620D99D1F865
:109A0000900040F00200C1F89000FFE79DF83000A0
:109A10000007002819D5FFE79DF82C0080060028D4
:109A200007D4FFE70A980121C1F2000108420CD0D7
:109A3000FFE70D980168082008620D99D1F89000A1
:109A400040F00800C1F89000FFE79DF831000007E2
:109A5000002813D5FFE79DF82F00400700280DD5FB
:109A6000FFE70D9801684FF4006008620D99D1F886
:109A7000900040F02000C1F89000FFE70D98D0F86A
:109A80009000002865D0FFE79DF830008006002890
:109A900015D5FFE79DF82C008006002806D4FFE7C7
:109AA0009DF82B00C006002809D5FFE70D98406FF0
:109AB00020B1FFE70D98416F8847FFE7FFE70D985A
:109AC000D0F8900008900D980068806800F0400081
:109AD000402806D0FFE79DF8200010F0280F2FD077
:109AE000FFE70D9801F000FD0D98006880684006C2
:109AF000002820D5FFE70D98D0F88000B0B1FFE72F
:109B00000D98D0F880104BF2D520C0F60000C86642
:109B10000D98D0F88000F8F7B3FC30B1FFE70D984E
:109B2000D0F88000C16E8847FFE703E00D98FFF78B
:109B3000DDFEFFE703E00D98FFF7D8FEFFE707E043
:109B40000D98FFF7D3FE0D990020C1F89000FFE7B4
:109B5000FFE76EE10D98C06E012840F00B81FFE732
:109B60009DF83000C006002840F10481FFE79DF811
:109B70002C00C006002840F1FD80FFE70D98016829
:109B8000102008620D98006880684006002840F1A7
:109B90008F80FFE70D98D0F880000068806CADF8EA
:109BA0001E00BDF81E00002867D0FFE7BDF81E00AC
:109BB0000D99B1F85C1088425FDAFFE7BDF81E002E
:109BC0000D99A1F85E000D98D0F88000006D8128F5
:109BD00046D0FFE7FFE7FFE70D98006850E8000F69
:109BE00020F480700690FFE706990D98026842E81D
:109BF00000100028F0D1FFE7FFE7FFE7FFE70D982F
:109C0000006850E8020F20F001000590FFE7059979
:109C10000D98026842E802100028F0D1FFE7FFE744
:109C20000D992020C1F88C000D990020C866FFE72F
:109C3000FFE70D98006850E8000F20F01000049036
:109C4000FFE704990D98026842E800100028F0D15F
:109C5000FFE7FFE70D98D0F88000F8F785FBFFE7F6
:109C60000D99022008670D98B0F85C10B0F85E20DE
:109C7000891A89B2FFF7DEFC19E0BDF81E000D99C4
:109C8000B1F85C10884211D1FFE70D98D0F8800040
:109C9000006D812809D1FFE70D99022008670D9812
:109CA000B0F85C10FFF7C6FCFFE7FFE7FFE7C0E096
:109CB0000D99B1F85C00B1F85E10401AADF80E00D5
:109CC0000D98B0F85E00002853D0FFE7BDF80E00F5
:109CD00000284ED0FFE7FFE7FFE70D98006850E847
:109CE000000F20F490700290FFE702990D9802682F
:109CF00042E800100028F0D1FFE7FFE7FFE7FFE7A9
:109D00000D98006850E8020F4FF6FE71CEF6FF7115
:109D100008400190FFE701990D98026842E802109F
:109D20000028EDD1FFE7FFE70D992020C1F88C0056
:109D30000D990020C8660D994867FFE7FFE70D9869
:109D4000006850E8000F20F010000090FFE7009935
:109D50000D98026842E800100028F0D1FFE7FFE705
:109D60000D99022008670D98BDF80E10FFF762FCF0
:109D7000FFE75EE09DF83200C00600280FD5FFE740
:109D80009DF82A004006002809D5FFE70D980168D4
:109D90004FF4801008620D98FFF718FD49E09DF818
:109DA00030000006002815D5FFE79DF82C000006BE
:109DB000002806D4FFE79DF82A000006002809D5F0
:109DC000FFE70D98806F20B1FFE70D98816F8847FE
:109DD000FFE72EE09DF83000400600280AD5FFE797
:109DE0009DF82C004006002804D5FFE70D9801F0EF
:109DF000CBFB1EE09DF83200000600280AD5FFE7E5
:109E00009DF82F004006002804D5FFE70D98FFF7C6
:109E1000D9FC0EE09DF83300C00750B1FFE79DF874
:109E20002F000006002804D5FFE70D98FFF73AFC45
:109E3000FFE70EB080BD000080B582B000900098B2
:109E400020B9FFE701208DF8070046E000988069FF
:109E500008B1FFE700E0FFE70098D0F8880040B9BC
:109E6000FFE70099002081F88400009800F03AF89C
:109E7000FFE700992420C1F888000098016808686D
:109E800020F0010008600098806A20B1FFE7009888
:109E900001F0D8F8FFE7009802F076F8012804D125
:109EA000FFE701208DF8070017E000980168486877
:109EB00020F49040486000980168886820F02A00EB
:109EC000886000980168086840F001000860009808
:109ED00001F05CF98DF80700FFE79DF8070002B07C
:109EE00080BD000080B5EEB06D9000206C906B904E
:109EF0006A90699068904DA86C21F6F736FC0AA824
:109F00004FF48471F6F731FC6D98006843F6000158
:109F1000C4F20101884240F0FF80FFE700200B906F
:109F200001210A9121900AA8FCF70EFA18B1FFE767
:109F3000F7F764FDFFE7FFE740F6A440C4F20240F4
:109F4000016841F480410160006800F4804009909C
:109F50000998FFE7FFE740F68C40C4F20240016831
:109F600041F002010160006800F0020008900898CA
:109F7000FFE74FF440406890022069900020059070
:109F80006A906B9004206C9040F20040C4F2022072
:109F900068A9F8F79BFE059821214D9115214E9156
:109FA0004F9050905190529053905490012156915F
:109FB00057914FF04021589159905A905E905B9084
:109FC0005C9040F28821C2F200014DA8F7F732FD03
:109FD00018B1FFE7F7F712FDFFE740F24C20C2F29D
:109FE000000040F28822C2F200020021F7F712FFBF
:109FF00018B1FFE7F7F702FDFFE740F24C20C2F28D
:10A000000000F8F7A7F818B1FFE7F7F7F7FCFFE74C
:10A0100040F6E420C2F2000040F2D021C4F2020176
:10A02000016000218163C1634FF400320264416426
:10A0300081218164F7F72CFD18B1FFE7F7F7DEFC0B
:10A04000FFE740F6E420C2F2000040F24C21C2F2E9
:10A050000001F7F7ADFF18B1FFE7F7F7CFFCFFE717
:10A06000FFE76D9840F6E421C2F20001C0F88010CD
:10A070006D98C865FFE740F6E420C2F200001021A9
:10A08000F8F728FA18B1FFE7F7F7B8FCFFE740F652
:10A090006C20C2F20000039040F25021C4F2020191
:10A0A0000160162141600021049181604FF48062BB
:10A0B000C2600822026141618161C16101620122C5
:10A0C00042628262C16201634163F8F7ADFB18B17D
:10A0D000FFE7F7F793FCFFE7FFE76D9840F66C2189
:10A0E000C2F20001C1676D98C865FFE740F66C20B9
:10A0F000C2F200001021F8F7EDF918B1FFE7F7F709
:10A100007DFCFFE73A20029000221146F9F70CF897
:10A110000298F8F7FFFFC7E06D98006844F200412D
:10A12000C4F20001884240F0BE80FFE700200B909F
:10A1300002210A9122900AA8FCF706F918B1FFE75C
:10A14000F7F75CFCFFE7FFE740F69C40C4F20240F3
:10A15000016841F400310160006800F400300790AC
:10A160000798FFE7FFE740F68C40C4F20240016821
:10A1700041F001010160006800F0010006900698BE
:10A18000FFE70C20689002206990002001906A90FF
:10A190006B9007206C900020C4F2022068A9F8F7A9
:10A1A00095FD019821214D9117214E914F9050908E
:10A1B000519052905390549001215691579158903C
:10A1C00059905A905E905B905C9040F26421C2F28C
:10A1D00000014DA8F7F72EFC18B1FFE7F7F70EFCCA
:10A1E000FFE740F23420C2F2000040F26422C2F2E3
:10A1F00000020021F7F70EFE18B1FFE7F7F7FEFBAC
:10A20000FFE740F23420C2F20000F7F7A3FF18B1D5
:10A21000FFE7F7F7F3FBFFE740F6F410C2F20000A8
:10A2200040F2D011C4F20201016000218163C163D8
:10A230000164416481218164F7F72AFC18B1FFE7CA
:10A24000F7F7DCFBFFE740F6F410C2F2000040F243
:10A250003421C2F20001F7F7ABFE18B1FFE7F7F7C0
:10A26000CDFBFFE7FFE76D9840F6F411C2F2000165
:10A27000C0F880106D98C865FFE740F6F410C2F290
:10A2800000001021F8F726F918B1FFE7F7F7B6FB41
:10A29000FFE73B20009000221146F8F745FF0098A9
:10A2A000F8F738FFFFE7FFE76EB080BD80B586B0F6
:10A2B00004900391ADF80A200498D0F88C0020286F
:10A2C00045D1FFE7039820B1FFE7BDF80A0020B9A8
:10A2D000FFE701208DF817003DE004990020C866D3
:10A2E0000498006842F20041C4F20041884225D03F
:10A2F000FFE70498006842F20041C5F2004188423D
:10A300001CD0FFE70498006840680002002814D5BC
:10A31000FFE7FFE7FFE70498006850E8000F40F010
:10A3200080600190FFE701990498026842E80010FC
:10A330000028F0D1FFE7FFE7FFE7FFE70498039964
:10A34000BDF80A2002F02CF88DF8170003E0022077
:10A350008DF81700FFE79DF8170006B080BD0000DC
:10A3600080B586B004900391ADF80A200498D0F827
:10A370008C00202853D1FFE7039820B1FFE7BDF8F8
:10A380000A0020B9FFE701208DF817004BE004997F
:10A390000020C8660498006880684006002807D539
:10A3A000FFE704980168886820F040008860FFE7B4
:10A3B0000498006842F20041C4F20041884225D06E
:10A3C000FFE70498006842F20041C5F2004188426C
:10A3D0001CD0FFE70498006840680002002814D5EC
:10A3E000FFE7FFE7FFE70498006850E8000F40F040
:10A3F00080600190FFE701990498026842E800102C
:10A400000028F0D1FFE7FFE7FFE7FFE70498039993
:10A41000BDF80A2002F0B0F88DF8170003E0022022
:10A420008DF81700FFE79DF8170006B080BD00000B
:10A4300080B582B001900198006843F60001C4F233
:10A440000101884245D1FFE740F6D040C2F200004A
:10A4500000780A2834D1FFE740F6D240C2F200006B
:10A460000088012813DBFFE740F6D241C2F2000169
:10A470000B8840F2B112C2F200020020D05440F624
:10A48000F013C2F2000301221A70088017E040F6B0
:10A49000D240C2F2000000887E2801DCFFE70DE018
:10A4A00040F6D241C2F200010020088040F2B11013
:10A4B000C2F200008021F6F736F9FFE7FFE7FFE779
:10A4C000019840F6D041C2F200010122FFF748FF97
:10A4D000FFE702B080BD000081B0009001B070477E
:10A4E00081B0009001B0704780B582B040F6A830CE
:10A4F000C2F20000019041F20811C2F200014022B4
:10A50000FFF7D4FE01980168086840F01000086069
:10A5100002B080BDFFE7FEE780B586B0FFE740F6FA
:10A520008840C4F20240016841F001010160006806
:10A5300000F0010005900598FFE71E200190002221
:10A5400003921146F8F7F0FD0198F8F7E3FD039A3E
:10A550001F2002901146F8F7E7FD0298F8F7DAFDA0
:10A56000039A202004901146F8F7DEFD0498F8F7CE
:10A57000D1FD06B080BD000083B0FFE740F68C40FF
:10A58000C4F20240016841F080010160006800F0FF
:10A59000800002900298FFE7FFE740F68C40C4F28B
:10A5A0000240016841F001010160006800F0010013
:10A5B00001900198FFE7FFE740F68C40C4F20240AB
:10A5C000016841F002010160006800F002000090A3
:10A5D0000098FFE703B0704780B502F0FBFA80BD3A
:10A5E00080B582B040F6A830C2F20000009043F679
:10A5F0000001C4F2010101604FF4165141600021D5
:10A6000001918160C16001610C2242618161C1617F
:10A61000016241628162FFF70FFC18B1FFE7F7F7B3
:10A62000EDF9FFE740F6A830C2F200000021FFF785
:10A6300083F818B1FFE7F7F7E1F9FFE740F6A83034
:10A64000C2F200000021FFF731F818B1FFE7F7F779
:10A65000D5F9FFE740F6A830C2F20000FEF754FF3C
:10A6600018B1FFE7F7F7CAF9FFE702B080BD0000B5
:10A6700080B582B040F63C40C2F20000009044F247
:10A680000041C4F2000101604FF416514160002105
:10A6900001918160C16001610C2242618161C161EF
:10A6A000016241628162FFF7C7FB18B1FFE7F7F76C
:10A6B000A5F9FFE740F63C40C2F200000021FFF799
:10A6C0003BF818B1FFE7F7F799F9FFE740F63C4090
:10A6D000C2F200000021FEF7E9FF18B1FFE7F7F72B
:10A6E0008DF9FFE740F63C40C2F20000FEF70CFF98
:10A6F00018B1FFE7F7F782F9FFE702B080BD00006D
:10A70000FFE7FEE7FFE7FEE788B0079006910592B6
:10A71000079800F0070004900498C0F1070005288E
:10A7200003D3FFE70420019004E00498C0F1070080
:10A730000190FFE70198039004980430062803D89D
:10A74000FFE70020009003E0049803380090FFE743
:10A750000098029006980399012202FA01F101394A
:10A760000840029B984005999A40013A11400843DD
:10A7700008B0704780B584B0029040F60041C4F242
:10A780000241086820F080600860F8F715FC01902D
:10A79000FFE740F60040C4F20240006800F00061AC
:10A7A0000020B0EBD16F0CD0FFE7F8F705FC019962
:10A7B000401A032804D3FFE703208DF80F008BE035
:10A7C000E7E7FFE740F62C41C4F20241086843F690
:10A7D00003729043029B1A685B6842EA03221043AB
:10A7E000086002998868D1F80CC00B694A69013881
:10A7F0006FF35F204FF60061CFF6FF7101EB4C2144
:10A8000089B208440021CFF6FF7101EB034101F446
:10A81000FE0108444FF07F4101EB026101F0FE416F
:10A82000084440F63C41C4F202410860FFE740F6AC
:10A830002C41C4F202410091086820F00C00029AF9
:10A84000926910430860086820F02000029AD269DB
:10A85000104308600298426A08681043086008685C
:10A8600020F01000086040F64042C4F20242106836
:10A870004FF6F8739843029B1B6A40EAC3001060CE
:10A88000086840F01000086040F60041C4F2024140
:10A89000086840F080600860F8F78EFB0190FFE7E1
:10A8A00040F60040C4F20240006800F00061002061
:10A8B000B0EBD16F0CD1FFE7F8F77EFB0199401A9E
:10A8C000032804D3FFE703208DF80F0004E0E7E737
:10A8D00000208DF80F00FFE79DF80F0004B080BD49
:10A8E00080B584B0029040F60041C4F2024108688D
:10A8F00020F080500860F8F75FFB0190FFE740F61A
:10A900000040C4F20240006800F000510020B0EBAB
:10A91000517F0CD0FFE7F8F74FFB0199401A03284D
:10A9200004D3FFE703208DF80F008BE0E7E7FFE794
:10A9300040F63041C4F20241086843F60372904386
:10A94000029B1A685B6842EA03221043086002997E
:10A950008868D1F80CC00B694A6901386FF35F2031
:10A960004FF60061CFF6FF7101EB4C2189B208442C
:10A970000021CFF6FF7101EB034101F4FE01084411
:10A980004FF07F4101EB026101F0FE41084440F6C7
:10A990004441C4F202410860FFE740F63041C4F28E
:10A9A00002410091086820F00C00029A926910435D
:10A9B0000860086820F02000029AD26910430860FD
:10A9C0000298426A086810430860086820F0100086
:10A9D000086040F64842C4F2024210684FF6F8732D
:10A9E0009843029B1B6A40EAC3001060086840F06D
:10A9F0001000086040F60041C4F20241086840F0CF
:10AA000080500860F8F7D8FA0190FFE740F6004060
:10AA1000C4F20240006800F000510020B0EB517F0A
:10AA20000CD1FFE7F8F7C8FA0199401A032804D3BC
:10AA3000FFE703208DF80F0004E0E7E700208DF822
:10AA40000F00FFE79DF80F0004B080BD80B59CB0FB
:10AA500008A85021F5F789FE002007900690059080
:10AA6000049003900290FFE740F61000C4F2024009
:10AA7000016841F030010160006800F03000019091
:10AA80000198FFE7FFE740F61400C4F202400068B7
:10AA900000F00800082801D0FFE7F4E71020089034
:10AAA0004FF480700F90202010900220129013908D
:10AAB000012114917D21159116901790189008206E
:10AAC000199000201A901B9008A8FDF7F1FC18B10E
:10AAD000FFE7F6F793FFFFE71F20029003200390A4
:10AAE0000020049005900690079002A80521FDF72C
:10AAF000A3F818B1FFE7F6F781FFFFE742F2000184
:10AB0000C4F202010868022262F3051008601CB05A
:10AB100080BD000082B04EF68851CEF20001086878
:10AB200040F47000086040F60042C4F20242012086
:10AB3000106040F61C41C4F2024100200090086001
:10AB400040F62041C4F20241086011684EF6E3234A
:10AB5000CEF6E2231940116040F62841C4F20241CA
:10AB6000086040F62C41C4F20241086040F63041D2
:10AB7000C4F20241086040F63443C4F2024340F29A
:10AB80008021C0F20111196040F63843C4F202433B
:10AB9000186040F63C43C4F20243196040F640435B
:10ABA000C4F20243186040F64443C4F20243196001
:10ABB00040F64841C4F202410860116821F4802146
:10ABC000116040F65041C4F2024108604EF608514F
:10ABD000CEF200014FF00060086042F21800C4F2AB
:10ABE0000200006800F0604001900198B0F1604FF1
:10ABF00005D0FFE70198B0F1404F24D1FFE742F2C2
:10AC00001C00C4F202000068C00778B1FFE742F2FE
:10AC10000C01C4F2020142F63B20C0F619000860A4
:10AC200046F67F60C4F65D400860FFE742F21C0113
:10AC3000C4F20201086840F002000860086840F0B1
:10AC400001000860FFE702B07047000080B540F6E1
:10AC50005C30C2F20000FEF7B9FA80BD83B002900A
:10AC60000191029800680090029842F60041C4F2F7
:10AC70000101884252D0FFE7029842F60041C5F236
:10AC8000010188424AD0FFE70298B0F1804F45D0D9
:10AC9000FFE70298B0F1A04F40D0FFE7029840F2E2
:10ACA0000041C4F20001884238D0FFE7029840F228
:10ACB0000041C5F20001884230D0FFE7029840F61B
:10ACC0000001C4F20001884228D0FFE7029840F654
:10ACD0000001C5F20001884220D0FFE7029840F64B
:10ACE0000041C4F20001884218D0FFE7029840F604
:10ACF0000041C5F20001884210D0FFE7029843F2FC
:10AD00000041C4F20101884208D0FFE7029843F2F3
:10AD10000041C5F2010188420AD1FFE7009820F006
:10AD20007000009001984168009808430090FFE788
:10AD3000029842F60041C4F20101884200F0BA8054
:10AD4000FFE7029842F60041C5F20101884200F097
:10AD5000B180FFE70298B0F1804F00F0AB80FFE7D1
:10AD60000298B0F1A04F00F0A580FFE7029840F2F2
:10AD70000041C4F20001884200F09C80FFE7029885
:10AD800040F20041C5F20001884200F09380FFE7E5
:10AD9000029840F60001C4F20001884200F08A8067
:10ADA000FFE7029840F60001C5F20001884200F07A
:10ADB0008180FFE7029840F60041C4F2000188421A
:10ADC00078D0FFE7029840F60041C5F200018842C2
:10ADD00070D0FFE7029843F20041C4F201018842BB
:10ADE00068D0FFE7029843F20041C5F201018842B2
:10ADF00060D0FFE7029841F60001C4F200018842EA
:10AE000058D0FFE7029841F60001C5F200018842E0
:10AE100050D0FFE7029841F60041C4F20001884299
:10AE200048D0FFE7029841F60041C5F20001884290
:10AE300040D0FFE7029842F20001C4F200018842CC
:10AE400038D0FFE7029842F20001C5F200018842C3
:10AE500030D0FFE7029844F20001C4F201018842B9
:10AE600028D0FFE7029844F20001C5F201018842B0
:10AE700020D0FFE7029844F20041C4F20101884269
:10AE800018D0FFE7029844F20041C5F20101884260
:10AE900010D0FFE7029844F60001C4F20101884295
:10AEA00008D0FFE7029844F60001C5F2010188428C
:10AEB0000AD1FFE7009820F4407000900198C16823
:10AEC000009808430090FFE7009820F08000019967
:10AED00049690843009000980299086001988068C9
:10AEE0000299C8620198006802998862029842F645
:10AEF0000041C4F20101884248D0FFE7029842F6BF
:10AF00000041C5F20101884240D0FFE7029843F2B8
:10AF10000041C4F20101884238D0FFE7029843F2B1
:10AF20000041C5F20101884230D0FFE7029844F2A7
:10AF30000001C4F20101884228D0FFE7029844F2E0
:10AF40000001C5F20101884220D0FFE7029844F2D7
:10AF50000041C4F20101884218D0FFE7029844F290
:10AF60000041C5F20101884210D0FFE7029844F683
:10AF70000001C4F20101884208D0FFE7029844F6BC
:10AF80000001C5F20101884205D1FFE7019800697F
:10AF900002990863FFE7029901204861029800695D
:10AFA000C00730B1FFE70299086920F0010008618D
:10AFB000FFE703B07047000082B001900198406E37
:10AFC00040B9FFE701990120A1F86A000199A1F8B1
:10AFD000680034E008208DF803008DF80200019825
:10AFE00000688068C0F342608DF801000198006835
:10AFF0008068400F8DF800009DF802009DF8002049
:10B000004DF6A243C0F60003995C00FB01F04DF63B
:10B010009A41C0F600018A5CB0FBF2F0019AA2F8F6
:10B020006A009DF803009DF801209B5C00FB03F083
:10B03000895CB0FBF1F00199A1F86800FFE702B06C
:10B040007047000081B00090009890F82800000739
:10B0500000280BD5FFE700980068406820F4004006
:10B06000009A1168926B10434860FFE7009890F8CF
:10B070002800C00758B1FFE700980068406820F436
:10B080000030009A1168D26A10434860FFE70098C8
:10B0900090F82800800700280BD5FFE7009800688B
:10B0A000406820F48030009A1168126B10434860A9
:10B0B000FFE7009890F82800400700280BD5FFE72D
:10B0C00000980068406820F48020009A1168526B54
:10B0D00010434860FFE7009890F82800C006002859
:10B0E0000BD5FFE700980068806820F48050009A34
:10B0F0001168D26B10438860FFE7009890F8280031
:10B10000800600280BD5FFE700980068806820F4CF
:10B110000050009A1168126C10438860FFE7009895
:10B1200090F82800400600281CD5FFE7009800682A
:10B13000406820F48010009A1168526C10434860F7
:10B140000098406CB0F5801F0BD1FFE700980068B5
:10B15000406820F4C000009A1168926C1043486067
:10B16000FFE7FFE7009890F82800000600280BD5BD
:10B17000FFE700980068406820F40020009A1168FA
:10B18000D26C10434860FFE701B0704780B588B0CB
:10B19000069006990020C1F89000F7F70DFF059082
:10B1A000069800680068000700282FD5FFE706987A
:10B1B000059B6A466FF07E4111604FF4001100223A
:10B1C00001F0ECFA08B3FFE7FFE7FFE70698006835
:10B1D00050E8000F20F080000490FFE704990698E3
:10B1E000026842E800100028F0D1FFE7FFE7069967
:10B1F0002020C1F88800FFE70699002081F884002C
:10B20000FFE703208DF81F005FE0FFE70698006866
:10B2100000684007002842D5FFE70698059B6A466C
:10B220006FF07E4111604FF48001002201F0B6FA08
:10B23000A0B3FFE7FFE7FFE70698006850E8000FBC
:10B2400020F490700390FFE703990698026842E8A3
:10B2500000100028F0D1FFE7FFE7FFE7FFE70698BF
:10B26000006850E8020F20F001000290FFE7029909
:10B270000698026842E802100028F0D1FFE7FFE7D5
:10B2800006992020C1F88C00FFE70699002081F87C
:10B290008400FFE703208DF81F0016E0FFE7069902
:10B2A0002020C1F888000699C1F88C00069900207A
:10B2B000C86606990867FFE70699002081F88400B0
:10B2C000FFE700208DF81F00FFE79DF81F0008B082
:10B2D00080BD000080B582B001900198C06D0090E3
:10B2E00000990020A1F85E000098FEF7FFFA02B076
:10B2F00080BD000080B584B003900398C06D0290BB
:10B300000298D0F8880001900298D0F88C00009044
:10B31000029800688068000600280CD5FFE70198B5
:10B32000212808D1FFE702990020A1F856000298D1
:10B3300000F04CF9FFE7029800688068400600289A
:10B340000CD5FFE70098222808D1FFE702990020DA
:10B35000A1F85E00029800F0C7F8FFE70299D1F863
:10B36000900040F01000C1F890000298FEF7BEFA7D
:10B3700004B080BD80B586B005900598C06D04907E
:10B380000598006D812848D0FFE704990020A1F8B6
:10B390005E00FFE7FFE70498006850E8000F20F424
:10B3A00080700390FFE703990498026842E8001058
:10B3B0000028F0D1FFE7FFE7FFE7FFE70498006808
:10B3C00050E8020F20F001000290FFE70299049874
:10B3D000026842E802100028F0D1FFE7FFE7049975
:10B3E0002020C1F88C000498C06E012814D1FFE71A
:10B3F000FFE7FFE70498006850E8000F20F0100016
:10B400000190FFE701990498026842E800100028C3
:10B41000F0D1FFE7FFE7FFE7FFE7049900200867A7
:10B420000498C06E012821D1FFE704990020A1F8FB
:10B430005E0005980068806CADF80200BDF802005F
:10B440000499B1F85C10884206DAFFE7BDF8020003
:10B450000499A1F85E00FFE70498B0F85C10B0F81A
:10B460005E20891A89B2FEF7E5F803E00498FEF73A
:10B47000DFFFFFE706B080BD80B584B0039003987E
:10B48000C06D02900299012008670298C06E0128E1
:10B4900023D1FFE70299B1F85C004008A1F85E00F3
:10B4A00003980068806CADF80600BDF806000299AC
:10B4B000B1F85C10884206DCFFE7BDF8060002998F
:10B4C000A1F85E00FFE70298B0F85C10B0F85E20CB
:10B4D000891A89B2FEF7AEF803E00298FEF7FCFF86
:10B4E000FFE704B080BD000084B00390FFE7FFE7F2
:10B4F0000398006850E8000F20F490700290FFE776
:10B5000002990398026842E800100028F0D1FFE792
:10B51000FFE7FFE7FFE70398006850E8020F4FF6E8
:10B52000FE71CEF6FF7108400190FFE70199039884
:10B53000026842E802100028EDD1FFE7FFE7039818
:10B54000C06E012814D1FFE7FFE7FFE7039800680A
:10B5500050E8000F20F010000090FFE700990398DA
:10B56000026842E800100028F0D1FFE7FFE7FFE79C
:10B5700003992020C1F88C0003990020C866039924
:10B58000486704B07047000080B582B00190FFE7C3
:10B59000FFE70198006850E8000F20F0400000909D
:10B5A000FFE700990198026842E800100028F0D1F6
:10B5B000FFE7FFE701992020C1F8880001990020EA
:10B5C00088670198FEF78CFF02B080BD83B00290BF
:10B5D000FFE7FFE70298006850E8000F20F0C00086
:10B5E0000190FFE701990298026842E800100028E4
:10B5F000F0D1FFE7FFE7FFE7FFE70298006850E8B8
:10B60000020F20F400000090FFE700990298026802
:10B6100042E802100028F0D1FFE7FFE7029920205E
:10B62000C1F8880003B0704780B588B007900798CC
:10B63000B0F86000ADF816000798D0F88C0022280A
:10B6400040F0B480FFE707980068406AADF8140046
:10B650000798806D0690BDF81400BDF816100840DC
:10B66000069908800799886D023088650799B1F8B6
:10B670005E000138A1F85E000798B0F85E0000286F
:10B6800040F09380FFE7FFE7FFE70798006850E886
:10B69000000F20F490700490FFE704990798026867
:10B6A00042E800100028F0D1FFE7FFE7FFE7FFE7DF
:10B6B0000798006850E8020F20F001000390FFE7B0
:10B6C00003990798026842E802100028F0D1FFE7CA
:10B6D000FFE707992020C1F88C00079900204867F0
:10B6E000079908670798006842F20041C4F20041D8
:10B6F000884225D0FFE70798006842F20041C5F272
:10B70000004188421CD0FFE70798006840680002AB
:10B71000002814D5FFE7FFE7FFE70798006850E827
:10B72000000F20F080600290FFE7029907980268FE
:10B7300042E800100028F0D1FFE7FFE7FFE7FFE74E
:10B740000798C06E01282BD1FFE707990020C86633
:10B75000FFE7FFE70798006850E8000F20F01000AF
:10B760000190FFE701990798026842E8001000285D
:10B77000F0D1FFE7FFE707980068C06900F010010B
:10B780000120B0EB111F05D1FFE7079801681020D9
:10B790000862FFE70798B0F85C10FDF74BFF03E085
:10B7A0000798FEF745FEFFE7FFE706E00798016808
:10B7B000886940F008008861FFE708B080BD00009C
:10B7C00080B58EB00D900D98B0F86000ADF82E00E9
:10B7D0000D980068C06909900D980068006808908D
:10B7E0000D980068806807900D98D0F88C0022288A
:10B7F00040F06A81FFE70D98B0F86800ADF82A00C4
:10B80000FFE7BDF82A100020009031B1FFE79DF856
:10B810002400C0F340100090FFE70098C007002804
:10B8200000F01381FFE70D980068406AADF82C0026
:10B830000D98806D0C90BDF82C00BDF82E100840BE
:10B840000C9908800D99886D023088650D99B1F8C2
:10B850005E000138A1F85E000D980068C06909908B
:10B860009DF824004007002852D0FFE79DF82400EF
:10B87000C00788B1FFE79DF82100C00760B1FFE76E
:10B880000D980168012008620D99D1F8900040F0F0
:10B890000100C1F89000FFE79DF824008007002810
:10B8A00011D5FFE79DF81C00C00760B1FFE70D98B8
:10B8B0000168022008620D99D1F8900040F0040060
:10B8C000C1F89000FFE79DF824004007002811D53B
:10B8D000FFE79DF81C00C00760B1FFE70D98016805
:10B8E000042008620D99D1F8900040F00200C1F8E0
:10B8F0009000FFE70D98D0F8900040B1FFE70D9859
:10B90000FDF7F4FF0D990020C1F89000FFE7FFE775
:10B910000D98B0F85E00002840F09680FFE7FFE742
:10B92000FFE70D98006850E8000F20F48070069043
:10B93000FFE706990D98026842E800100028F0D150
:10B94000FFE7FFE7FFE7FFE70D98006850E8020F09
:10B950004FF6FE71CEF6FF7108400590FFE705999E
:10B960000D98026842E802100028EDD1FFE7FFE7DA
:10B970000D992020C1F88C000D99002048670D9981
:10B9800008670D98006842F20041C4F20041884205
:10B9900025D0FFE70D98006842F20041C5F2004152
:10B9A00088421CD0FFE70D9800684068000200281C
:10B9B00014D5FFE7FFE7FFE70D98006850E8000F98
:10B9C00020F080600490FFE704990D98026842E837
:10B9D00000100028F0D1FFE7FFE7FFE7FFE70D9831
:10B9E000C06E01282BD1FFE70D990020C866FFE744
:10B9F000FFE70D98006850E8000F20F0100003905A
:10BA0000FFE703990D98026842E800100028F0D182
:10BA1000FFE7FFE70D980068C06900F01001012002
:10BA2000B0EB111F05D1FFE70D98016810200862E7
:10BA3000FFE70D98B0F85C10FDF7FCFD03E00D98F2
:10BA4000FEF7F6FCFFE700E0DBE60D98B0F85E00DD
:10BA5000ADF82800BDF82800A8B3FFE7BDF828001E
:10BA60000D99B1F8681088422DDAFFE7FFE7FFE78C
:10BA70000D98006850E8020F20F080500290FFE718
:10BA800002990D98026842E802100028F0D1FFE701
:10BA9000FFE70D994BF22960C0F600004867FFE709
:10BAA000FFE70D98006850E8000F40F0200001907B
:10BAB000FFE701990D98026842E800100028F0D1D4
:10BAC000FFE7FFE7FFE706E00D980168886940F0AF
:10BAD00008008861FFE70EB080BD000080B586B029
:10BAE00005900598B0F86000ADF812000598D0F800
:10BAF0008C00222840F0B280FFE705980068406A79
:10BB0000ADF81000BDF810009DF81210084005991E
:10BB1000896D08700599886D013088650599B1F8BF
:10BB20005E000138A1F85E000598B0F85E000028BC
:10BB300040F09380FFE7FFE7FFE70598006850E8D3
:10BB4000000F20F490700390FFE7039905980268B6
:10BB500042E800100028F0D1FFE7FFE7FFE7FFE72A
:10BB60000598006850E8020F20F001000290FFE7FE
:10BB700002990598026842E802100028F0D1FFE718
:10BB8000FFE705992020C1F88C000599002048673F
:10BB9000059908670598006842F20041C4F2004127
:10BBA000884225D0FFE70598006842F20041C5F2BF
:10BBB000004188421CD0FFE70598006840680002F9
:10BBC000002814D5FFE7FFE7FFE70598006850E875
:10BBD000000F20F080600190FFE70199059802684E
:10BBE00042E800100028F0D1FFE7FFE7FFE7FFE79A
:10BBF0000598C06E01282BD1FFE705990020C86683
:10BC0000FFE7FFE70598006850E8000F20F01000FC
:10BC10000090FFE700990598026842E800100028AC
:10BC2000F0D1FFE7FFE705980068C06900F0100158
:10BC30000120B0EB111F05D1FFE705980168102026
:10BC40000862FFE70598B0F85C10FDF7F3FC03E02D
:10BC50000598FEF7EDFBFFE7FFE706E005980168B2
:10BC6000886940F008008861FFE706B080BD0000E9
:10BC700080B58EB00D900D98B0F86000ADF8320030
:10BC80000D980068C0690A900D98006800680990D6
:10BC90000D980068806808900D98D0F88C002228D4
:10BCA00040F06881FFE70D98B0F86800ADF82E000D
:10BCB000FFE7BDF82E100020019031B1FFE79DF89D
:10BCC0002800C0F340100190FFE70198C00700284A
:10BCD00000F01181FFE70D980068406AADF8300070
:10BCE000BDF830009DF8321008400D99896D08703C
:10BCF0000D99886D013088650D99B1F85E000138A5
:10BD0000A1F85E000D980068C0690A909DF82800AF
:10BD10004007002852D0FFE79DF82800C00788B1EF
:10BD2000FFE79DF82500C00760B1FFE70D980168A7
:10BD3000012008620D99D1F8900040F00100C1F88F
:10BD40009000FFE79DF828008007002811D5FFE745
:10BD50009DF82000C00760B1FFE70D980168022040
:10BD600008620D99D1F8900040F00400C1F89000ED
:10BD7000FFE79DF828004007002811D5FFE79DF850
:10BD80002000C00760B1FFE70D9801680420086239
:10BD90000D99D1F8900040F00200C1F89000FFE743
:10BDA0000D98D0F8900040B1FFE70D98FDF79EFD8B
:10BDB0000D990020C1F89000FFE7FFE70D98B0F85B
:10BDC0005E00002840F09680FFE7FFE7FFE70D9850
:10BDD000006850E8000F20F480700790FFE7079993
:10BDE0000D98026842E800100028F0D1FFE7FFE755
:10BDF000FFE7FFE70D98006850E8020F4FF6FE716D
:10BE0000CEF6FF7108400690FFE706990D9802688C
:10BE100042E802100028EDD1FFE7FFE70D9920204E
:10BE2000C1F88C000D99002048670D9908670D989E
:10BE3000006842F20041C4F20041884225D0FFE789
:10BE40000D98006842F20041C5F2004188421CD0C2
:10BE5000FFE70D98006840680002002814D5FFE74E
:10BE6000FFE7FFE70D98006850E8000F20F08060C2
:10BE70000590FFE705990D98026842E80010002838
:10BE8000F0D1FFE7FFE7FFE7FFE70D98C06E01285D
:10BE90002BD1FFE70D990020C866FFE7FFE70D985B
:10BEA000006850E8000F20F010000490FFE70499AC
:10BEB0000D98026842E800100028F0D1FFE7FFE784
:10BEC0000D980068C06900F010010120B0EB111F4F
:10BED00005D1FFE70D98016810200862FFE70D9873
:10BEE000B0F85C10FDF7A6FB03E00D98FEF7A0FA92
:10BEF000FFE700E0DDE60D98B0F85E00ADF82C003D
:10BF0000BDF82C00A8B3FFE7BDF82C000D99B1F8DF
:10BF1000681088422DDAFFE7FFE7FFE70D98006819
:10BF200050E8020F20F080500390FFE703990D982E
:10BF3000026842E802100028F0D1FFE7FFE70D9900
:10BF40004BF6DD20C0F600004867FFE7FFE70D98DD
:10BF5000006850E8000F40F020000290FFE70299CF
:10BF60000D98026842E800100028F0D1FFE7FFE7D3
:10BF7000FFE706E00D980168886940F008008861D5
:10BF8000FFE70EB080BD000080B58AB009900020A8
:10BF90008DF813000998006842F20041C4F2004194
:10BFA000884209D0FFE70998006842F20041C5F2D3
:10BFB0000041884201D1FFE700E0FFE70999886866
:10BFC0000B694A69C96918431043084308900998E6
:10BFD0000068006846F6F311CCF6FF710840089936
:10BFE000084309990968086009980068406820F4C6
:10BFF0004050099A1168D2681043486009988069D6
:10C0000008900998006842F20041C4F20041884259
:10C010000FD0FFE70998006842F20041C5F20041E5
:10C02000884206D0FFE70998016A089808430890FB
:10C03000FFE70998006880684FF2FF41C1F2FF11E5
:10C0400008400899084309990968886009980068B8
:10C05000C06A20F00F00099A1168526A1043C86242
:10C06000FFE70998006843F60001C4F20101884225
:10C0700003D1FFE701200690A3E00998006844F28D
:10C080000041C4F20001884203D1FFE7022006907C
:10C0900096E00998006844F60001C4F20001884265
:10C0A00003D1FFE70420069089E00998006844F670
:10C0B0000041C4F20001884203D1FFE70820069046
:10C0C0007CE00998006845F20001C4F20001884252
:10C0D00003D1FFE7102006906FE00998006846F250
:10C0E0000041C4F20001884203D1FFE720200690FE
:10C0F00062E00998006847F60001C4F20001884236
:10C1000003D1FFE74020069055E00998006847F604
:10C110000041C4F20001884203D1FFE7802006906D
:10C1200048E00998006848F20001C4F20001884222
:10C1300004D1FFE74FF4807006903AE00998006858
:10C1400046F60001C4F20001884204D1FFE74FF433
:10C15000007006902CE00998006846F60041C4F291
:10C160000001884204D1FFE74FF4806006901EE092
:10C170000998006848F20041C4F20001884204D1E5
:10C18000FFE74FF40060069010E00998006842F263
:10C190000041C4F20041884204D1FFE74FF48050CF
:10C1A000069002E000200690FFE7FFE7FFE7FFE7C9
:10C1B000FFE7FFE7FFE7FFE7FFE7FFE7FFE7FFE74F
:10C1C000FFE7FFE70998006842F20041C4F200412E
:10C1D000884209D0FFE70998006842F20041C5F2A1
:10C1E000004188425CD1FFE706980021F7F730FC58
:10C1F00002900298002852D0FFE7029809994A6AF3
:10C200004DF6AA41C0F6000131F81210B0FBF1F072
:10C21000039003980999496801EB4101884207D3CB
:10C22000FFE7039809994968B0EB013F04D9FFE79C
:10C2300001208DF8130031E0029809994A680092B4
:10C240004A6A4DF6AA41C0F6000131F812200023D7
:10C2500001931946F4F7A2F9009A019B090241EAF9
:10C260001061000210EB520041F10001F4F796F961
:10C2700005900598B0F5407F0BD3FFE705990020A6
:10C28000B0EB115F05D1FFE7059809990968C8600F
:10C2900003E001208DF81300FFE7FFE7FFE76FE001
:10C2A0000998C069B0F5004F3CD1FFE7069800211E
:10C2B000F7F7CEFB0290029898B3FFE70298099A2D
:10C2C0005168536A4DF6AA42C0F6000232F81320B4
:10C2D000B0FBF2F0400000EB5100B0FBF1F0059034
:10C2E0000598102818D3FFE7BDF81600A0B9FFE79E
:10C2F000059820F00F00ADF81E00059800F00E0123
:10C30000BDF81E0040EA5100ADF81E00BDF81E0049
:10C3100009990968C86003E001208DF81300FFE760
:10C32000FFE72CE006980021F7F792FB02900298B5
:10C3300020B3FFE70298099A5168536A4DF6AA4262
:10C34000C0F6000232F81320B0FBF2F000EB51000F
:10C35000B0FBF1F00590059810280AD3FFE7BDF86F
:10C36000160030B9FFE7BDF8140009990968C860E4
:10C3700003E001208DF81300FFE7FFE7FFE7FFE789
:10C3800009990120A1F86A000999A1F868000999A2
:10C3900000204867099988679DF813000AB080BD9E
:10C3A00080B588B006900591ADF81220BDF8120056
:10C3B000ADF80E00059806998865BDF8120006993B
:10C3C000A1F85C0006990020C1F89000069922208F
:10C3D000C1F88C000698D0F88000002800F0868014
:10C3E000FFE70698D0F880104BF27530C0F60000D9
:10C3F00008660698D0F880104BF27940C0F600002D
:10C4000048660698D0F880104BF2F520C0F6000080
:10C4100088660698D0F880100020C8660698806864
:10C42000B0F5805F0AD1FFE70698006930B9FFE7F1
:10C43000BDF812004000ADF80E00FFE70698D0F8F6
:10C44000800090F850000006002831D5FFE70698DC
:10C45000D0F88000406F30B3FFE70698D0F8800036
:10C46000406F0068F8B1FFE7BDF80E000699D1F8FB
:10C470008010496F0968886006990868D1F88010B3
:10C480002430496F0968C8600699886DD1F880101A
:10C49000496F096808610698D0F88000F5F7C0FE7A
:10C4A0008DF8110003E001208DF81100FFE70CE08A
:10C4B00006980168826DD0F880002431BDF80E30F6
:10C4C000F6F792FB8DF81100FFE79DF8110060B1BF
:10C4D000FFE706991020C1F8900006992020C1F8C6
:10C4E0008C0001208DF81F0042E0FFE706980069EC
:10C4F000A0B1FFE7FFE7FFE70698006850E8000FEC
:10C5000040F480700290FFE702990698026842E8C2
:10C5100000100028F0D1FFE7FFE7FFE7FFE7FFE7A4
:10C520000698006850E8020F40F001000190FFE714
:10C5300001990698026842E802100028F0D1FFE74E
:10C54000FFE7FFE7FFE70698006850E8020F40F0BA
:10C5500040000090FFE700990698026842E8021048
:10C560000028F0D1FFE7FFE700208DF81F00FFE76C
:10C570009DF81F0008B080BD88B007900691ADF807
:10C580001620069807998865BDF816000799A1F846
:10C590005C00BDF816000799A1F85E00079900201D
:10C5A0004867FFE707988068B0F5805F10D1FFE724
:10C5B0000798006930B9FFE7079940F2FF10A1F82A
:10C5C000600004E00799FF20A1F86000FFE72EE07B
:10C5D0000798806878B9FFE70798006928B9FFE7EE
:10C5E0000799FF20A1F8600004E007997F20A1F8D7
:10C5F0006000FFE71AE007988068B0F1805F0FD114
:10C60000FFE70798006928B9FFE707997F20A1F89D
:10C61000600004E007993F20A1F86000FFE704E014
:10C6200007990020A1F86000FFE7FFE7FFE7FFE7B9
:10C6300007990020C1F8900007992220C1F88C00CA
:10C64000FFE7FFE70798006850E8020F40F001009D
:10C650000490FFE704990798026842E80210002856
:10C66000F0D1FFE7FFE70798406EB0F1005F4CD1D3
:10C67000FFE7BDF816000799B1F86810884244DB5F
:10C68000FFE707988068B0F5805F0BD1FFE7079858
:10C69000006938B9FFE707994BF2C170C0F6000096
:10C6A000486706E007994BF67140C0F600004867FE
:10C6B000FFE707980069A0B1FFE7FFE7FFE70798EA
:10C6C000006850E8000F40F480700390FFE7039982
:10C6D0000798026842E800100028F0D1FFE7FFE762
:10C6E000FFE7FFE7FFE70798006850E8020F40F018
:10C6F00080500290FFE702990798026842E8021012
:10C700000028F0D1FFE7FFE744E007988068B0F524
:10C71000805F0BD1FFE70798006938B9FFE70799F9
:10C720004BF22960C0F60000486706E007994BF617
:10C73000DD20C0F600004867FFE707980069A0B158
:10C74000FFE7FFE7FFE70798006850E8000F40F4B5
:10C7500090700190FFE701990798026842E8001085
:10C760000028F0D1FFE7FFE713E0FFE7FFE70798B6
:10C77000006850E8000F40F020000090FFE70099AB
:10C780000798026842E800100028F0D1FFE7FFE7B1
:10C79000FFE7FFE7002008B07047000080B586B0D3
:10C7A000DDF820C0049003918DF80B200193FFE782
:10C7B00004980068C06903990840401AB0FA80F0F4
:10C7C00040099DF80B10884266D1FFE708980130B8
:10C7D000002860D0FFE7F6F7EFFB0199401A0899AF
:10C7E000884203D8FFE7089820B9FFE703208DF8B7
:10C7F000170055E00498006800684007002849D5F4
:10C80000FFE70398802845D0FFE70398402841D0F0
:10C81000FFE704980068C06900F008010120B0EB50
:10C82000D10F16D1FFE70498016808200090086234
:10C830000498FEF759FE00980499C1F89000FFE7AC
:10C840000499002081F88400FFE701208DF817008B
:10C8500026E004980068C06900F400610120B0EB94
:10C86000D12F16D1FFE7049801684FF400600862E9
:10C870000498FEF739FE04992020C1F89000FFE7E4
:10C880000499002081F88400FFE703208DF8170049
:10C8900006E0FFE7FFE78BE700208DF81700FFE7D2
:10C8A0009DF8170006B080BD80B582B040F6A83074
:10C8B000C2F200000090FDF71DF800980068C06902
:10C8C000C00600283ED5FFE740F6A830C2F20000BF
:10C8D000026810211162D0F880000068806CC0F1FD
:10C8E0004000ADF806000020ADF80400FFE7BDF8F9
:10C8F0000400BDF8061088421BDAFFE7BDF80410FB
:10C9000041F20810C2F20000405C40F6EC01C2F2B5
:10C910000001B1F800218854B1F800010130C0B223
:10C92000A1F80001FFE7BDF804000130ADF80400F4
:10C93000DDE740F6A830C2F20000FCF74BFFFDF740
:10C94000D3FDFFE702B080BD80B540F63C40C2F2A7
:10C950000000FCF7CFFF80BDFFE7FEE781B0ADF838
:10C960000200BDF9020000280ED4FFE7BDF9021055
:10C9700001F01F02012090404A094EF20011CEF250
:10C98000000141F82200FFE701B070474EF60C505D
:10C99000CEF200000068C0F30220704782B0ADF80C
:10C9A00006000091BDF9060000280AD4FFE70098B0
:10C9B0000001BDF906104EF20042CEF2000288548A
:10C9C0000BE000980001BDF8061001F00F014EF6D3
:10C9D0001452CEF200028854FFE702B07047000004
:10C9E00083B00290029800F0070000904EF60C51C0
:10C9F000CEF200010868019001984FF6FF02104046
:10CA000001900198009A40EA02200022C0F2FA52F6
:10CA1000104301900198086003B0704780B58EB054
:10CA20000A900991089207930A983421F3F79DFE22
:10CA3000079820F00300079009980A994860089821
:10CA40000A99886107980A99C86108980A99086143
:10CA500008980A994861079808380A9988600A99DD
:10CA60000220C86008980590059807990844059029
:10CA70000598043805900A98039005980490039847
:10CA80000499086005980438059005980490089862
:10CA900004990860089803900398049005980499F5
:10CAA0000860089805900598043005900598009056
:10CAB00000994EF6EE60CFF6FF7008600A990020EC
:10CAC0000862EFF310800D900D980B9072B60B98E2
:10CAD00006900A9945F24540C4F25920086040F298
:10CAE000B820C2F20000006858B9FFE70A9840F287
:10CAF000BC21C2F2000108600A98C0620A98006373
:10CB000015E040F2BC20C2F20000006802900298DA
:10CB1000006B01900A98029908630A980199C8620B
:10CB200001980A99086302980A99C862FFE740F2DF
:10CB3000B821C2F2000108680130086006980C9024
:10CB40000C9880F3108800200EB080BD80B500F0F6
:10CB500083F900F051FD40F2E021C2F20001002013
:10CB6000086040F2DC21C2F20001086040F2D821E6
:10CB7000C2F20001086040F2D421C2F20001086054
:10CB800040F2C421C2F20001086040F2C021C2F2AA
:10CB90000001086040F2B021C2F20001086040F2DA
:10CBA000AC21C2F20001086040F2BC21C2F20001D7
:10CBB000086040F2B821C2F20001086040F2D021C2
:10CBC000C2F20001086040F2CC21C2F2000108600C
:10CBD00080BD000080B582B040F20400C2F20000C7
:10CBE000006810F10F3F13D0FFE740F20401C2F2DA
:10CBF00000014FF0F0300860F3F7B0FBFFF7A6FF3D
:10CC000040F2FC21C2F20001086801300860FFE731
:10CC100040F20401C2F2000101914FF0F0300860CF
:10CC200040F2C820C2F20000006800F0F1FF019954
:10CC300000200860F3F7CEFB02B080BD80B592B053
:10CC4000DDF864C0DDF860C0DDF85CC0DDF858C018
:10CC5000DDF854C0DDF850C00990089107920693A2
:10CC60000020019014981599EF22F3F754FD0998CC
:10CC7000B021F3F77AFD0898099988620798099915
:10CC8000486406980999886414980999C8601598A9
:10CC90000999486116980999C86216980999C1F8C6
:10CCA000940018980999886118980999C861099998
:10CCB0002020C1F89C001498009000991598084411
:10CCC00001380090009809990861169817998842D0
:10CCD00007D0FFE709990020C8630999C1F89800B7
:10CCE00007E016980999C86316980999C1F8980041
:10CCF000FFE709990320086309994DF24950C0F6EE
:10CD0000000048650998806509984CF6D961C0F61D
:10CD10000001F3F7C7FBEFF31080109010980B9011
:10CD200072B60B980590099945F24420C5F2484027
:10CD3000086040F2E420C2F20000006868B9FFE732
:10CD4000099840F2E821C2F2000108600998C0F891
:10CD500088000998C0F88C001AE040F2E820C2F27E
:10CD60000000006804900498D0F88C0003900998A3
:10CD70000499C1F88C0009980399C1F888000398B8
:10CD80000999C1F88C0004980999C1F88800FFE757
:10CD900040F2E421C2F2000108680130086040F26C
:10CDA000FC21C2F2000108680130086019980128CE
:10CDB00032D1FFE740F20400C2F200000068EFF356
:10CDC00005810C910C990843B0F1F03F11D3FFE7B6
:10CDD00040F2F020C2F2000000680290029838B1E0
:10CDE000FFE70298C06B01900299C86AC863FFE729
:10CDF00002E000200290FFE705980F900F9880F363
:10CE00001088099800F0EAF8029820B1FFE701982D
:10CE10000299C863FFE71BE005980E900E9880F317
:10CE20001088EFF31080119011980A9072B60A984A
:10CE3000059040F2FC21C2F2000108680138086048
:10CE400005980D900D9880F3108800F08FF8FFE79B
:10CE5000002012B080BD000080B582B040F2EC210D
:10CE6000C2F2000100200190086040F2F021C2F2FD
:10CE70000001086040F28031C2F20001086040F217
:10CE8000F421C2F200012020086040F20030C2F21A
:10CE900000008021F3F769FC019840F2E821C2F21A
:10CEA0000001086040F2E421C2F20001086040F293
:10CEB000FC21C2F20001086040F2F821C2F2000138
:10CEC000086040F2B421C2F20001086840F08570A9
:10CED000086002B080BD000080B588B040F2EC2050
:10CEE000C2F20000006801900198416C806C884794
:10CEF00040F2F820C2F20000006840B1FFE740F2C3
:10CF0000F820C2F20000016801988847FFE7EFF3BC
:10CF1000108007900798039072B6039802900199C9
:10CF2000012008630199886301990020C86440F2D8
:10CF3000FC21C2F2000108680130086002980490E8
:10CF4000049880F31088EFF3148005900598009002
:10CF5000009820F00400009000980690069880F356
:10CF60001488019800F05EF908B080BD87B040F2E7
:10CF7000FC20C2F2000000680290029860BBFFE74C
:10CF800040F2EC20C2F200000068019040F2F02074
:10CF9000C2F20000006800900198009988421AD0FF
:10CFA000FFE74EF60451CEF200014FF080500860CA
:10CFB000EFF305800490049860B9FFE7EFF3108069
:10CFC00005900598039062B603980690069880F342
:10CFD0001088FFE7FFE7FFE707B0704780B596B01E
:10CFE0000990EFF31080139013980C9072B60C9880
:10CFF00008900998406E28B1FFE709984C3000F07E
:10D00000F5FB03E009990020C864FFE740F2FC212A
:10D01000C2F200010868013808600998806B002896
:10D0200040F0A880FFE70998006B002800F0A1807D
:10D03000FFE70998406B002840F09380FFE70999CB
:10D04000002008630998C06A0790079940F20030F1
:10D05000C2F2000050F821000590059800286FD119
:10D06000FFE70998079A40F20031C2F2000141F847
:10D0700022000998006209984062079901208840BF
:10D08000069040F28031C2F200010868069A10430F
:10D090000860079840F2F421C2F200010968884252
:10D0A0004DD2FFE7079840F2F421C2F20001086078
:10D0B00040F2F020C2F2000000680390039838B9F3
:10D0C000FFE7099840F2F021C2F20001086035E064
:10D0D00007980399C96B88422FD2FFE7099840F25D
:10D0E000F021C2F20001086008981090109880F3B7
:10D0F000108840F2FC20C2F2000000680190019804
:10D10000D0B9FFE74EF60451CEF200014FF0805047
:10D110000860EFF305801190119860B9FFE7EFF315
:10D120001080149014980B9062B60B980D900D9887
:10D1300080F31088FFE7FFE772E0FFE7FFE70FE00B
:10D140000598406A0490099804990862099805991D
:10D150004862049809994862059809990862FFE7AE
:10D1600006E0099900204863099903200863FFE756
:10D17000FFE71DE00998006B012818D0FFE7099828
:10D18000006B022812D0FFE70998406B30B9FFE727
:10D190000999002088630999086306E0099900202D
:10D1A0004863099903200863FFE7FFE7FFE7FFE70C
:10D1B00040F2EC20C2F200000068029008980F9044
:10D1C0000F9880F31088029840F2F021C2F200011B
:10D1D0000968884224D0FFE740F2FC20C2F2000038
:10D1E000006801900198D0B9FFE74EF60451CEF2E5
:10D1F00000014FF080500860EFF305801290129804
:10D2000060B9FFE7EFF31080159015980A9062B6A9
:10D210000A980E900E9880F31088FFE7FFE7FFE76B
:10D2200016B080BD80B59CB00A9040F2EC20C2F2EE
:10D23000000000680190EFF31080189018980E908D
:10D2400072B60E9809900A980199884218D1FFE7A2
:10D250000A98C06C0090009850B1FFE70098013028
:10D2600028B1FFE70A984C3000F056FAFFE7FFE7D5
:10D270000A98C06940F6E801C2F200010860FFE7C1
:10D2800040F2FC21C2F200010868013808600A98E7
:10D29000806B012840F0D180FFE70A990020886365
:10D2A0000A98C06A08900A98006A039003980A993D
:10D2B00088421ED0FFE70A98406A029002980399BC
:10D2C0004862039802990862089940F20030C2F25D
:10D2D000000050F821000A99884209D1FFE703981D
:10D2E000089A40F20031C2F2000141F82200FFE743
:10D2F00060E0089A40F20030C2F20000002140F8DD
:10D300002210089A01209040059040F28030C2F22D
:10D3100000000268059B9A4302600791006806902E
:10D320000698A8BBFFE740F2F421C2F200012020DA
:10D33000086040F2F021C2F2000100200860099864
:10D340001490149880F3108840F2FC20C2F2000080
:10D35000006804900498D0B9FFE74EF60451CEF26D
:10D3600000014FF080500860EFF30580159015988C
:10D3700060B9FFE7EFF31080199019980D9062B62D
:10D380000D980F900F9880F31088FFE7FFE787E074
:10D39000069890FAA0F006900698B0FA80F00590F2
:10D3A00007980599084440F2F421C2F20001086090
:10D3B000FFE7FFE70A9840F2F021C2F20001096896
:10D3C000884239D1FFE740F2F420C2F20000016840
:10D3D00040F20030C2F2000050F8210040F2F0218B
:10D3E000C2F20001086009981390139880F3108826
:10D3F00040F2FC20C2F20000006804900498D0B90A
:10D40000FFE74EF60451CEF200014FF08050086065
:10D41000EFF305801690169860B9FFE7EFF31080E0
:10D420001A901A980C9062B60C981090109880F38D
:10D430001088FFE7FFE733E0FFE7099812901298A2
:10D4400080F31088019840F2F021C2F200010968CF
:10D45000884224D0FFE740F2FC20C2F200000068BE
:10D4600004900498D0B9FFE74EF60451CEF20001C3
:10D470004FF080500860EFF305801790179860B95F
:10D48000FFE7EFF310801B901B980B9062B60B9890
:10D490001190119880F31088FFE7FFE7FFE7FFE79F
:10D4A0001CB080BD85B040F2EC20C2F200000068E4
:10D4B0000090EFF3108004900498029072B60298E6
:10D4C000019040F29831C2F20001002008600098FB
:10D4D00090B3FFE70098006B68BBFFE70099C8694D
:10D4E00088610098806940F6E801C2F20001086096
:10D4F0000099086A88421DD0FFE70099C86AC96B85
:10D50000884216D1FFE70098016AC26A40F20030F3
:10D51000C2F2000040F8221040F2F421C2F20001F1
:10D52000096850F8210040F2F021C2F200010860C1
:10D53000FFE7FFE7FFE7FFE701980390039880F319
:10D54000108805B07047000080B58AB00590059836
:10D550000390EFF3108009900998069072B6069830
:10D5600004900398006B042810D1FFE740F2FC21DF
:10D57000C2F2000108680130086004980890089819
:10D5800080F310880398FFF729FD14E00398806E5C
:10D5900002900398D0F8AC00019004980790079887
:10D5A00080F31088029828B1FFE7029A0398019946
:10D5B0009047FFE7FFE70AB080BD000080B584B068
:10D5C000EFF3108003900398019072B601980090D9
:10D5D00040F2FC21C2F200010868013008600098A6
:10D5E0000290029880F3108840F23840C2F20000A6
:10D5F000FFF7F4FC04B080BD80B58AB040F234413E
:10D60000C2F2000100200890086040F6E801C2F272
:10D610000001086040F29831C2F20001086040F257
:10D620009431C2F20001086040F29C31C2F2000164
:10D63000086040F2A030C2F2000007908021F3F7AA
:10D6400094F80799089840F22442C2F2000211604F
:10D6500040F29032C2F2000211607C3140F220426E
:10D66000C2F20002116011680431116040F23042D0
:10D67000C2F2000240F2E841C2F20001116040F241
:10D680002C42C2F200024FF48061116040F2284146
:10D69000C2F200010860FFE740F23040C2F2000031
:10D6A000006840F22C41C2F200010A6840F22841B1
:10D6B000C2F200010B6869464FF0000CC1F814C0BB
:10D6C000C1F810C0CB608B604A60086040F23840FF
:10D6D000C2F200004DF6D541C0F600014DF65D02E4
:10D6E000C0F6000244F64D13C4F25413FFF7A6FA35
:10D6F0000990FFE709980028CED1FFE740F28C316E
:10D70000C2F200010020086040F28831C2F200013C
:10D7100008600AB080BD000087B0069006980068D7
:10D720000190019800285FD0FFE7019801300028A0
:10D7300059D0FFE706988069002853D1FFE7019888
:10D74000212803D3FFE71F20009003E00198013850
:10D750000090FFE740F29030C2F2000000680099AC
:10D7600000EB81000590059840F22041C2F20001D3
:10D770000968884213D3FFE7059840F22041C2F2BE
:10D7800000010968401A8010029040F22440C2F261
:10D7900000000068029900EB81000590FFE7059802
:10D7A000006840B9FFE70698006106984061069856
:10D7B0000599086012E00598006804900498406993
:10D7C00003900698039908610698049948610498A3
:10D7D00006990861039806994861FFE7059806993C
:10D7E0008861FFE7FFE7FFE707B0704784B0039069
:10D7F000039880690290029870B3FFE7039800696C
:10D8000001900398019988420BD1FFE702980068C4
:10D810000399884204D1FFE7029900200860FFE7DE
:10D8200016E00398406900900098019948610198BA
:10D8300000990861029800680399884207D1FFE7C0
:10D84000029801998861019802990860FFE7FFE753
:10D85000039900208861FFE704B0704780B598B055
:10D860000A90002002900A9844F64D11C4F2541117
:10D87000884240F0FD80FFE7FFE7EFF3108014904F
:10D8800014980E9072B60E98099040F29030C2F241
:10D890000000006800680890089820B1FFE7089928
:10D8A00008A88861FFE740F29030C2F200000268E9
:10D8B00000211160016804310160006840F22041DC
:10D8C000C2F20001096888420BD1FFE740F2244010
:10D8D000C2F20000006840F29031C2F2000108601C
:10D8E000FFE740F29431C2F200010020086009987D
:10D8F0001390139880F31088EFF31080159015980B
:10D900000D9072B60D980990FFE70898002800F076
:10D910008680FFE708980490089800690690002028
:10D92000079004980699884203D1FFE700200890E9
:10D930000EE004984069059005980699486106989C
:10D9400005990861069908A8886106980890FFE77C
:10D950000498006821280ED3FFE70499086820384E
:10D96000086000200390049907A88861049800616A
:10D970000498079019E00498806803900498C068A0
:10D9800002900499486808600498006840B1FFE775
:10D99000049907A88861049800610498079003E03F
:10D9A000049900208861FFE7FFE7049840F29C316A
:10D9B000C2F20001086009981290129880F3108852
:10D9C000039820B1FFE7039902988847FFE7EFF338
:10D9D0001080169016980C9072B60C98099040F230
:10D9E0009C31C2F200010020086007980499884227
:10D9F00007D1FFE70499002088610498FFF78CFEA7
:10DA0000FFE709981190119880F31088EFF31080C8
:10DA1000179017980B9072B60B98099075E740F223
:10DA20009430C2F200000068D8B9FFE740F23840F5
:10DA3000C2F20000019001990320086301990120BE
:10DA4000886340F2FC21C2F20001086801300860DE
:10DA500009981090109880F310880198FFF7E2FB66
:10DA600005E009980F900F9880F31088FFE704E70E
:10DA700018B080BD80B592B0DDF850C00990089113
:10DA80000792069300200490099818B9FFE7022036
:10DA900004909BE01498342803D0FFE70220049000
:10DAA00093E0EFF31080109010980B9072B60B98E3
:10DAB000059040F2FC21C2F20001086801300860C4
:10DAC00005980D900D9880F3108840F2BC20C2F2AA
:10DAD00000000068029000200390FFE7039840F2E6
:10DAE000B821C2F20001096888420FD2FFE7099805
:10DAF0000299884201D1FFE708E00298C06A0290CB
:10DB0000FFE7FFE7039801300390E7E7EFF31080AA
:10DB1000119011980A9072B60A98059040F2FC2173
:10DB2000C2F2000108680138086005980C900C9852
:10DB300080F31088FFF71AFA09980299884203D1F6
:10DB4000FFE7022004903FE0079818B9FFE70320A1
:10DB5000049038E00698632803D8FFE70520049076
:10DB600030E040F2EC20C2F2000000680190019821
:10DB700040F23841C2F20001884203D1FFE713208E
:10DB80000490FFE740F20400C2F200000068EFF3E7
:10DB900005810F910F99084398B1FFE740F2040007
:10DBA000C2F200000068EFF305810E910E99084360
:10DBB0000009B0F10F3F03D2FFE713200490FFE705
:10DBC000FFE7FFE7FFE7FFE7FFE7FFE7049840B95C
:10DBD000FFE709980899079A069BFEF71FFF049034
:10DBE000FFE7049812B080BD80B582B0002001909C
:10DBF000F5F7F6F9FCF72AFFFCF7BEFCFCF78CFC06
:10DC0000FCF7EEFCFCF734FDFCF7E6FCFFE7FEE773
:10DC100080B584B0039000200290694634200860EB
:10DC200040F6D440C2F200004DF6C241C0F60001F9
:10DC300040F60852C2F200024FF48063FFF71AFF69
:10DC400008B1FFE70EE040F6D440C2F200000190B8
:10DC50000198F2F721FE0290029810B1FFE7FFE76A
:10DC6000FEE7FFE704B080BDF1EE100A4FF6FF714A
:10DC7000C0F2C03120EA010040F04070E1EE100A2D
:10DC800070470000000000000000010203040607C6
:10DC9000080900000000010203040804020408014E
:10DCA000010101010103070100000100020004005D
:10DCB000060008000A000C00100020004000800050
:10DCC0000001547820417070206D656D6F7279206D
:10DCD000706F6F6C0053797374656D2054696D6556
:10DCE00072205468726561640000000010DD000855
:10DCF0000000002010000000B002000820DD000835
:10DD00001000002040170000D002000800000000B2
:10DD10000090D003F0F0F0F00100000010000000CF
:040000050800024DA0
:00000001FF
